:020000040800F2
:1000000000060020E1010008E3010008E301000808
:10001000E3010008E3010008E3010008E301000830
:10002000E3010008E3010008E301000809300008CB
:10003000E3010008E3010008E3010008E301000810
:10004000E3010008E3010008E3010008E301000800
:10005000E3010008E3010008B1320008D9320008CA
:10006000013300082933000851330008E301000878
:10007000E3010008E3010008E3010008E3010008D0
:10008000E3010008E3010008E3010008E3010008C0
:10009000E3010008E3010008E301000879330008E8
:1000A000E3010008E3010008E3010008E3010008A0
:1000B0004D340008E3010008E3010008E3010008F3
:1000C000E3010008E3010008E3010008E301000880
:1000D000E3010008E3010008E3010008E301000870
:1000E000DD330008E3010008E3010008E301000834
:1000F000E3010008E3010008E3010008E301000850
:10010000E3010008E3010008E3010008E30100083F
:10011000E3010008E3010008E3010008E30100082F
:10012000E3010008E3010008E3010008E30100081F
:10013000E3010008E3010008E3010008E30100080F
:10014000E3010008E3010008E3010008BD270008FF
:10015000E3010008E3010008E3010008E3010008EF
:10016000E3010008E3010008E3010008E3010008DF
:10017000E3010008E3010008E3010008E3010008CF
:10018000E3010008E3010008E3010008E3010008BF
:10019000E3010008E3010008E3010008E3010008AF
:1001A000E3010008E3010008E3010008E30100089F
:1001B000E3010008E3010008E3010008E30100088F
:1001C000E3010008E3010008E3010008E30100087F
:1001D000E3010008E3010008E3010008E30100086F
:1001E00002E000F000F8FEE772B6384880F30888B5
:1001F000374880F3098837483749086040F20000E3
:10020000CCF200004EF63471CEF200010860BFF36C
:100210004F8FBFF36F8F40F20000C0F2F0004EF638
:100220008851CEF200010860BFF34F8FBFF36F8F8C
:100230004FF00000E1EE100A4EF63C71CEF20001E4
:100240000860062080F31488BFF36F8F01F09EFFD3
:1002500001F07AFF02F076FE4FF055301F491B4A3D
:1002600091423CBF41F8040BFAE71D49184A9142FC
:100270003CBF41F8040BFAE71A491B4A1B4B9A4250
:100280003EBF51F8040B42F8040BF8E70020184970
:10029000184A91423CBF41F8040BFAE701F058FFBD
:1002A00002F0A4FE144C154DAC4203DA54F8041BC2
:1002B0008847F9E700F042F8114C124DAC4203DADE
:1002C00054F8041B8847F9E701F040BF00060020FE
:1002D000002200200000000808ED00E000000020DF
:1002E00000060020283800080022002040220020BC
:1002F00040220020602E0020E0010008E0010008FC
:10030000E0010008E00100082DE9F04F2DED108A12
:10031000C1F80CD0C3689D46BDEC108ABDE8F08FD3
:10032000002383F311882846A047002001F0A8FA93
:10033000FEE701F011FA00DFFEE7000038B501F03A
:10034000D3FE054601F0F6FE0446D8B90F4B9D4298
:100350001AD001339D4218BF044641F2883504BFCC
:1003600001240025002001F0C9FE0CB100F076F850
:1003700000F012FD00F0A4FB284600F0C3F800F0E6
:100380006DF8F9E70025EDE70546EBE7010007B05A
:1003900008B500F067FBA0F120035842584108BDA2
:1003A00007B541F21203022101A8ADF8043000F0B4
:1003B00077FB03B05DF804FB38B5302383F3118875
:1003C000174803680BB101F027FB164A14480023B5
:1003D0004FF47A7101F016FB002383F31188124C5D
:1003E000236813B12368013B2360636813B163681A
:1003F000013B63600D4D2B7833B963687BB90220F4
:1004000000F03CFC322363602B78032B07D1636838
:100410002BB9022000F032FC4FF47A73636038BDD0
:1004200040220020B9030008602300205822002049
:10043000084B187003280CD8DFE800F00805020804
:10044000022000F00BBC022000F0F8BB024B00229F
:100450005A6070475822002060230020244B254A10
:1004600010B51C461968013140D004339342F9D1CC
:100470006268214B9A4239D9204B9B6803F1006393
:1004800003F580339A4231D2002000F033FB022082
:10049000FFF7CEFF1A4B1A6C00221A64196E1A6607
:1004A000196E596C5A64596E5A665A6E5A6942F0FE
:1004B00080025A615A6922F080025A615A691A69A7
:1004C00042F000521A611A6922F000521A611B6947
:1004D00072B64FF0E0233021C3F8084DD4E9003262
:1004E00081F311889D4683F30888104710BD00BF33
:1004F0000000010820000108FFFF00080022002082
:10050000003802402DE9F04F93B0AA4B0090202212
:10051000FF210AA89D6800F0E9FBA74A1378A3B958
:10052000A648012103601170302383F3118803680A
:100530000BB101F071FAA24AA04800234FF47A717E
:1005400001F060FA002383F31188009B13B19D4BE7
:10055000009A1A609C4A009C1378032B1EBF00234C
:100560001370984A4FF0000A18BF5360D34656469E
:10057000D146012000F072FB24B1924B1B68002B86
:1005800000F01182002000F06DFA0390039B002B15
:10059000F2DB012000F052FB039B213B162BE8D835
:1005A00001A252F823F000BF050600082D0600083E
:1005B000C1060008730500087305000873050008EC
:1005C0004B0700081B0900083508000897080008B9
:1005D000BF080008E508000873050008F7080008D0
:1005E0007305000869090008A506000873050008DE
:1005F000AD09000811060008A506000873050008EB
:10060000970800080220FFF7C3FE002840F0F5819C
:10061000009B0221BAF1000F08BF1C4605A841F259
:100620001233ADF8143000F03BFAA2E74FF47A70C1
:1006300000F018FA071EEBDB0220FFF7A9FE0028E6
:10064000E6D0013F052F00F2DA81DFE807F0030A68
:100650000D10133605230593042105A800F020FA98
:1006600017E054480421F9E758480421F6E75848B0
:100670000421F3E74FF01C08404600F03DFA08F172
:1006800004080590042105A800F00AFAB8F12C0F1F
:10069000F2D1012000FA07F747EA0B0B5FFA8BFB58
:1006A0004FF0000900F06EFB26B10BF00B030B2B93
:1006B00008BF0024FFF774FE5BE746480421CDE73E
:1006C000002EA5D00BF00B030B2BA1D10220FFF7BE
:1006D0005FFE074600289BD0012000F00BFA0220A5
:1006E000FFF7A6FE00265FFA86F8404600F012FAF1
:1006F000044690B10021404600F01CFA0136002863
:10070000F1D1BA46044641F21213022105A8ADF810
:1007100014303E4600F0C4F92BE70120FFF788FEB5
:100720002546244B9B68AB4207D9284600F0E4F9E4
:10073000013040F067810435F3E7234B00251D703D
:10074000204BBA465D603E46ACE7002E3FF460AFFA
:100750000BF00B030B2B7FF45BAF0220FFF768FE5F
:10076000322000F07FF9B0F10008FFF651AF18F029
:1007700003077FF44DAF0F4A926808EB05039342DD
:100780003FF646AFB8F5807F3FF742AF124B01937B
:10079000B84523DD4FF47A7000F064F90390039AB2
:1007A000002AFFF635AF019B039A03F8012B0137AE
:1007B000EDE700BF002200205C2300204022002043
:1007C000B9030008602300205822002004220020E2
:1007D000082200200C2200205C220020C820FFF705
:1007E000D7FD074600283FF413AF1F2D11D8C5F1E0
:1007F000200242450AAB25F0030028BF4246834948
:100800000192184400F04CFA019A8048FF2100F050
:100810006DFA4FEAA8037D490193C8F38702284681
:1008200000F06CFA064600283FF46DAF019B05EB23
:10083000830537E70220FFF7ABFD00283FF4E8AE61
:1008400000F0A4F900283FF4E3AE0027B846704B4F
:100850009B68BB4218D91F2F11D80A9B01330ED0B9
:1008600027F0030312AA134453F8203C0593404693
:10087000042205A900F0BAFA04378046E7E73846B3
:1008800000F03AF90590F2E7CDF81480042105A8AC
:1008900000F006F906E70023642104A8049300F0A1
:1008A000F5F800287FF4B4AE0220FFF771FD0028B0
:1008B0003FF4AEAE049800F051F90590E6E700234E
:1008C000642104A8049300F0E1F800287FF4A0AEAE
:1008D0000220FFF75DFD00283FF49AAE049800F077
:1008E0004DF9EAE70220FFF753FD00283FF490AEF0
:1008F00000F05CF9E1E70220FFF74AFD00283FF431
:1009000087AE05A9142000F057F90421074604908A
:1009100004A800F0C5F83946B9E7322000F0A2F883
:10092000071EFFF675AEBB077FF472AE384A9268B9
:1009300007EB090393423FF66BAE0220FFF728FD59
:1009400000283FF465AE27F003074F44B9453FF454
:10095000A9AE484600F0D0F80421059005A800F0A3
:100960009FF809F10409F1E74FF47A70FFF710FDE1
:1009700000283FF44DAE00F009F9002844D00A9B4E
:1009800001330BD008220AA9002000F0B7F9002893
:100990003AD02022FF210AA800F0A8F9FFF700FDB5
:1009A0001C4800F073FF13B0BDE8F08F002E3FF439
:1009B0002FAE0BF00B030B2B7FF42AAE0023642128
:1009C00005A8059300F062F8074600287FF420AEE2
:1009D0000220FFF7DDFC804600283FF419AEFFF748
:1009E000DFFC41F2883000F051FF059800F0FCF97F
:1009F000464600F0C7F93C46BBE5064652E64FF0D6
:100A0000000905E6BA467EE637467CE65C22002011
:100A100000220020A086010070B50F4B1B78013327
:100A2000DBB2012B0C4611D80C4D29684FF47A73B8
:100A30000E6AA2FB0332014622462846B047844292
:100A400004D1074B00221A70012070BD4FF4FA70D8
:100A500000F01CFF0020F8E71022002008260020EC
:100A60009423002007B50023024601210DF1070061
:100A70008DF80730FFF7D0FF20B19DF8070003B0D5
:100A80005DF804FB4FF0FF30F9E700000A4608B5B7
:100A90000421FFF7C1FF80F00100C0B2404208BD51
:100AA00030B4054C2368DD69044B0A46AC46014668
:100AB000204630BC604700BF08260020A086010009
:100AC00070B501F003FA094E094D30800024286802
:100AD0003388834208D901F0F3F92B6804440133C9
:100AE000B4F5803F2B60F2D370BD00BF9623002089
:100AF0006823002001F0ACBA00F1006000F58030FE
:100B00000068704700F10060920000F5803001F04D
:100B10002BBA0000054B1A68054B1B889B1A8342B1
:100B200002D9104401F0CCB900207047682300209E
:100B30009623002038B5084D044629B12868204482
:100B4000BDE8384001F0DCB92868204401F0C0F964
:100B50000028F3D038BD00BF6823002010F0030345
:100B60000AD1B0F5047F05D200F10050A0F5104085
:100B7000D0F80038184670470023FBE700F100501A
:100B8000A0F51040D0F8100A70470000064991F80F
:100B9000243033B10023086A81F824300822FFF79B
:100BA000B1BF0120704700BF6C230020014B1868C3
:100BB000704700BF002004E0F0B51C4B02461868E7
:100BC0001B4BC0F30B050424000C1E88AE421BD146
:100BD0005C6893F90850174B05261F88874208BFA9
:100BE00093F90250013E03F10403F6D1013A0A449D
:100BF000013C0B4693420ED214F9016F581C66B1AA
:100C000000F8016C0346F5E7013C03F10C03DCD16D
:100C1000094C3F25DFE7184605E02C2490421C7064
:100C200001D2981C5D70401AF0BD00BF002004E0A6
:100C3000303500081C350008F0340008022804D1C3
:100C4000054B4FF080429A6170470128FCD1024B5E
:100C50004FF00052F7E700BF00000240022804D125
:100C6000054B4FF480429A6170470128FCD1024B3A
:100C70004FF40052F7E700BF00000240022805D100
:100C8000064A536983F48043536170470128FCD1BD
:100C9000024A536983F40053F6E700BF00000240A4
:100CA00010B50023934203D0CC5CC4540133F9E760
:100CB00010BD000010B5013810F9013F3BB191F9AA
:100CC00000409C4203D11AB10131013AF4E71AB154
:100CD00091F90020981A10BD1046FCE70346024621
:100CE000D01A12F9011B0029FAD1704702440346B9
:100CF000934202D003F8011BFAE770472DE9F8434D
:100D00001F4D144695F824200746884652BBDFF84D
:100D100070909CB395F824302BB92022FF214846CF
:100D20002F62FFF7E3FF95F82400C0F10802A2420A
:100D300028BF2246D6B24146920005EB8000FFF75D
:100D4000AFFF95F82430A41B1E44F6B2082E1744BA
:100D50009044E4B285F82460DBD1FFF717FF002848
:100D6000D7D108E02B6A03EB82038342CFD0FFF791
:100D70000DFF0028CBD10020BDE8F8830120FBE760
:100D80006C230020024B1A78024B1A70704700BF88
:100D9000942300201022002010B50F4C0F4800F0C3
:100DA000B5F821460D4800F0DDF824680C48626D66
:100DB000D2F8043843F00203C2F8043800F066FDAC
:100DC0000849204600F0D4F9626DD2F8043823F0C7
:100DD0000203C2F8043810BD0C36000808260020B3
:100DE00040420F00143600087047000030B5094D2E
:100DF0000A4491420DD011F8013B5840082340F3BA
:100E00000004013B2C4013F0FF0384EA5000F6D1AC
:100E1000EFE730BD2083B8ED0268436811430160FD
:100E200003B118477047000013B5446BD4F89434ED
:100E30001A681178042915D1217C022912D1197957
:100E4000128901238B4013420CD101A904F14C00FB
:100E500001F034FFD4F89444019B217902462068C4
:100E600000F0D0F902B010BD143001F0B7BE0000A0
:100E70004FF0FF33143001F0B1BE00004C3001F0F0
:100E800089BF00004FF0FF334C3001F083BF0000FA
:100E9000143001F085BE00004FF0FF31143001F036
:100EA0007FBE00004C3001F055BF00004FF0FF3214
:100EB0004C3001F04FBF00000020704710B5D0F853
:100EC00094341A6811780429044617D1017C022948
:100ED00014D15979528901238B4013420ED1143019
:100EE00001F018FE024648B1D4F894444FF48073E0
:100EF00061792068BDE8104000F072B910BD0000B3
:100F0000406BFFF7DBBF0000704700007FB5124B5E
:100F1000036000234360C0E90233012502260F4B22
:100F2000057404460290019300F18402294600965C
:100F30004FF48073143001F0C9FD094B0294CDE9E0
:100F4000006304F523724FF48073294604F14C00CA
:100F500001F090FE04B070BD60350008010F00087C
:100F6000290E00080B68302282F311880A7903EBFE
:100F7000820290614A79093243F822008A7912B1DB
:100F800003EB820398610223C0F8941403740020D9
:100F900080F311887047000038B5037F044613B111
:100FA00090F85430ABB9201D01250221FFF734FF22
:100FB00004F1140025776FF0010100F08FFC84F834
:100FC000545004F14C006FF00101BDE8384000F0CE
:100FD00085BC38BD10B5012104460430FFF71CFF65
:100FE0000023237784F8543010BD000038B5044640
:100FF0000025143001F082FD04F14C00257701F04A
:1010000051FE201D84F854500121FFF705FF2046B2
:10101000BDE83840FFF752BF90F8443003F060035A
:10102000202B07D190F84520212A4FF0000303D848
:101030001F2A06D800207047222AFBD1C0E90E33B0
:1010400003E0034A82630722C263036401207047FE
:101050001122002037B5D0F894341A681178042989
:1010600004461AD1017C022917D11979128901236A
:101070008B40134211D100F14C05284601F0D2FEFD
:1010800058B101A9284601F019FED4F89444019BF7
:1010900021790246206800F0B5F803B030BD0000A9
:1010A000F0B500EB810385B09E6904460D46FEB1A4
:1010B000302383F3118804EB8507301D0821FFF7E7
:1010C000ABFEFB685B691B6806F14C001BB101902D
:1010D00001F002FE019803A901F0F0FD024648B1BB
:1010E000039B2946204600F08DF8002383F31188E6
:1010F00005B0F0BDFB685A691268002AF5D01B8A5A
:10110000013B1340F1D104F14402EAE7093138B55B
:1011100050F82140DCB1302383F31188D4F89424B3
:101120001368527903EB8203DB689B695D6845B104
:1011300004216018FFF770FE294604F1140001F045
:10114000F3FC2046FFF7BAFE002383F3118838BD75
:101150007047000001F052B8012303700023C0E97A
:101160000133C36183620362C362436203637047F6
:1011700038B50446302383F311880025C0E90355B0
:10118000C0E90555416001F049F80223237085F359
:101190001188284638BD000070B500EB8103054674
:1011A0005069DA600E46144618B110220021FFF78C
:1011B0009DFDA06918B110220021FFF797FD31466F
:1011C0002846BDE8704001F0F3B80000826802F0E4
:1011D000011282600022C0E90422826101F074B928
:1011E000F0B400EB81044789E4680125A4698D40CF
:1011F0003D43458123600023A2606360F0BC01F0A1
:101200008FB90000F0B400EB81040789E468012580
:1012100064698D403D43058123600023A2606360C3
:10122000F0BC01F009BA000070B5022300250446A5
:101230000370C0E90255C0E90455C564856180F8B2
:10124000345001F051F863681B6823B129462046E9
:10125000BDE87040184770BD0378052B10B50446F3
:101260000AD080F850300523037043681B680BB127
:10127000042198470023A36010BD000001780529D0
:1012800006D190F85020436802701B6803B11847DC
:101290007047000070B590F83430044613B1002355
:1012A00080F8343004F14402204601F02FF96368DD
:1012B0009B68B3B994F8443013F0600535D0002131
:1012C000204601F0CFFB0021204601F0C1FB6368FE
:1012D0001B6813B1062120469847062384F8343052
:1012E00070BD204698470028E4D0B4F84A30E26B3D
:1012F0009A4288BFE36394F94430E56B002B4FF0CA
:10130000300380F20381002D00F0F280092284F87E
:10131000342083F311880021D4E90E232046FFF7FF
:1013200071FF002383F31188DAE794F8452003F076
:101330007F0343EA022340F20232934200F0C58069
:1013400021D8B3F5807F48D00DD8012B3FD0022B98
:1013500000F09380002BB2D104F14C02A263022270
:10136000E2632364C1E7B3F5817F00F09B80B3F5AE
:10137000407FA4D194F84630012BA0D1B4F84C3072
:1013800043F0020332E0B3F5006F4DD017D8B3F548
:10139000A06F31D0A3F5C063012B90D8636894F897
:1013A00046205E6894F84710B4F848302046B047AD
:1013B000002884D04368A3630368E3631AE0B3F5AD
:1013C000106F36D040F6024293427FF478AF5C4B08
:1013D000A3630223E3630023C3E794F84630012BA1
:1013E0007FF46DAFB4F84C3023F00203C4E90E551E
:1013F000A4F84C30256478E7B4F84430B3F5A06F16
:101400000ED194F8463084F84E30204600F0C4FFE8
:1014100063681B6813B1012120469847032323709A
:101420000023C4E90E339CE704F14F03A3630123B7
:10143000C3E72378042B10D1302383F3118820468F
:10144000FFF7C4FE85F311880321636884F84F50C9
:1014500021701B680BB12046984794F84630002B4A
:10146000DED084F84F300423237063681B68002BA0
:10147000D6D0022120469847D2E794F848301D067E
:1014800003F00F0120460AD501F032F8012804D0FC
:1014900002287FF414AF2B4B9AE72B4B98E701F00F
:1014A00019F8F3E794F84630002B7FF408AF94F86E
:1014B000483013F00F01B3D01A06204602D501F0D0
:1014C000E5FAADE701F0D8FAAAE794F84630002B28
:1014D0007FF4F5AE94F8483013F00F01A0D01B064E
:1014E000204602D501F0BEFA9AE701F0B1FA97E77B
:1014F000142284F8342083F311882B462A46294687
:101500002046FFF76DFE85F31188E9E65DB11522EF
:1015100084F8342083F311880021D4E90E23204677
:10152000FFF75EFEFDE60B2284F8342083F311887A
:101530002B462A4629462046FFF764FEE3E700BF14
:1015400090350008883500088C35000838B590F8CB
:1015500034300446002B3ED0063BDAB20F2A34D892
:101560000F2B32D8DFE803F0373131082232313126
:101570003131313131313737C56BB0F84A309D42A6
:1015800014D2C3681B8AB5FBF3F203FB12556DB985
:10159000302383F311882B462A462946FFF732FE73
:1015A00085F311880A2384F834300EE0142384F87C
:1015B0003430302383F3118800231A46194620461D
:1015C000FFF70EFE002383F3118838BD036C03B1CF
:1015D00098470023E7E70021204601F043FA002165
:1015E000204601F035FA63681B6813B106212046D6
:1015F00098470623D7E7000010B590F83430142B35
:10160000044629D017D8062B05D001D81BB110BD30
:10161000093B022BFBD80021204601F023FA0021D0
:10162000204601F015FA63681B6813B106212046B5
:101630009847062319E0152BE9D10B2380F83430A5
:10164000302383F3118800231A461946FFF7DAFD89
:10165000002383F31188DAE7C3689B695B68002B7A
:10166000D5D1036C03B19847002384F83430CEE71A
:1016700000230375826803691B6899689142FBD255
:101680005A68036042601060586070470023037519
:10169000826803691B6899689142FBD85A680360A5
:1016A000426010605860704708B50846302383F3E5
:1016B00011880B7D032B05D0042B0DD02BB983F3A0
:1016C000118808BD8B6900221A604FF0FF338361D7
:1016D000FFF7CEFF0023F2E7D1E9003213605A6032
:1016E000F3E70000FFF7C4BF054BD9680875186819
:1016F00002681A60536001220275D860FEF704BECA
:101700009823002030B50C4BDD684B1C87B0044695
:101710000FD02B46094A684600F074F92046FFF7BF
:10172000E3FF009B13B1684600F076F9A86907B0A3
:1017300030BDFFF7D9FFF9E798230020A91600086C
:10174000044B1A68DB6890689B68984294BF00203D
:101750000120704798230020084B10B51C68D868FA
:1017600022681A60536001222275DC60FFF78EFF49
:1017700001462046BDE81040FEF7C6BD9823002074
:10178000044B1A68DB6892689B689A4201D9FFF79C
:10179000E3BF70479823002038B5074C0749084835
:1017A000012300252370656001F074FB0223237080
:1017B00085F3118838BD00BF002600209835000849
:1017C0009823002000F05EB9EFF3118020B9EFF309
:1017D0000583302282F311887047000010B530B9BC
:1017E000EFF30584C4F3080414B180F3118810BD2D
:1017F000FFF7C6FF84F31188F9E70000034A516838
:1018000053685B1A9842FBD8704700BF001000E095
:101810008B60022308618B82084670478368A3F1BE
:10182000840243F8142C026943F8442C426943F8BB
:10183000402C094A43F8242CC26843F8182C022291
:1018400003F80C2C002203F80B2C044A43F8102C4C
:10185000A3F12000704700BF210300089823002057
:1018600008B5FFF7DBFFBDE80840FFF73BBF00000E
:10187000024BDB6898610F20FFF736BF98230020EA
:10188000302383F31188FFF7F3BF000008B501464A
:10189000302383F311880820FFF734FF002383F3FC
:1018A000118808BD064BDB6839B1426818605A6080
:1018B000136043600420FFF725BF4FF0FF307047EF
:1018C000982300200368984206D01A68026050608E
:1018D00099611846FFF706BF7047000038B5044607
:1018E0000D462068844200D138BD036823605C60E7
:1018F0008561FFF7F7FEF4E710B503689C68A24224
:101900000CD85C688A600B604C60216059609968F3
:101910008A1A9A604FF0FF33836010BD1B68121B58
:10192000ECE700000A2938BF0A2170B504460D46CD
:101930000A26601901F0A8FA01F094FA041BA542E6
:1019400003D8751C2E460446F3E70A2E04D9BDE8D9
:101950007040012001F0DEBA70BD0000F8B5144BF4
:101960000D46D96103F1100141600A2A19698260AC
:1019700038BF0A22016048601861A818144601F0B7
:1019800075FA0A2701F06EFA431BA342064606D3F6
:101990007C1C281901F078FA27463546F2E70A2F11
:1019A00004D9BDE8F840012001F0B4BAF8BD00BF89
:1019B00098230020F8B506460D4601F053FA0F4A69
:1019C000134653F8107F9F4206D12A4601463046FF
:1019D000BDE8F840FFF7C2BFD169BB68441A2C19B3
:1019E00028BF2C46A34202D92946FFF79BFF224677
:1019F00031460348BDE8F840FFF77EBF982300203A
:101A0000A823002010B4C0E9032300235DF8044B91
:101A10004361FFF7CFBF000010B5194C236998420E
:101A20000DD0D0E90032816813605A609A680A4488
:101A30009A60002303604FF0FF33A36110BD23467B
:101A4000026843F8102F53600022026022699A4214
:101A500003D1BDE8104001F011BA936881680B44CE
:101A6000936001F0FFF92269E1699268441AA24289
:101A7000E4D91144BDE81040091AFFF753BF00BF75
:101A8000982300202DE9F047DFF8BC8008F110070B
:101A90002C4ED8F8105001F0E5F9D8F81C40AA688F
:101AA000031B9A423ED81444D5E900324FF0000996
:101AB000C8F81C4013605A60C5F80090D8F8103080
:101AC000B34201D101F0DAF989F31188D5E9033184
:101AD00028469847302383F311886B69002BD8D0B0
:101AE00001F0C0F96A69A0EB04094A4582460DD2AB
:101AF000022001F00FFA0022D8F81030B34208D1CA
:101B000051462846BDE8F047FFF728BF121A224485
:101B1000F2E712EB090938BF4A4629463846FFF773
:101B2000EBFEB5E7D8F81030B34208D01444211AC0
:101B3000C8F81C00A960BDE8F047FFF7F3BEBDE898
:101B4000F08700BFA82300209823002000207047C2
:101B5000FEE70000704700004FF0FF3070470000C4
:101B600002290CD0032904D00129074818BF0020FE
:101B70007047032A05D8054800EBC20070470448A7
:101B800070470020704700BF7036000820220020F8
:101B90002436000870B59AB00546084601A91446D7
:101BA00000F0C2F801A8FFF799F8431C5B00C5E9F3
:101BB00000340022237003236370C6B201AB0234E9
:101BC0001046D1B28E4204F1020401D81AB070BDA1
:101BD00013F8011B04F8021C04F8010C0132F0E7B1
:101BE00008B5302383F311880348FFF733FA002345
:101BF00083F3118808BD00BF0826002090F8443008
:101C000003F01F02012A07D190F845200B2A03D1C7
:101C10000023C0E90E3315E003F06003202B08D148
:101C2000B0F848302BB990F84520212A03D81F2A54
:101C300004D8FFF7F1B9222AEBD0FAE7034A82630E
:101C40000722C26303640120704700BF18220020EE
:101C500007B5052917D8DFE801F01916031919206F
:101C6000302383F31188104A01900121FFF794FA81
:101C700001980E4A0221FFF78FFA0D48FFF7B6F9D7
:101C8000002383F3118803B05DF804FB302383F352
:101C900011880748FFF780F9F2E7302383F31188B2
:101CA0000348FFF797F9EBE7C4350008E83500086B
:101CB0000826002038B50C4D0C4C0D492A4604F17D
:101CC0000800FFF767FF05F1CA0204F11000094997
:101CD000FFF760FF05F5CA7204F118000649BDE878
:101CE0003840FFF757BF00BFD02A00202022002035
:101CF000A4350008AE350008B935000870B50446B3
:101D000008460D46FEF7EAFFC6B2204601340378C6
:101D10000BB9184670BD32462946FEF7CBFF0028A6
:101D2000F3D10120F6E700002DE9F04705460C4607
:101D3000FEF7D4FF2B49C6B22846FFF7DFFF08B1F4
:101D40000A36F6B228492846FFF7D8FF08B1103600
:101D5000F6B2632E0BD8DFF88C80DFF88C90234F1F
:101D6000DFF894A02E7846B92670BDE8F0872946A2
:101D70002046BDE8F04701F0B3BB252E2ED1072247
:101D800041462846FEF796FF70B9194B224603F1EB
:101D9000100153F8040B42F8040B8B42F9D11B7865
:101DA000137007351134DDE7082249462846FEF74F
:101DB00081FF98B90F4BA21C197809090232C95D3D
:101DC00002F8041C13F8011B01F00F015345C95D13
:101DD00002F8031CF0D118340835C3E704F8016B8E
:101DE0000135BFE790360008B9350008AA3600086B
:101DF00098360008107AFF1F1C7AFF1FBFF34F8F21
:101E0000024AD368DB03FCD4704700BF003C0240A9
:101E100008B5094B1B7873B9FFF7F0FF074B1A6938
:101E2000002ABFBF064A5A6002F188325A601A6817
:101E300022F480621A6008BD2E2D0020003C024072
:101E40002301674508B50B4B1B7893B9FFF7D6FF05
:101E5000094B1A6942F000421A611A6842F4805232
:101E60001A601A6822F480521A601A6842F480627A
:101E70001A6008BD2E2D0020003C02400B28F0B552
:101E800016D80C4C0C4923787BB90C4D0E460C230C
:101E90004FF0006255F8047B46F8042B013B13F029
:101EA000FF033A44F6D10123237051F82000F0BD1E
:101EB0000020FCE7602D0020302D0020BC360008FB
:101EC000014B53F820007047BC3600080C207047C7
:101ED0000B2810B5044601D9002010BDFFF7CEFF36
:101EE000064B53F824301844C21A0BB90120F4E70A
:101EF00012680132F0D1043BF6E700BFBC3600089F
:101F00000B2838B5044628D8FFF75EFCFFF776FFAC
:101F1000FFF77EFF124AF323D360E300DBB243F402
:101F2000007343F002031361136943F480331361B8
:101F300005462046FFF762FFFFF7A0FF094B53F865
:101F4000241000F0E9F82846FFF77CFFFFF746FC75
:101F50002046BDE83840FFF7BBBF002038BD00BFBA
:101F6000003C0240BC36000812F001032DE9F041AC
:101F700005460E4614464BD18218B2F1016F61D866
:101F8000314B1B6813F001035CD0304FFFF71CFC92
:101F9000FFF73EFFF323FB60FFF730FF314640F2CF
:101FA0000128032C18D824F00104284E0C446D1A83
:101FB00040F20118A142336905EB01072AD123F051
:101FC00001033361FFF73EFFFFF708FC0120BDE886
:101FD000F081043C0435E4E7AB07E4D13B6923F42A
:101FE00040733B613B6943EA08033B6151F8046B72
:101FF0002E60BFF34F8FFFF701FF2B689E42E8D0A2
:102000003B6923F001033B61FFF71CFFFFF7E6FB91
:102010000020DCE723F440733361336943EA0803AB
:1020200033610B883B80BFF34F8FFFF7E7FE3F889C
:1020300031F8023BBFB2BB42BCD0336923F001038D
:102040003361E1E71846C2E700380240003C024035
:10205000084908B50B7828B11BB9FFF7D9FE012351
:102060000B7008BD002BFCD0BDE808400870FFF7DE
:10207000E9BE00BF2E2D002010B50244064BD2B29F
:10208000904200D110BD441C00B253F8200041F82A
:10209000040BE0B2F4E700BF502800400F4B30B50E
:1020A0001C6F240407D41C6F44F400741C671C6F5D
:1020B00044F400441C670A4C236843F48073236093
:1020C0000244084BD2B2904200D130BD441C00B251
:1020D00051F8045B43F82050E0B2F4E700380240C6
:1020E000007000405028004007B5012201A90020DF
:1020F000FFF7C2FF019803B05DF804FB13B5044677
:10210000FFF7F2FFA04205D0012201A900200194AF
:10211000FFF7C4FF02B010BD70470000034B1A6800
:102120001AB9034AD2F874281A607047642D002047
:102130000030024008B5FFF7F1FF024B1868C0F30A
:10214000407008BD642D002070470000FEE70000CD
:102150000A4B0B480B4A90420BD30B4BDA1C121A5A
:10216000C11E22F003028B4238BF00220021FEF77D
:10217000BDBD53F8041B40F8041BECE768380008A9
:10218000602E0020602E0020602E0020704700008E
:1021900070B5D0E915439E6800224FF0FF3504EB7F
:1021A00042135101D3F800090028BEBFD3F800093B
:1021B00040F08040C3F80009D3F8000B0028BEBFF0
:1021C000D3F8000B40F08040C3F8000B01326318D5
:1021D0009642C3F80859C3F8085BE0D24FF00113E8
:1021E000C4F81C3870BD0000890141F02001016174
:1021F00003699B06FCD41220FFF700BB10B5054C09
:102200002046FEF7A9FF4FF0A0436365024BA3658C
:1022100010BD00BF682D00201037000870B503788E
:10222000012B054650D12A4B446D98421BD1294BB6
:102230005A6B42F080025A635A6D42F080025A652E
:102240005A6D5A6942F080025A615A6922F080023E
:102250005A610E2143205B6900F022FC1E4BE360B3
:102260001E4BC4F800380023C4F8003EC02323608E
:102270006E6D4FF40413A3633369002BFCDA012362
:1022800033610C20FFF7BAFA3369DB07FCD4122064
:10229000FFF7B4FA3369002BFCDA0026A660284663
:1022A000FFF776FF6B68C4F81068DB68C4F8146841
:1022B000C4F81C684BB90A4BA3614FF0FF3363614C
:1022C000A36843F00103A36070BD064BF4E700BFB1
:1022D000682D002000380240401400400300200216
:1022E000003C30C0083C30C0F8B5446D05460021C4
:1022F0002046FFF779FFA96D00234FF001128F6888
:10230000C4F834384FF00066C4F81C284FF0FF3092
:1023100004EB431201339F42C2F80069C2F8006B1C
:10232000C2F80809C2F8080BF2D20B686A6DEB65B7
:10233000636210231361166916F01006FBD1122098
:10234000FFF75CFAD4F8003823F4FE63C4F80038D1
:10235000A36943F4402343F01003A3610923C4F8A5
:102360001038C4F814380A4BEB604FF0C043C4F87F
:10237000103B084BC4F8003BC4F81069C4F800399E
:10238000EB6D03F1100243F48013EA65A362F8BD1C
:10239000EC36000840800010426D90F84E10D2F8E4
:1023A000003823F4FE6343EA0113C2F80038704793
:1023B0002DE9F84300EB8103456DDA68166806F0F5
:1023C0000306731E022B05EB41130C4680460FFAE1
:1023D00081F94FEA41104FF00001C3F8101B4FF094
:1023E000010104F1100398BFB60401FA03F39169E7
:1023F0008EBF334E06F1805606F5004600293AD0CE
:10240000578A04F15801490137436F50D5F81C1819
:102410000B43C5F81C382B180021C3F81019536959
:102420000127611EA7409BB3138A928B9B08012A48
:1024300088BF5343D8F85C20981842EA034301F15F
:10244000400205EB8202C8F85C0021465360284632
:10245000FFF7CAFE08EB8900C3681B8A43EA84536E
:10246000483464011E432E51D5F81C381F43C5F86B
:102470001C78BDE8F88305EB4917D7F8001B21F459
:102480000041C7F8001BD5F81C1821EA0303C0E778
:1024900004F13F0305EB83030A4A5A6028462146AC
:1024A000FFF7A2FE05EB4910D0F8003923F40043F2
:1024B000C0F80039D5F81C3823EA0707D7E700BF72
:1024C0000080001000040002826D1268C265FFF7F0
:1024D0005FBE00005831436D49015B5813F4004062
:1024E00004D013F4001F0CBF02200120704700002D
:1024F0004831436D49015B5813F4004004D013F494
:10250000001F0CBF022001207047000000EB81017A
:10251000CB68196A0B6813604B6853607047000002
:1025200000EB810330B5DD68AA691368D36019B97F
:10253000402B84BF402313606B8A1468426D1C4497
:10254000013CB4FBF3F46343033323F0030302EBD6
:10255000411043EAC44343F0C043C0F8103B2B682A
:1025600003F00303012B09B20ED1D2F8083802EBB5
:10257000411013F4807FD0F8003B14BF43F0805328
:1025800043F00053C0F8003B02EB4112D2F8003B8D
:1025900043F00443C2F8003B30BD00002DE9F04198
:1025A000244D6E6D06EB40130446D3F8087BC3F848
:1025B000087B38070AD5D6F81438190706D505EB75
:1025C00084032146DB6828465B689847FA071FD5D5
:1025D000D6F81438DB071BD505EB8403D968CCB9D2
:1025E0008B69488A5A68B2FBF0F600FB16228AB95A
:1025F0001868DA6890420DD2121AC3E90024302319
:1026000083F311880B482146FFF78AFF84F3118872
:10261000BDE8F081012303FA04F26B8923EA020387
:102620006B81CB68002BF3D021460248BDE8F04116
:10263000184700BF682D002000EB810370B5DD68EE
:10264000436D6C692668E6604A0156BB1A444FF434
:102650000020C2F810092A6802F00302012A0AB217
:102660000ED1D3F8080803EB421410F4807FD4F89D
:10267000000914BF40F0805040F00050C4F8000939
:1026800003EB4212D2F8000940F00440C2F80009FE
:10269000D3F83408012202FA01F10143C3F83418D7
:1026A00070BD19B9402E84BF4020206020682E8A5A
:1026B0008419013CB4FBF6F440EAC44040F00050F9
:1026C0001A44C6E72DE9F8433B4D6E6D06EB401307
:1026D0000446D3F80889C3F8088918F0010F4FEAB7
:1026E00040171AD0D6F81038DB0716D505EB800353
:1026F000D9684B691868DA68904230D2121A4FF0E4
:1027000000091A60C3F80490302383F3118821462E
:102710002846FFF791FF89F3118818F0800F1CD02D
:10272000D6F834380126A640334216D005EB840390
:102730006D6DD3F80CC0DCF814200134E4B2D2F88B
:1027400000E005EB04342F445168714515D3D5F8EA
:10275000343823EA0606C5F83468BDE8F883012357
:1027600003FA04F22B8923EA02032B818B68002BE6
:10277000D3D0214628469847CFE7BCF81000AEEBEF
:102780000103834228BF0346D7F8180980B2B3EB90
:10279000800FE2D89068A0F1040959F8048FC4F8BA
:1027A0000080A0EB09089844B8F1040FF5D818444C
:1027B0000B4490605360C7E7682D00202DE9F74F68
:1027C000A24C656D6E69AB691E4016F480586E614F
:1027D00007D02046FEF728FD03B0BDE8F04F00F01B
:1027E00047BC002E12DAD5F8003E98489B071EBF62
:1027F000D5F8003E23F00303C5F8003ED5F80438B1
:1028000023F00103C5F80438FEF738FD370505D578
:102810008E48FFF7BDFC8D48FEF71EFDB0040CD5B9
:10282000D5F8083813F0060FEB6823F470530CBF8B
:1028300043F4105343F4A053EB6031071BD5636896
:10284000DB681BB9AB6923F00803AB612378052B68
:102850000CD1D5F8003E7D489A071EBFD5F8003E42
:1028600023F00303C5F8003EFEF708FD6368DB684C
:102870000BB176489847F30274D4B70227D5D4F841
:102880005490DFF8C8B100274FF0010A09EB471256
:10289000D2F8003B03F44023B3F5802F11D1D2F8D6
:1028A000003B002B0DDA62890AFA07F322EA0303E0
:1028B000638104EB8703DB68DB6813B13946584654
:1028C0009847A36D01379B68FFB29F42DED9F0069F
:1028D00017D5676D3A6AC2F30A1002F00F0302F4CB
:1028E000F012B2F5802F00F08580B2F5402F08D1AC
:1028F00004EB83030022DB681B6A07F580579042D4
:102900006AD13003D5F8184813D5E10302D5002069
:10291000FFF744FEA20302D50120FFF73FFE630349
:1029200002D50220FFF73AFE270302D50320FFF766
:1029300035FE75037FF550AFE00702D50020FFF7A5
:10294000C1FEA10702D50120FFF7BCFE620702D538
:102950000220FFF7B7FE23077FF53EAF0320FFF706
:10296000B1FE39E7636DDFF8E4A0019300274FF073
:102970000109A36D9B685FFA87FB9B453FF67DAF1E
:10298000019B03EB4B13D3F8001901F44021B1F57F
:10299000802F1FD1D3F8001900291BDAD3F80019B2
:1029A00041F09041C3F80019D3F800190029FBDB6E
:1029B0005946606DFFF718FC218909FA0BF321EAEB
:1029C0000303238104EB8B03DB689B6813B1594637
:1029D000504698470137CCE7910708BFD7F80080E9
:1029E000072A98BF03F8018B02F1010298BF4FEA52
:1029F000182884E7023304EB830207F580575268F6
:102A0000D2F818C0DCF80820DCE9001CA1EB0C0CA3
:102A1000002188420AD104EB830463689B699A68A9
:102A200002449A605A6802445A606AE711F0030F40
:102A300008BFD7F800808C4588BF02F8018B01F1F0
:102A4000010188BF4FEA1828E3E700BF682D002086
:102A5000436D03EB4111D1F8003B43F40013C1F87F
:102A6000003B7047436D03EB4111D1F8003943F44B
:102A70000013C1F800397047436D03EB4111D1F8E1
:102A8000003B23F40013C1F8003B7047436D03EB98
:102A90004111D1F8003923F40013C1F8003970470F
:102AA00000F1604303F561430901C9B283F80013E3
:102AB000012200F01F039A4043099B0003F1604389
:102AC00003F56143C3F880211A60704730B5039C59
:102AD0000172043304FB0325C0E90653049B03631E
:102AE0000021059BC160C0E90000C0E90422C0E9E3
:102AF0000842C0E90A11436330BD0000416A002268
:102B0000C0E90411C0E90A22C2606FF00101FEF7BA
:102B1000E5BE0000D0E90432934201D1C2680AB98F
:102B2000181D70470020704703691960C2680132A0
:102B3000C260C269134482690361934224BF436A3D
:102B400003610021FEF7BEBE38B504460D46E368BA
:102B50003BB16269131D1268A3621344E362002053
:102B600007E0237A33B929462046FEF79BFE00286A
:102B7000EDDA38BD6FF00100FBE70000C368C26901
:102B8000013BC3604369134482694361934224BF9C
:102B9000436A436100238362036B03B118477047A4
:102BA00070B53023044683F31188866A3EB9FFF777
:102BB000CBFF054618B186F31188284670BDA36A7D
:102BC000E26A13F8015BA362934202D32046FFF747
:102BD000D5FF002383F31188EFE700002DE9F84FBC
:102BE00004460E46174698464FF0300989F311887F
:102BF0000025AA46D4F828B0BBF1000F09D1414600
:102C00002046FFF7A1FF20B18BF311882846BDE8CD
:102C1000F88FD4E90A12A7EB050B521A934528BF87
:102C20009346BBF1400F1BD9334601F1400251F8E6
:102C3000040B43F8040B9142F9D1A36A40334036A8
:102C4000A3624035D4E90A239A4202D32046FFF713
:102C500095FF8AF31188BD42D8D289F31188C9E75C
:102C600030465A46FEF71CF8A36A5B445E44A362F2
:102C70005D44E7E710B5029C0172043303FB0421B5
:102C8000C0E906130023C0E90A33039B0363049BD6
:102C9000C460C0E90000C0E90422C0E908424363FF
:102CA00010BD0000026AC260426AC0E9042200222C
:102CB000C0E90A226FF00101FEF710BED0E904233B
:102CC0009A4201D1C26822B9184650F8043B0B6001
:102CD000704700231846FAE7C368C2690133C3602E
:102CE0004369134482694361934224BF436A436149
:102CF0000021FEF7E7BD000038B504460D46E36845
:102D00003BB123691A1DA262E2691344E362002009
:102D100007E0237A33B929462046FEF7C3FD002891
:102D2000EDDA38BD6FF00100FBE7000003691960C0
:102D3000C268013AC260C269134482690361934266
:102D400024BF436A036100238362036B03B1184706
:102D50007047000070B530230D460446114683F3DA
:102D60001188866A2EB9FFF7C7FF10B186F3118864
:102D700070BDA36A1D70A36AE26A01339342A36225
:102D800004D3E16920460439FFF7D0FF002080F327
:102D90001188EDE72DE9F84F04460D469046994617
:102DA0004FF0300A8AF311880026B346A76A4FB95C
:102DB00049462046FFF7A0FF20B187F3118830462F
:102DC000BDE8F88FD4E90A073A1AA8EB060797423C
:102DD00028BF1746402F1BD905F1400355F8042B97
:102DE00040F8042B9D42F9D1A36A4033A3624036D8
:102DF000D4E90A239A4204D3E16920460439FFF753
:102E000095FF8BF311884645D9D28AF31188CDE717
:102E100029463A46FDF744FFA36A3B443D44A3627A
:102E20003E44E5E7D0E904239A4217D1C3689BB139
:102E3000836A8BB1043B9B1A0ED01360C368013BBD
:102E4000C360C3691A44836902619A4224BF436A1A
:102E50000361002383620123184670470023FBE7C8
:102E600000F030B94FF08043586A70474FF080430C
:102E7000002258631A610222DA6070474FF08043E3
:102E80000022DA60704700004FF0804358637047BB
:102E9000FEE7000070B51B4B01630025044686B0B9
:102EA000586085620E4600F0BFF804F11003C4E9D3
:102EB00004334FF0FF33C4E90635C4E90044A5608C
:102EC000E562FFF7CFFF2B460246C4E9082304F171
:102ED00034010D4A256580232046FEF799FC012325
:102EE000E0600A4A0375009272680192B268CDE907
:102EF0000223074B6846CDE90435FEF7B1FC06B066
:102F000070BD00BF002600201C37000821370008D4
:102F1000912E0008024AD36A1843D062704700BF5E
:102F2000982300204B6843608B688360CB68C36044
:102F30000B6943614B6903628B6943620B680360F1
:102F40007047000008B5264B26481A6940F2FF1169
:102F50000A431A611A6922F4FF7222F001021A610F
:102F60001A691A6B0A431A631A6D0A431A651E4AD4
:102F70001B6D1146FFF7D6FF02F11C0100F58060C2
:102F8000FFF7D0FF02F1380100F58060FFF7CAFFBC
:102F900002F1540100F58060FFF7C4FF02F17001F7
:102FA00000F58060FFF7BEFF02F18C0100F5806044
:102FB000FFF7B8FF02F1A80100F58060FFF7B2FF4C
:102FC00002F1C40100F58060FFF7ACFF02F1E001FF
:102FD00000F58060FFF7A6FFBDE8084000F0EEB8FE
:102FE00000380240000002402837000808B500F011
:102FF00059FAFEF7D1FBFFF791F8BDE80840FEF75C
:1030000059BE000070470000EFF3098305494A6B81
:1030100022F001024A63683383F30988002383F3B3
:103020001188704700EF00E0302080F3118862B60D
:103030000C4B0D4AD96821F4E0610904090C0A43DC
:10304000DA60D3F8FC20094942F08072C3F8FC2012
:103050000A6842F001020A602022DA7783F822002F
:10306000704700BF00ED00E00003FA05001000E02B
:1030700010B5302383F311880E4B5B6813F40063A3
:1030800014D0F1EE103AEFF30984683C4FF08073EE
:10309000E361094BDB6B236684F30988FEF750FB81
:1030A00010B1064BA36110BD054BFBE783F31188FC
:1030B000F9E700BF00ED00E000EF00E03303000897
:1030C000360300080F4B1A6C42F001021A641A6EA4
:1030D00042F001021A660C4A1B6E936843F001032A
:1030E00093604FF0804353229A624FF0FF32DA62CE
:1030F00000229A615A63DA605A6001225A611A60AA
:10310000704700BF00380240002004E04FF08042CA
:1031100008B51169D3680B40D9B2C9439B07116147
:1031200007D5302383F31188FEF74CFB002383F38C
:10313000118808BD1F4B1A696FEAC2526FEAD2525A
:103140001A611A69C2F308021A614FF0FF301A6956
:103150005A69586100215A6959615A691A6A62F0BC
:1031600080521A621A6A02F080521A621A6A5A6A05
:1031700058625A6A59625A6A1A6C42F080521A644A
:103180001A6E42F080521A661A6E0B4A106840F4AA
:1031900080701060186F00F44070B0F5007F1EBFA3
:1031A0004FF4803018671967536823F40073536035
:1031B00000F054B90038024000700040334B4FF02B
:1031C00080521A64324A4FF4404111601A6842F04A
:1031D00001021A601A689107FCD59A6822F003026E
:1031E0009A602A4B9A6812F00C02FBD1196801F020
:1031F000F90119609A601A6842F480321A601A68FC
:103200009203FCD55A6F42F001025A671F4B5A6F66
:103210009007FCD51F4A5A601A6842F080721A6003
:103220001B4A53685904FCD5184B1A689201FCD507
:10323000194A9A60194B1A68194B9A42194B21D1B5
:10324000194A1168194A91421CD140F205121A60BC
:10325000144A136803F00F03052BFAD10B4B9A683D
:1032600042F002029A609A6802F00C02082AFAD12F
:103270005A6C42F480425A645A6E42F480425A6652
:103280005B6E704740F20572E1E700BF0038024014
:10329000007000400854400700948838002004E083
:1032A00011640020003C024000ED00E041C20F41EB
:1032B000074A08B5536903F00103536123B1054A76
:1032C00013680BB150689847BDE80840FFF7D0BEBF
:1032D000003C0140E02D0020074A08B5536903F087
:1032E0000203536123B1054A93680BB1D068984734
:1032F000BDE80840FFF7BCBE003C0140E02D0020C7
:10330000074A08B5536903F00403536123B1054A22
:1033100013690BB150699847BDE80840FFF7A8BE94
:10332000003C0140E02D0020074A08B5536903F036
:103330000803536123B1054A93690BB1D0699847DB
:10334000BDE80840FFF794BE003C0140E02D00209E
:10335000074A08B5536903F01003536123B1054AC6
:10336000136A0BB1506A9847BDE80840FFF780BE6A
:10337000003C0140E02D0020164B10B55C6904F4C0
:1033800078725A61A30604D5134A936A0BB1D06AC6
:103390009847600604D5104A136B0BB1506B9847E1
:1033A000210604D50C4A936B0BB1D06B9847E2050C
:1033B00004D5094A136C0BB1506C9847A30504D58A
:1033C000054A936C0BB1D06C9847BDE81040FFF7ED
:1033D0004FBE00BF003C0140E02D0020194B10B54E
:1033E0005C6904F47C425A61620504D5164A136D87
:1033F0000BB1506D9847230504D5134A936D0BB15B
:10340000D06D9847E00404D50F4A136E0BB1506E8F
:103410009847A10404D50C4A936E0BB1D06E98471F
:10342000620404D5084A136F0BB1506F9847230408
:1034300004D5054A936F0BB1D06F9847BDE8104093
:10344000FFF716BE003C0140E02D002008B5FFF755
:103450005DFEBDE80840FFF70BBE0000062108B581
:103460000846FFF71DFB06210720FFF719FB062181
:103470000820FFF715FB06210920FFF711FB0621A5
:103480000A20FFF70DFB06211720FFF709FB062195
:103490002820FFF705FBBDE8084007211C20FFF7A7
:1034A000FFBA000008B5FFF745FE00F00BF8FDF786
:1034B00051FEFDF729FDFFF7A5FDBDE80840FFF728
:1034C000CFBC00000023054A19460133102BC2E986
:1034D000001102F10802F8D1704700BFE02D002072
:1034E000034611F8012B03F8012B002AF9D170478C
:1034F00053544D3332463F3F3F00000053544D3349
:1035000032463430780053544D33324634327800EA
:1035100053544D333246343436585800012033006A
:103520000010410001105A0003105900071031002B
:1035300000000000F03400083F0000001304000009
:10354000FC3400083F0000001904000006350008A4
:103550003F00000021040000103500083F0000007B
:1035600000000000850E0008710E0008AD0E000876
:10357000990E0008A50E0008910E00087D0E0008A7
:10358000690E0008B90E00080000000001000000EC
:10359000000000006330000094350008F023002094
:1035A000002600204172647550696C6F74002542DA
:1035B0004F415244252D424C002553455249414C20
:1035C000250000000200000000000000A11000081B
:1035D0000D11000840004000A02A0020B02A002061
:1035E00002000000000000000300000000000000D6
:1035F000511100080000000010000000C02A002047
:10360000000000000100000000000000682D002004
:1036100001010200511C0008611B0008FD1B00088D
:10362000E11B0008430000002C360008090243009B
:10363000020100C032090400000102020100052459
:1036400000100105240100010424020205240600E3
:1036500001070582030800FF09040100020A0000B7
:10366000000705010240000007058102400000003C
:10367000120000007836000812011001020000401C
:10368000091241570002010203010000040309046A
:1036900025424F4152442500537065656479426567
:1036A000654634303557494E470030313233343572
:1036B0003637383941424344454600000040000057
:1036C0000040000000400000004000000000010039
:1036D00000000200000002000000020000000200E2
:1036E00000000200000002000000020000000000D4
:1036F000951200084D150008F9150008400040001B
:10370000C82D0020C82D002001000000D82D002069
:103710008000000040010000030000006D61696E40
:103720000069646C65000000000180160000000064
:10373000AAAAAAAA00010000FF9F00000000000042
:1037400000A00A000000000100000000AAAAAAAA26
:1037500000000001FFFF000000000000000000006A
:103760000000001000000000AAAAAAAA0000001091
:10377000FFFF00000000000000000000000000004B
:1037800000000000AAAAAAAA00000000FFFF000093
:103790000000000000000000000000000000000029
:1037A000AAAAAAAA00000000FFFF00000000000073
:1037B000000000000000000000000000AAAAAAAA61
:1037C00000000000FFFF00000000000000000000FB
:1037D0000000000000000000AAAAAAAA0000000041
:1037E000FFFF0000000000000000000000000000DB
:1037F000000000000A0000000000000003000000BC
:1038000000000000000000000000000000000000B8
:1038100000000000000000000000000000000000A8
:103820000000000000000000520400000000000042
:1038300000000F0000000000FF00960000000008DC
:103840000096000000000800040000008C3600080C
:103850000000000000000000000000000000000068
:103860000000000000000000FFFFFFFFFFFFFFFF60
:10387000FFFFFFFFFFFFFFFFFFFFFFFFFFFFFFFF58
:10388000FFFFFFFFFFFFFFFFFFFFFFFFFFFFFFFF48
:10389000FFFFFFFFFFFFFFFFFFFFFFFFFFFFFFFF38
:1038A000FFFFFFFFFFFFFFFFFFFFFFFFFFFFFFFF28
:020000040801F1
:10000000000600209912010821910A087D900A0833
:10001000E9900A087D900A08B5900A089B12010829
:100020009B1201089B1201089B120108F9F10C08B0
:100030009B1201089B1201089B1201089B120108E8
:100040009B1201089B1201089B1201089B120108D8
:100050009B1201089B12010891FD0C08B9FD0C08C8
:10006000E1FD0C0809FE0C0831FE0C0885A10C0806
:10007000ADA10C08D9A10C0805A20C0831A20C08EE
:1000800059A20C0885A20C0809A10C089B120108B2
:100090009B1201089B1201089B12010859FE0C08D3
:1000A000A5FF0C08B9FF0C08CDFF0C08D1FF0C0808
:1000B000D5FF0C08E9FF0C08FDFF0C0811A80C087F
:1000C000B9A90C089B1201089B1201089B12010898
:1000D0009B1201082DFF0C0841FF0C0855FF0C086E
:1000E000BDFE0C089B1201089B12010821000D089F
:1000F00025000D0839000D083D000D08B1A20C08BF
:100100009B1201089B12010811000D089B120108A7
:1001100069FF0C087DFF0C089B1201089B12010867
:10012000DDA20C0805A30C0831A30C085DA30C0884
:1001300089A30C089B1201089B1201089B1201085D
:100140009B1201089B1201089B12010825F90C085B
:10015000B1A30C08DDA30C0809A40C0891FF0C083E
:100160009B1201089B1201089B1201089B120108B7
:100170009B1201089B1201089B1201089B120108A7
:100180009B1201089B1201089B1201089B12010897
:100190009B1201089B1201089B1201089B12010887
:1001A0009B1201089B1201089B1201089B12010877
:1001B0009B1201089B1201089B1201089B12010867
:1001C0009B1201089B1201089B1201089B12010857
:1001D0009B1201089B1201089B1201089B12010847
:1001E00035660108D1400308DDB40408513B060818
:1001F0007541060829C106086D240708312C070837
:10020000692F0708D9920708D9B90708A971080802
:1002100075C50808CDD20808ED810A0891870A083B
:100220004D660B08C1D20B08D9F90B0899100C08C0
:10023000FD3F0C0829460C080000000000000000EB
:1002400081F0004102E000BF83F0004330B54FEA87
:1002500041044FEA430594EA050F08BF90EA020FF4
:100260001FBF54EA000C55EA020C7FEA645C7FEA87
:10027000655C00F0E2804FEA5454D4EB5555B8BFAA
:100280006D420CDD2C4480EA020281EA030382EA1B
:10029000000083EA010180EA020281EA0303362DAD
:1002A00088BF30BD11F0004F4FEA01314FF4801C80
:1002B0004CEA113102D0404261EB410113F0004F92
:1002C0004FEA03334CEA133302D0524263EB430349
:1002D00094EA050F00F0A780A4F10104D5F1200EE7
:1002E0000DDB02FA0EFC22FA05F2801841F1000142
:1002F00003FA0EF2801843FA05F359410EE0A5F116
:1003000020050EF1200E012A03FA0EFC28BF4CF046
:10031000020C43FA05F3C01851EBE37101F00045FC
:1003200007D54FF0000EDCF1000C7EEB00006EEB09
:100330000101B1F5801F1BD3B1F5001F0CD3490893
:100340005FEA30004FEA3C0C04F101044FEA4452EA
:1003500012F5800F80F09A80BCF1004F08BF5FEA71
:10036000500C50F1000041EB045141EA050130BD51
:100370005FEA4C0C404141EB0101013C28BFB1F563
:10038000801FE9D291F0000F04BF01460020B1FAAE
:1003900081F308BF2033A3F10B03B3F120020CDA81
:1003A0000C3208DD02F1140CC2F10C0201FA0CF05F
:1003B00021FA02F10CE002F11402D8BFC2F1200CC4
:1003C00001FA02F120FA0CFCDCBF41EA0C0190407A
:1003D000E41AA2BF01EB0451294330BD6FEA0404C3
:1003E0001F3C1CDA0C340EDC04F11404C4F12002AE
:1003F00020FA04F001FA02F340EA030021FA04F3C0
:1004000045EA030130BDC4F10C04C4F1200220FA16
:1004100002F001FA04F340EA0300294630BD21FA54
:1004200004F0294630BD94F0000F83F4801306BF1A
:1004300081F480110134013D4EE77FEA645C18BF0E
:100440007FEA655C29D094EA050F08BF90EA020FA5
:1004500005D054EA000C04BF1946104630BD91EA9D
:10046000030F1EBF0021002030BD5FEA545C05D1A0
:100470004000494128BF41F0004130BD14F58004DF
:100480003CBF01F5801130BD01F0004545F0FE4153
:1004900041F470014FF0000030BD7FEA645C1ABF88
:1004A000194610467FEA655C1CBF0B46024650EABF
:1004B000013406BF52EA033591EA030F41F40021EB
:1004C00030BD00BF90F0000F04BF0021704730B571
:1004D0004FF4806404F132044FF000054FF0000146
:1004E00050E700BF90F0000F04BF0021704730B507
:1004F0004FF4806404F1320410F0004548BF4042DC
:100500004FF000013EE700BF42004FEAE2014FEA30
:1005100031014FEA02701FBF12F07F4393F07F4F0B
:1005200081F06051704732F07F4208BF704793F00E
:100530007F4F04BF41F40021704730B54FF4607421
:1005400001F0004521F000411CE700BF50EA010224
:1005500008BF704730B54FF000050AE050EA0102CD
:1005600008BF704730B511F0004502D5404261EB3D
:1005700041014FF4806404F132045FEA915C3FF47E
:10058000D8AE4FF003025FEADC0C18BF03325FEA1B
:10059000DC0C18BF033202EBDC02C2F1200300FACC
:1005A00003FC20FA02F001FA03FE40EA0E0021FAF1
:1005B00002F11444BDE600BF70B54FF0FF0C4CF4DF
:1005C000E06C1CEA11541DBF1CEA135594EA0C0F91
:1005D00095EA0C0F00F0DEF82C4481EA030621EACC
:1005E0004C5123EA4C5350EA013518BF52EA033507
:1005F00041F4801143F4801338D0A0FB02CE4FF0B9
:100600000005E1FB02E506F00042E0FB03E54FF0E8
:100610000006E1FB03569CF0000F18BF4EF0010EE0
:10062000A4F1FF04B6F5007F64F5407404D25FEADC
:100630004E0E6D4146EB060642EAC62141EA55518F
:100640004FEAC52040EA5E504FEACE2EB4F1FD0CD1
:1006500088BFBCF5E06F1ED8BEF1004F08BF5FEA4F
:10066000500E50F1000041EB045170BD06F0004601
:1006700046EA010140EA020081EA0301B4EB5C04AE
:10068000C2BFD4EB0C0541EA045170BD41F48011A6
:100690004FF0000E013C00F3AB8014F1360FDEBFCB
:1006A000002001F0004170BDC4F10004203C35DAA7
:1006B0000C341BDC04F11404C4F1200500FA05F32A
:1006C00020FA04F001FA05F240EA020001F00042CB
:1006D00021F0004110EBD37021FA04F642EB060141
:1006E0005EEA430E08BF20EAD37070BDC4F10C046B
:1006F000C4F1200500FA04F320FA05F001FA04F22F
:1007000040EA020001F0004110EBD37041F100011A
:100710005EEA430E08BF20EAD37070BDC4F1200525
:1007200000FA05F24EEA020E20FA04F301FA05F28D
:1007300043EA020321FA04F001F0004121FA04F235
:1007400020EA020000EBD3705EEA430E08BF20EA05
:10075000D37070BD94F0000F0FD101F0004640003F
:1007600041EB010111F4801F08BF013CF7D041EAC1
:10077000060195F0000F18BF704703F000465200C5
:1007800043EB030313F4801F08BF013DF7D043EA96
:100790000603704794EA0C0F0CEA135518BF95EA4C
:1007A0000C0F0CD050EA410618BF52EA4306D1D1D3
:1007B00081EA030101F000414FF0000070BD50EAF2
:1007C000410606BF1046194652EA430619D094EA7C
:1007D0000C0F02D150EA013613D195EA0C0F05D166
:1007E00052EA03361CBF104619460AD181EA0301BA
:1007F00001F0004141F0FE4141F470014FF0000072
:1008000070BD41F0FE4141F4780170BD70B54FF00C
:10081000FF0C4CF4E06C1CEA11541DBF1CEA13558C
:1008200094EA0C0F95EA0C0F00F0A7F8A4EB05046E
:1008300081EA030E52EA03354FEA013100F0888065
:100840004FEA03334FF0805545EA131343EA12632E
:100850004FEA022245EA111545EA10654FEA0026E3
:100860000EF000419D4208BF964244F1FD0404F59C
:10087000407402D25B084FEA3202B61A65EB0305F8
:100880005B084FEA32024FF480104FF4002CB6EBB5
:10089000020E75EB030E22BFB61A754640EA0C0035
:1008A0005B084FEA3202B6EB020E75EB030E22BF75
:1008B000B61A754640EA5C005B084FEA3202B6EBB6
:1008C000020E75EB030E22BFB61A754640EA9C0075
:1008D0005B084FEA3202B6EB020E75EB030E22BF45
:1008E000B61A754640EADC0055EA060E18D04FEA03
:1008F000051545EA16754FEA06164FEAC30343EAA3
:1009000052734FEAC2025FEA1C1CC0D111F4801F6F
:100910000BD141EA00014FF000004FF0004CB6E768
:1009200011F4801F04BF01430020B4F1FD0C88BF07
:10093000BCF5E06F3FF6AFAEB5EB030C04BFB6EB12
:10094000020C5FEA500C50F1000041EB045170BD05
:100950000EF0004E4EEA113114EB5C04C2BFD4EB32
:100960000C0541EA045170BD41F480114FF0000EB6
:10097000013C90E645EA060E8DE60CEA135594EA32
:100980000C0F08BF95EA0C0F3FF43BAF94EA0C0F35
:100990000AD150EA01347FF434AF95EA0C0F7FF4AA
:1009A00025AF104619462CE795EA0C0F06D152EAFE
:1009B00003353FF4FDAE1046194622E750EA4106E2
:1009C00018BF52EA43067FF4C5AE50EA41047FF4F3
:1009D0000DAF52EA43057FF4EBAE12E74FF0FF3C58
:1009E00006E000BF4FF0010C02E000BF4FF0010C29
:1009F0004DF804CD4FEA410C7FEA6C5C4FEA430CA2
:100A000018BF7FEA6C5C1BD001B050EA410C0CBFF0
:100A100052EA430C91EA030F02BF90EA020F002052
:100A2000704710F1000F91EA030F58BF994208BFB9
:100A300090422CBFD8176FEAE37040F00100704776
:100A40004FEA410C7FEA6C5C02D150EA013C07D1CD
:100A50004FEA430C7FEA6C5CD6D152EA033CD3D018
:100A60005DF8040B704700BF8446104662468C4612
:100A70001946634600E000BF01B5FFF7B7FF002845
:100A800048BF10F1000F01BD4DF808EDFFF7F4FF6E
:100A90000CBF012000205DF808FB00BF4DF808EDF9
:100AA000FFF7EAFF34BF012000205DF808FB00BF1C
:100AB0004DF808EDFFF7E0FF94BF012000205DF83E
:100AC00008FB00BF4DF808EDFFF7CEFF94BF0120F3
:100AD00000205DF808FB00BF4DF808EDFFF7C4FFEC
:100AE00034BF012000205DF808FB00BF4FEA410C35
:100AF0007FEA6C5C02D150EA013C0AD14FEA430C18
:100B00007FEA6C5C02D152EA033C02D14FF0000054
:100B100070474FF0010070474FEA410212F5001292
:100B200015D211D56FF47873B3EB625212D94FEA34
:100B3000C12343F0004343EA505311F0004F23FA1E
:100B400002F018BF404270474FF00000704750EA73
:100B5000013005D111F0004008BF6FF00040704730
:100B60004FF00000704700BF4A0011D212F500128A
:100B700011D20DD56FF47873B3EB62520ED44FEAF5
:100B8000C12343F0004343EA505323FA02F0704775
:100B90004FF00000704750EA013002D14FF0FF30B3
:100BA00070474FF0000070474FEA4102B2F1E04356
:100BB00024BFB3F5001CDCF1FE5C0DD901F0004C44
:100BC0004FEAC0024CEA5070B2F1004F40EB830094
:100BD00008BF20F00100704711F0804F21D113F1C0
:100BE0003872BCBF01F00040704741F480114FEAF9
:100BF0005252C2F11802C2F1200C10FA0CF320FA82
:100C000002F018BF40F001004FEAC1234FEAD3239E
:100C100003FA0CFC40EA0C0023FA02F34FEA430308
:100C2000CCE77FEA625307D150EA01331EBF4FF091
:100C3000FE4040F44000704701F0004040F0FE40AC
:100C400040F40000704700BF80F0004002E000BFA9
:100C500081F0004142001FBF5FEA410392EA030FA7
:100C60007FEA226C7FEA236C6AD04FEA1262D2EBF1
:100C70001363C1BFD218414048404140B8BF5B42F6
:100C8000192B88BF704710F0004F40F4000020F08F
:100C90007F4018BF404211F0004F41F4000121F0A5
:100CA0007F4118BF494292EA030F3FD0A2F10102EF
:100CB00041FA03FC10EB0C00C3F1200301FA03F12D
:100CC00000F0004302D5494260EB4000B0F5000F50
:100CD00013D3B0F1807F06D340084FEA310102F10F
:100CE0000102FE2A51D2B1F1004F40EBC25008BFC1
:100CF00020F0010040EA03007047490040EB00008B
:100D0000013A28BFB0F5000FEDD2B0FA80FCACF18B
:100D1000080CB2EB0C0200FA0CF0AABF00EBC250B8
:100D200052421843BCBFD0401843704792F0000FA6
:100D300081F4000106BF80F400000132013BB5E7F9
:100D40004FEA41037FEA226C18BF7FEA236C21D06F
:100D500092EA030F04D092F0000F08BF08467047D4
:100D600090EA010F1CBF0020704712F07F4F04D1A2
:100D7000400028BF40F00040704712F100723CBFB5
:100D800000F50000704700F0004343F0FE4040F4DF
:100D9000000070477FEA226216BF08467FEA23639D
:100DA0000146420206BF5FEA412390EA010F40F488
:100DB000800070474FF0000304E000BF10F00043D4
:100DC00048BF40425FEA000C08BF704743F09643BB
:100DD00001464FF000001CE050EA010208BF7047D6
:100DE0004FF000030AE000BF50EA010208BF70475D
:100DF00011F0004302D5404261EB41015FEA010C72
:100E000002BF84460146002043F0B64308BFA3F169
:100E10008053A3F50003BCFA8CF2083AA3EBC2534B
:100E200010DB01FA02FC634400FA02FCC2F120026A
:100E3000BCF1004F20FA02F243EB020008BF20F0A1
:100E40000100704702F1200201FA02FCC2F1200207
:100E500050EA4C0021FA02F243EB020008BF20EAFC
:100E6000DC7070477BB972B90029BEBF00204FF01B
:100E7000004106E008BF00281CBF6FF000414FF0A2
:100E8000FF3000F007BAADF1080C6DE904CE00297F
:100E900009DB002B1ADB00F095F8DDF804E0DDE952
:100EA000022304B07047404261EB4101002B1BDB81
:100EB00000F088F8DDF804E0DDE9022304B04042E8
:100EC00061EB4101524263EB43037047524263EBD3
:100ED000430300F077F8DDF804E0DDE9022304B015
:100EE000404261EB41017047524263EB430300F023
:100EF00069F8DDF804E0DDE9022304B0524263EB57
:100F00004303704753B94AB9002908BF00281CBFE2
:100F10004FF0FF314FF0FF3000F0BCB9ADF1080CDD
:100F20006DE904CE00F04EF8DDF804E0DDE90223BF
:100F300004B07047430803F05533C01A830803F028
:100F4000333300F03330184400EB101000F00F3052
:100F500000EB002000EB0040000E704707EE900A07
:100F6000F5EEC07AF1EE10FA01D400F00BB8F1EE14
:100F7000677A08B517EE900A00F004F8404261EB7A
:100F8000410108BDD0B5FFF7BFFA0C4B0022064661
:100F90000F46FFF711FBFFF7E7FD0446FFF792FA54
:100FA000074B0022FFF708FB02460B463046394646
:100FB000FFF74AF9FFF7D8FD2146D0BD0000F03D0C
:100FC0000000F0412DE9F047089D04468E46002BB5
:100FD0004DD18A42944669D9B2FA82F252B101FAED
:100FE00002F3C2F1200120FA01F10CFA02FC41EAFD
:100FF000030E94404FEA1C48210CBEFBF8F61FFA82
:101000008CF708FB16E341EA034306FB07F199421C
:101010000AD91CEB030306F1FF3080F01F819942CF
:1010200040F21C81023E63445B1AA4B2B3FBF8F0A9
:1010300008FB103344EA034400FB07F7A7420AD930
:101040001CEB040400F1FF3380F00A81A74240F258
:1010500007816444023840EA0640E41B00261DB1C3
:10106000D4400023C5E900433146BDE8F0878B42F8
:1010700009D9002D00F0EF800026C5E900013046B7
:101080003146BDE8F087B3FA83F6002E4AD18B4291
:1010900002D3824200F2F980841A61EB030301203B
:1010A0009E46002DE0D0C5E9004EDDE702B9FFDE27
:1010B000B2FA82F2002A40F09280A1EB0C014FEAD2
:1010C0001C471FFA8CFE0126200CB1FBF7F307FB2F
:1010D000131140EA01410EFB03F0884208D91CEBD2
:1010E000010103F1FF3802D2884200F2CB8043466F
:1010F000091AA4B2B1FBF7F007FB101144EA01444E
:101100000EFB00FEA64508D91CEB040400F1FF31DC
:1011100002D2A64500F2BB800846A4EB0E0440EACA
:1011200003409CE7C6F12007B34022FA07FC4CEAD3
:10113000030C20FA07F401FA06F31C43F9404FEAC6
:101140001C4900FA06F3B1FBF9F8200C1FFA8CFEDB
:1011500009FB181140EA014108FB0EF0884202FA2F
:1011600006F20BD91CEB010108F1FF3A80F08880F0
:10117000884240F28580A8F102086144091AA4B2AD
:10118000B1FBF9F009FB101144EA014100FB0EFE2E
:101190008E4508D91CEB010100F1FF346CD28E455D
:1011A0006AD90238614440EA0840A0FB0294A1EBEE
:1011B0000E01A142C846A64656D353D05DB1B3EB4B
:1011C000080261EB0E0101FA07F722FA06F3F1407B
:1011D0001F43C5E9007100263146BDE8F087C2F122
:1011E0002003D8400CFA02FC21FA03F3914001439A
:1011F0004FEA1C471FFA8CFEB3FBF7F007FB1036D3
:101200000B0C43EA064300FB0EF69E4204FA02F47E
:1012100008D91CEB030300F1FF382FD29E422DD9D1
:10122000023863449B1B89B2B3FBF7F607FB163306
:1012300041EA034106FB0EF38B4208D91CEB010186
:1012400006F1FF3816D28B4214D9023E6144C91A06
:1012500046EA004638E72E46284605E70646E3E616
:101260001846F8E64B45A9D2B9EB020864EB0C0E20
:101270000138A3E74646EAE7204694E74046D1E72F
:10128000D0467BE7023B614432E7304609E76444DD
:10129000023842E7704700BF02E000F000F8FEE7C6
:1012A00072B6374880F30888364880F30988364894
:1012B0003649086040F20000CCF200004EF634716E
:1012C000CEF200010860BFF34F8FBFF36F8F40F283
:1012D0000000C0F2F0004EF68851CEF20001086026
:1012E000BFF34F8FBFF36F8F4FF00000E1EE100A96
:1012F0004EF63C71CEF200010860062080F314889F
:10130000BFF36F8FBDF0D6FFBDF03EF84FF0553004
:101310001F491B4A91423CBF41F8040BFAE71D49A3
:10132000184A91423CBF41F8040BFAE71A491B4A9C
:101330001B4B9A423EBF51F8040B42F8040BF8E7EE
:1013400000201849184A91423CBF41F8040BFAE7C3
:10135000BDF0B4FFBDF06CF8144C154DAC4203DA8F
:1013600054F8041B8847F9E701F0A4FB114C124D17
:10137000AC4203DA54F8041B8847F9E7BDF09CBF80
:1013800000060020002200200000010808ED00E017
:10139000000000200006002038A20F0800220020D4
:1013A0002C2C0020302C0020F0680120E0010108E6
:1013B0003802010838020108380201082DE9F04F0F
:1013C0002DED108AC1F80CD0C3689D46BDEC108A83
:1013D000BDE8F08F002383F311882846A047002042
:1013E000BCF058FDFEE7BCF0B5FB00DFFEE70000F7
:1013F00001F0FF01102A2BDB10F0070F08D010F8C6
:10140000013B013A8B422DD010F0070F42B3F6D1C9
:10141000F0B441EA012141EA014122F007047FF0E2
:1014200000070023F0E80256083C85EA010586EA39
:10143000010685FA47F5A3FA87F586FA47F6A5FA75
:1014400087F68EB9EED1F0BC01F0FF0102F0070281
:1014500032B110F8013B013A83EA010313B1F8D12C
:101460000020704701387047002D06BF354603380D
:10147000073815F0010F07D1013015F4807F02BF46
:10148000013015F4C03F0130F0BC0138704700BF97
:1014900010F8012B11F8013B012A28BF9A42F7D01E
:1014A000D01A7047034613F8012B002AFBD1181AF3
:1014B0000138704738B50022002304460D46FFF777
:1014C000EDFA28B920462946BDE8384000F00AB8B0
:1014D000204605F1004100F005F8404261EB410172
:1014E00038BD00BFD0B50C4B002206460F46FFF7B3
:1014F00063F8FFF739FB0446FEF7E4FF074B0022D1
:10150000FFF75AF802460B4630463946FEF79CFE76
:10151000FFF72AFB2146D0BD0000F03D0000F0415E
:10152000036800221B68184710B503685B6804460F
:10153000984708B194F84D0010BD00002DE9F04126
:10154000664B03F5C04490B094F9682206460F46F6
:10155000002A00F0C08094F8B05235B9604A85F096
:10156000ADFE284610B0BDE8F081B3F9A4201AB949
:10157000B3F8A220A3F8A420B3F8A430632B05D8B5
:10158000584A3946304685F099FE002500212E2222
:1015900004A80391C1F0E8FDD4F8C801036803AAC8
:1015A0001B6832219847804630B94F4A03AB394611
:1015B000304685F083FE4546B4F8A431A3F57A732E
:1015C0009BB241F65832934206D9484B3A46202105
:1015D000304685F06BFC002594F9D833002B69DD8B
:1015E00094F99033002B59DD414B3A462021304687
:1015F00085F05CFC00253F49D4F8D401322303AACE
:1016000090F09CFE804640B903AB00933A463A4BBB
:101610002021304685F04AFC45463849D4F8D001AF
:10162000322303AA8DF0BCFE804640B903AB009381
:101630003A46314B2021304685F038FC4546202182
:10164000304685F02BFCB8B1D4ED897A9FED2C7A29
:10165000F0EEE77AF4EEC77AF1EE10FA0CD594F9D1
:10166000D833002B02DD94F83C342BB9254A394697
:10167000304685F023FE002594F9D833002B7FF700
:1016800070AF94F99532002B3FF46BAF1E4B3A4686
:101690002021304685F00AFC002562E794F83C845E
:1016A000B8F1000F06D1194B3A462021304685F09B
:1016B000FDFB454694F99033002B9CDD94F8C183E3
:1016C000B8F1000F97D1124B3A462021304685F0F1
:1016D000EDFB45468FE7012543E700BF402C002086
:1016E00040760D0862760D0889760D0894760D080F
:1016F000A6760D0817770D081B770D082D770D08B6
:101700000000003431770D084B770D08CC760D08BA
:10171000F2760D0838B5044685F0A4FB114B93F81A
:101720007413114B1D68EB6A1A68002908BF014643
:101730001268184690475CF075FCEB6A93F89C10B1
:101740005BF05CFC94F837305BB197F01FFDEB6AFF
:10175000D3F8A030C01AB0F5FA6F24BF002384F884
:10176000373038BD408C00203C2C002008B5FFF7F6
:10177000D1FF054B05481B68DB6A93F89C10BDE858
:10178000084011F045BB00BF3C2C0020DC8D002040
:1017900070B50E46054667F0BFFF67F081FF10B9D0
:1017A0000124204670BD0A4B93F94A32012BF7D130
:1017B00067F0B2FF437A002BF2D167F0ADFF847A75
:1017C000002CEDD1034A3146284685F077FDE8E745
:1017D000404C002064770D08034BD3F8B4320BB9AA
:1017E00085F0F6BA01207047404C00202DE9F04703
:1017F0002DED028BC47F90B006460F468CB990F950
:101800000430002B00F00581834B1D68A86A036833
:101810005B6B9847044650B9804A3946304685F09C
:101820004DFD204610B0BDEC028BBDE8F087B368DB
:101830004BB933685B6B3946304610B0BDEC028B58
:10184000BDE8F0471847E86AFFF76EFE0446002837
:10185000E7D13946304686F0FFFBDFF8F4810546D4
:101860003946304685F052FD98ED977AD8ED967A54
:10187000B4EEE77A2840F1EE10FAC5B209D598F92E
:101880005432032B05D0664A3946304685F016FDA2
:101890002546D8ED7F7AB0EE088AF4EEC87AF1EEEC
:1018A00010FA0BD517EE900AFEF72EFE5D4ACDE931
:1018B00000013946304685F001FD0025D8ED807ADB
:1018C000F4EEC87AF1EE10FA0BD517EE900AFEF797
:1018D0001BFE554ACDE900013946304685F0EEFC45
:1018E0000025D8ED817AB8EE087AF4EEC77AF1EEE9
:1018F00010FA0BDD17EE900AFEF706FE4B4ACDE913
:1019000000013946304685F0D9FC0025B8F9E831A8
:10191000042B07DC052200923946454A304685F003
:10192000CDFC0025D8F8700C67F052FF80B198F913
:101930004A326BB1D8F8703CB8F94C22B3F90E308A
:101940009A4205DA3B4A3946304685F0B7FC002515
:1019500039463046FFF71CFFDFF8F8A081463946CC
:101960003046FFF7EBFD9AF8753F002B4AD109EAA4
:10197000050500EA050430484FF4806101F07CF869
:1019800078B1D8F8703CB3F90C30A3F2E24292B2CD
:10199000B2F5FA7F05D9294A3946304685F08EFCE2
:1019A0000024274890F8C8355BB100F5B86038F0DE
:1019B00015FE054628B9234A3946304685F07EFC97
:1019C0002C4600212E2204A80DF10C080391C1F031
:1019D000CBFBDAF8600F4246322109F0A1FE054642
:1019E00000287FF41EAFDAF8600F03689B68984701
:1019F000154ACDF8008003463946304685F05EFC36
:101A00002C460EE7114A3946304685F057FC002433
:101A1000B1E7012405E700BF3C2C002074770D08D6
:101A20008B770D08AE770D08CE770D08F0770D088F
:101A300012780D0831780D08402C00206C780D08C4
:101A4000407C002094780D0870470E0857780D08E8
:101A5000404C0020406C002070B505460E46FFF754
:101A600097FE31460446284686F0A2F92040C0B2CF
:101A700070BD0000F0B591B005460E4685F0E6FC5D
:101A80000446D8B11021284685F008FAB0B10021EB
:101A90002E2204A803AF0391C1F066FB1CF002F9EB
:101AA00032233A4601211BF0BDFB044630B9054BF9
:101AB000009732461021284685F0F8F9204611B0EB
:101AC000F0BD00BFA8780D0870B505460E46B1B947
:101AD00090F910408CB1164814F0C8F8DFED157A73
:101AE000B0EEC00AB4EEE70AF1EE10FA07D4124ADB
:101AF0000121284685F0E2FB3446204670BDAB68E4
:101B00009BB10E4B1B68D86AFFF70EFD044630B13F
:101B100066F038FB0A4A04215FF04EFBEDE73146E0
:101B20002846BDE8704085F05DBF0124E5E700BFB1
:101B3000402C002000000034B4780D083C2C00201C
:101B4000C6780D0838B5044686F046FB0546A8B1B0
:101B50000B4806F067FC38B10A490B481BF0BAFC89
:101B600010B1074800F05CFF2046FFF7FFFD01239E
:101B7000064984F83730204686F03EFA284638BDBC
:101B8000402C0020848C0020003F0020E8780D08C5
:101B9000F8B505460E461746C2B1232901D00129E2
:101BA00014D8254809F078F8044668B10024204686
:101BB000F8BD95F91030022B08D066F0E3FA1F4A01
:101BC00006215FF0F9FAF2E7002EF2D03A463146EC
:101BD000284686F0B7FB04460028E7D0184ED6F812
:101BE000602F06F54C639A4203D006F5AE5039F0EB
:101BF0002BF9D6F8600F134F03689B6B984787F853
:101C0000980507F58057D7F8EC31012B07D167F01D
:101C100083FD542168F0C8FD08B9C7F8EC012846D7
:101C2000FFF7A4FD4FF0FF330749C6F8983F284659
:101C300086F0E2F9BBE700BF402C0020F8780D08E1
:101C4000406C0020407C002010790D082DE9F04FF9
:101C50002DED028BDFF8489191B00746884685F05C
:101C6000C9F999F91F520446D5B9BD2109F5575054
:101C700039F080F838B1434B42464FF48041384642
:101C800085F014F92C464048BC2139F073F838B17E
:101C90003E4B42464FF48041384685F007F9002418
:101CA0003B4E96F8B032002B66D0A6F580531C222E
:101CB000002102A8B3F8F4A5DFED368AC1F054FA8A
:101CC00004A821F0D9FDA6F5246B0125A6F5C04690
:101CD000554551D20BA821F0CFFD09AA29465846F7
:101CE00036F0E8FC002847D0BDF82610304608F052
:101CF000E1F880B3BDF80A30102B2CD104A90BA851
:101D000022F01CF909F68853B0EE408A93ED000AE0
:101D10002148B4EEE80AF1EE10FAB8BF99ED7B0A5B
:101D200020EE000A0FF08AF9F6EE087A60EE277AC4
:101D3000B4EEE78AF1EE10FA0DD517EE900AFEF731
:101D4000E3FB164BCDE9000142464FF48041384693
:101D500085F0ACF800240DF1240CBCE80F000DF167
:101D6000080EAEE80F009CE80700AEE8030001355E
:101D70008EF80020ADB2ABE7204611B0BDEC028B6F
:101D8000BDE8F08F24790D080082002050790D08FD
:101D9000408C002000000034DC8D002083790D0889
:101DA000404C002000207047014800F0B9BD00BF42
:101DB000402C002003685B68184700006CF006BFE9
:101DC00067F0F8BB30F0FABB5BF09ABA09F0B8B82C
:101DD00059F086BB0DF058BD15F0BEB903F056BBE7
:101DE00057F01ABF1FF05EBE6AF0C8BE6AF058BB5B
:101DF00015F018BA13F0B8BF1FF0B2B96EF09ABC64
:101E000067F0F2B865F028BA08F038BA05F092BA6F
:101E10000DF020B80DF09CBC14F0D8BF15F0B0BA8E
:101E200013F0D6BD15F012B901F0C4BB00F2545046
:101E300022F0ECBD08F0BEBD90F8C432B02202FB27
:101E4000030390F8082393F8A13012B1012B28BFA7
:101E5000012318467047000090F814310BB190F838
:101E60004131184670470000034808602B2111706B
:101E700008221A60704700BFB47C0D08F8B504460C
:101E800000F5C240543004F59656FFF743FC00219C
:101E900030461BF079FE8021204615F0E7FC18B192
:101EA00031F080FF30F050F804F50055D5ED7F7A21
:101EB0009FED317A67EE877A05F68447FDEEE77A83
:101EC00004F5C74017EE903AC5F8803CD5F80432C7
:101ED0003B60543015F0CCFEF8B9D5F8803C07EEE5
:101EE000903A04F5805303F20C5292ED007AF8EE2A
:101EF000E77A03F5A16367EE877AFDEEE77A17EEDE
:101F0000902AC5F8802CD3ED007A97ED007AF0EE98
:101F1000E77A67EE877AC7ED007A04F5AF5118319A
:101F200006F5457035F044FE04F5AA4594ED467A71
:101F3000D5ED067AE7EE007AC5ED067AB0EE670ACF
:101F400032F054FC04F5C34085ED060A1C300EF057
:101F500083F904F5C340002128308AF033F94FF4A7
:101F60000011204615F082FC20B13046BDE8F84053
:101F700019F034BFF8BD00BF0000C842FFF77EBFB4
:101F800070B500F580430546D3F8600F03689B6B7E
:101F9000984705F5C3441C340646204610F0FAFE67
:101FA00005F5A043002893F8573518BF00262BB934
:101FB00026B105F5345018308AF068F8204610F044
:101FC0007FFB18B92046FFF747FF20B12046BDE848
:101FD000704011F02DB970BDFFF7D2BF38B54FF486
:101FE0008011044615F042FC054620B90121204627
:101FF00015F03CFC05460221204615F037FC40B1A7
:1020000015B9204603F068F904F5965019F0E4FD7F
:1020100001E0002DF8D14FF48051204615F026FC48
:1020200030B104F5C1405030BDE838406AF0CCBE54
:1020300038BD0000FFF7D2BF38B54FF48011044619
:1020400015F014FC01210546204615F00FFC18B1CF
:1020500015B9204603F040F91021204615F006FC82
:1020600060B1204603F02AFA4FF48001204615F0B3
:10207000FDFB18B931F096FE30F058F820212046CB
:1020800015F0F4FB28B1204603F08EFA204603F049
:10209000A5FB4FF40051204615F0E8FB10B1204697
:1020A00003F084FB8021204615F0E0FB28B131F0DD
:1020B00079FEBDE838402FF06BBF38BDFFF7BCBFDD
:1020C00010B5044622F092FD90F921308BB190F8C2
:1020D000403373B194F978355BB1064B1B68DB6A0A
:1020E00093F89C302BB904F25450BDE8104022F014
:1020F000A5BA10BD3C2C0020FFF7E2BF2DE9F84344
:10210000434B1B68DB6A93F89C300446002B7CD061
:1021100000F5805797F8C935002B76D008F0BCFD44
:10212000002872D004F5F95507F58059083599F85B
:102130007610284619F0F4F8002866D004F5907659
:102140003046FFF779FE02285FD994F8E4334FF068
:10215000B00808FB034393ED777AF1EE007AB4EE12
:10216000E77AF1EE10FA50D499F87610284619F073
:1021700087FB04F50053B3F9E82107EE902AB8EE87
:10218000E77AB4EEC07AF1EE10FA0CDD94F8E423AD
:1021900008FB0242F8EE677A92ED777AF4EEC77A9E
:1021A000F1EE10FA31DCD7F8B824D3F8801C002AFD
:1021B000B8BF52428A4228DC07F2BC42D2ED007A14
:1021C000D3ED806A9FED136AF8EEE77A66EE866AD1
:1021D000F4EEE67AF1EE10FA17DC03F6844292EDA3
:1021E000007A27EE067AF4EEC77AF1EE10FA0CD4F4
:1021F00094F8E413B02202FB01612846B3F9EA2106
:10220000D431BDE8F84318F009BFBDE8F88300BF3A
:102210003C2C00200000C842FFF770BF2DE9F041C0
:1022200090F8E4332B4D00EB03132F68D3F894811F
:1022300000F5907604463046FFF7FEFD474512D084
:10224000022812D904F58047C5F8008097F8903F1E
:10225000012B13D815D104F5C045EB6CDBB92B6D00
:10226000CBB905230BE0022810D804F5804393F87E
:10227000902F5AB1052283F8902F07E0013B87F891
:10228000903F04F5B7501C301CF0C0FE2046BDE85E
:10229000F0410CF0C9BF104B1B68D86A03685B683B
:1022A000984780460028ECD194F8E413B02303FB50
:1022B0000161AC31204606F025F92B6B0FCB05F1FF
:1022C0003406543586E80F0085E80F0087F8908FB4
:1022D000D7E700BF302C00203C2C0020FFF79EBF2A
:1022E00070B500F5C043044693F8B03200F580564F
:1022F000BBB100F5C740543015F0C0FF18B1012341
:1023000086F8C93570BD04F5C3451C35284610F064
:10231000D7F908B10023F3E72846FFF79DFD002811
:10232000F8D104F5A04393F85725002AF2D1D3F849
:102330009C35042BE3D104F5BE40743093F0E2F8F1
:1023400086F8C905DEE7000010B500F5804400F509
:102350009943D4F8601F4033994200F5A04308D058
:1023600000F59C42483291421CBF4FF0FF32C3F847
:10237000102500F5AA4203F2045306491160064AEB
:102380001A60FFF7ADFFD4F8600F0368BDE8104096
:102390001B6918470000C8420000C8C2FFF7D4BF3D
:1023A000F7B500F5A0470446D7F89C358B420D469B
:1023B00024D00B1F00F5BE46594206F17406594160
:1023C0003046019192F08EFF0199304692F08AFFDB
:1023D000072D0BD104F55050D7F820256423052193
:1023E00092FBF3F32830064A5EF0E6FE2046C7F87B
:1023F0009C5503B0BDE8F04003F03EB903B0F0BD1A
:10240000147A0D0870B500F580460446D6F8600FC2
:1024100003689B6B9847B8B104F5A04595F89835CB
:1024200093B9D6F8602F04F5994340339A424CD1C2
:1024300004F5C3461C3630460FF05EFB60B995F8D4
:1024400050357BB9012108E004F5C3451C35284609
:1024500010F036F900283ED002212046BDE8704039
:10246000FFF79EBFB5F8FE35152B27D195F8781FDD
:1024700011F0010120D1D5F89C35072B1CD095F91E
:10248000EE3F0BB90421E8E7204613F0EFFBDFED48
:10249000137AB4EEE70AF1EE10FAF3DB04F5BE406E
:1024A000743092F06FFF0028ECD004F550500C4AC5
:1024B000062128305EF080FE0721CEE73046FFF788
:1024C000CBFC0028C8D10321C7E704F59C4348335F
:1024D0009A42F8D170BD2846F1E700BF0000B4422F
:1024E000387A0D0838B5314CD4F8602F04F54C63B8
:1024F0009A422DED028B0546B0EE408A03D00020B3
:10250000BDEC028B38BD2A480FF0F6FA40B1BDECA5
:10251000028B05F5C3401C30BDE8384010F008BC04
:1025200004F58055D5F89C35042B35D194F8913FAE
:1025300033B12049A1F6842038F0FEFE0028DFD117
:102540001D4C94F8B0325BB104F5CE700FF0D4FAA4
:102550000028D4D104F5CE700FF08EFA0028CED129
:102560009FED167AF0EEC87AF4EEC77AF1EE10FA23
:1025700009D49FED130A28EE008ABDEEC88A18EE32
:10258000103AC5F820350F4892F0FCFE0028B6D06E
:10259000002385F85335B3E7B5F8FE15A4F5804060
:1025A00007F088FC0028C1D1A9E700BF406C0020DB
:1025B000DC8D0020848C0020408C00200000003442
:1025C0000000C842B48B002010B52DED028B00F541
:1025D000A0430446D3F89C35042B0BD105F020F919
:1025E0002046B0EE408A05F03DFA38EE400ABDECD8
:1025F000028B10BD00F5C04494ED200AF7E70000FF
:102600002DE9F0412DED028B00F586658AB0044678
:1026100028461DF0B3FE002307A904F59650079342
:10262000089309931BF03CF9002800F090809DED81
:10263000090ADFED5E7A04F5A04505F5A66393ED82
:10264000007A20EE270ADFED5A7AA7EE270A04F572
:10265000AD40383004F5804683ED000A6EF0BEF9D7
:102660002046FFF7CFFED6F8600F03689B6B9847B4
:10267000074604F5C3401C3010F08CFB95F8573525
:10268000002818BF0027002B5CD1002F5AD095F8E6
:102690009835002B56D1D5F89C35042B6ED09FED84
:1026A000458A204605F000FA04F5C04204F5994336
:1026B000C2F8FC04D6F8601F6C3399421AD192F824
:1026C000C830BBB904F50053B3F94C3C002B04DC13
:1026D0003949D1F82C1CC9060CD5176B916B7F6852
:1026E0000A33C91B64277B438142ACBF5B181B18AC
:1026F000C2F8FC34D5F89C35D2F8FC14D6F8942FE7
:10270000059120460492039316F0B4FDB6F9A26F2A
:1027100007462046FFF758FFCDE9007604F5005044
:10272000D0EDA11A059905F5B76504F53450F0EE22
:10273000400ADDE9033295ED001AB0EE480A183080
:1027400089F048F90AB0BDEC028BBDE8F08104F5D0
:102750009070FFF771FB02280AD994F8E433B02295
:1027600002FB034393F8102212B193ED7F0A60E756
:1027700028461DF09DFCB1EE400A5AE704F5C0471B
:1027800004F5C048443708F1540804F5C0414246F6
:102790003431384621F03EFB002880D0414638468F
:1027A00021F0CCFBB0EE408A7BE700BFCDCC4C3EA5
:1027B000CDCC4C3F00000000404C0020FFF720BF74
:1027C000F8B500F5804200F59A43D2F8602F6033E7
:1027D0009A4204460E4623D000F5C3471C373846BC
:1027E0000FF06EFF0546A8B138460EF0EFFB70B152
:1027F00004F5C044D4F8D80103689B689847DFED1E
:10280000097A20EE270A86ED000A2846F8BD9FEDDA
:10281000060AF8E704F5AA440125A36B3360F4E740
:102820000025F2E70AD7233C00000000F8B500F5C8
:10283000804200F59A43D2F8602F60339A420446F2
:102840000E4630D000F5C3471C3738460FF038FF2E
:102850000546A8B138460EF0B9FB70B104F5C04486
:10286000D4F8D8010368DB68984707EE900AF8EEC1
:10287000E77AC6ED007A2846F8BDDFED0C7AF8E776
:1028800004F540540125D4F8440603681B699847B1
:1028900007EE900A9FED067AF8EEE77A67EE877A00
:1028A000C6ED007AE7E70025E5E700BF000000007D
:1028B0000AD7233CF8B500F5804200F59A43D2F8D8
:1028C000602F60339A4204460E4624D000F5C34779
:1028D0001C3738460FF0F4FE054688B138460EF036
:1028E00075FB50B104F5C044D4F8D83118698EF0A6
:1028F0008FFC86ED000A2846F8BD9FED080AF8E730
:1029000004F540540125D4F8440603685B699847F0
:1029100086ED000AEFE70025EDE700BF00000000AC
:1029200030B505460FC985B06C4684E80F0040F20B
:1029300079322146284605F083FC0C4B03F62452DD
:10294000D3F8603F93420ED19DF8001011F00401BE
:1029500002D1204621F05AF80548214605F022FD13
:10296000012005B030BD0020FBE700BF406C002017
:10297000402C002010B5044606480FF0D5FC40B9A5
:1029800004F58044D4F8600F0368BDE810409B6CE8
:10299000184710BDDC8D002010B5044606480FF026
:1029A00019F940B904F58044D4F8600F0368BDE814
:1029B0001040DB6C184710BDDC8D002070B504465C
:1029C00000F5C3401C300E4615460EF061FC50B1B8
:1029D00004F5C044D4F850349B682B60D4F85034CC
:1029E0005B68336070BD04F5805303F5996203F2B0
:1029F000C44312682A601B68336004F50054D4F89D
:102A00002C3C9B05EED4D4EDA16AD5ED007A9FED68
:102A1000037AE6EEC77AC5ED007AE3E735FA8E3C35
:102A200038B50C4D044629460B481AF065FE04F5EE
:102A3000804305F13C0183F8910F04F5965004F5AD
:102A4000C0441AF0F1FCD4ED207AF1EE677AC4EDBF
:102A5000207A38BD848C0020003F002010B5044649
:102A600000F590702AF044FC2046BDE81040FFF7C6
:102A7000D7BF0000FFF7F2BF00F50050D0F82C3CA4
:102A8000194214BF012000207047000010B500F566
:102A900080430446D3F8600F03689B6D9847014656
:102AA00004F59D402030BDE8104094F0D9BE0000F0
:102AB000FFF7ECBF38B5054B1C6823680A461D6854
:102AC000034B01462046A847002038BD3C2C00207F
:102AD000402C002070B52DED028B0446036804F5F0
:102AE00000559B6D9847D5F82C3C1B0617D5B5F9BA
:102AF000E831B5F9EA11CA1A0B4402EBD27203EBC2
:102B0000D37352105B1000EE902A00EE103AF8EEEC
:102B1000E00AB8EEC00A04F596501AF00BFA604BC2
:102B2000B5F81A221A7004F5C24568F04FFF543503
:102B300068F086FB00212846FEF758FE594E012317
:102B4000B0712846F37184F08DF928B9284685F0D4
:102B500067FAB0FA80F0400930710421204614F081
:102B600085FE20B104F5AD40583058F06BFD284685
:102B700084F078F904F5C045D8B994F8E43304EB4F
:102B8000031341F28832D3F89461D5F8CC30F31AAC
:102B900093420ED904F59070FFF74EF9022808D938
:102BA000C5F8CC60204605F03DFC04F5BE4300228C
:102BB0005A67B4F9A4301BB9B4F8A230A4F8A43011
:102BC000B4F8A430DFED388A07EE903AF8EEE77AF1
:102BD000B7EE008A88EE270AD4ED2B7AF0EEE77A7A
:102BE000F4EEE87AF1EE10FA09D5B4F9A23007EE66
:102BF000903AF8EEE77A88EE277A84ED2B7AD4EDD6
:102C00002B0A31F0F5FC70BB59F0FAFB40F27D1253
:102C10004FF4801159F0ACFB57F0B4F856F01CFD9E
:102C200095F8B032B0EE408A23B1D5F8D0010368F0
:102C30001B6F984704F53F50B0EE480A14307CF003
:102C400065F804F54450B0EE480A30307CF05EF888
:102C5000B0EE480ABDEC028B04F549502430BDE8C3
:102C600070407CF053B8D4ED2B7A94ED460AF0EE28
:102C7000E77AF4EEE87AF1EE10FA09D5B4F9A23069
:102C800007EE903AF8EEE77A88EE277A84ED2B7A11
:102C9000D4ED2B0A31F0ACFC0028B5D0BCE700BF66
:102CA00094230020ED91002000000034FFF712BFB4
:102CB00070B500F5A046044696F9EC3F002B28DDE0
:102CC00007F0EAFF28BB04F5C2455435284685F0D5
:102CD000A7F9F0B1284684F0C5F8D0B196F056FABD
:102CE000D6F84035C01A96F9EC3F4FF47A72534348
:102CF00098420ED301221C212846FEF749FF40B11D
:102D000004F55050034ABDE87040062128305EF0BB
:102D100053BA70BD587A0D0800B52DED028B9FEDAA
:102D20000B8AD0ED4E7A67EE887A83B0C0ED4E7A8A
:102D3000383001907CF048F8019820EE080A03B082
:102D4000BDEC028B5DF804EB7CF056B952B87E3FC7
:102D500000B52DED028B9FED0B8AD0ED4F7A67EE1B
:102D6000887A83B0C0ED4F7A3C3001907CF02CF82B
:102D7000019820EE080A03B0BDEC028B5DF804EB6D
:102D80007CF03AB952B87E3F30B52DED048B83B05C
:102D9000044601A900F596501AF054FD002800F0F1
:102DA000B98004F5AA4595ED0A7ADDED017AB4EE15
:102DB000E77AF1EE10FA05F1280507D504F5C240CF
:102DC000543084F059F808B1019B2B6004F500558C
:102DD00095ED8F7AB5F9E831DFED606A052BB8BF64
:102DE000052307EE903AB5F9EA31F8EEE78A07EEE7
:102DF000903AF8EEE77AB6EE009A77EEA77A1820C6
:102E0000C7EE270ADFED567A68EEA77AF4EE490A94
:102E100087EE271AF0EE007AF1EE10FAB4EE671A98
:102E2000C8BFF0EE490AF1EE10FA48BFB0EE671ADB
:102E3000DDED017AF4EEE67AF1EE10FACCBF87EE22
:102E4000270AB0EE410A31F0E5FC04F5C3401C301E
:102E5000B0EE408A0FF034FC38B904F5C04393F863
:102E6000B022D2B393F8DD32BBB304F5C240543084
:102E700084F002F888B328EE892A9DED011AB4EE99
:102E8000C21AF1EE10FA28D5D5ED8F0ADFED351A0A
:102E90009FED350AC0EE820A31F0EEFB04F53E509C
:102EA0001C30B4EE408AF0EE408AF1EE10FA48BFD2
:102EB000F0EE488AFFF730FF04F54350343004F554
:102EC0004054FFF745FFD4EDE97A9FED287A67EE8D
:102ED000877AB0EE688AC4EDE97A254819F060FC7B
:102EE00090B924484021FFF7C7FD68B1224BD3F8C1
:102EF0009C35012B08D1F7EE007AB4EEE78AF1EEAB
:102F000010FA58BFB0EE678AB0EE480A03B0BDECC5
:102F1000048B30BD04F5C240543083F0ADFFB7EEF2
:102F2000008A0028D9D0462067F0A0FFB4EEC80A76
:102F3000DFED127AF1EE10FAD8BFB0EE480A87EE54
:102F4000800ABEF061F82F209FED0D1ADFED0D0A0B
:102F500031F060FCB0EE408ABFE700BF17B7D13850
:102F60003333333F000000006F12833A52B87E3F84
:102F7000003F0020402C0020407C00200000344214
:102F80008FC2D53F9A99193FF8B5044666F0C4FB45
:102F90000368DB689847054610B900252846F8BD48
:102FA00004F58046204607F0F3FCD6F8602F04F5C0
:102FB0009B4370339A42074605D104F5C04393F80A
:102FC0007033022BE9D804F5C3401C300FF09EFD8E
:102FD0000028E2D1D6F8600F03689B6B984758B978
:102FE00096F8743F002BD9D004F5005494F954524C
:102FF000023D18BF0125D1E7084BD3F8600F0368E5
:103000005B6B98470028EBD004F5005494F991329B
:10301000002BC2D0032BC0D03D46BFE7406C002040
:1030200070B52DED028B044600F5804600F5C340D7
:1030300006F57B6382B01C3093ED008A0FF07AFCBA
:1030400004F53E551C35002846D104F5C046D6F897
:10305000D00103689B689847D6F860345B0225D599
:10306000D6F8D03193ED437AD3ED097A67EE877ABB
:103070009FED327AF4EEC77AF1EE10FA16DB04F522
:10308000005404F57A6393ED007A67EE877AF7EEE1
:10309000006A86EEA77A04F69C74B4EE667AF1EEC6
:1030A00010FAC8BFB0EE667A84ED497ADFED247A73
:1030B00090ED250AF0EE480A20EE270A284685F012
:1030C00059FE28468DED010AFFF726FE9DED010A07
:1030D00002B0BDEC028B70BDD6F8602F04F59743AB
:1030E00050339A4228D104F50053D3F8683CB3F921
:1030F0000860003E18BF012604F5A04204F5805484
:10310000D2F8B035D4F8B8441C1B92F8AC353BB1BA
:103110000C484FF40061FFF7AFFC80F00100C3B230
:103120003246B0EE480A2146284602B0BDEC028B7A
:10313000BDE8704085F022BE0026DDE700000034C7
:10314000E02E6542402C002010B5044606F0DAFF60
:1031500098B104F5A042D2F8B03503F58C41503156
:10316000C2F8B01504F58051D1F8B8140029BEBFDB
:10317000A3F58C43503BC2F8B0352046FFF750FF13
:10318000BDE81040042067F05DBE00002DE9F04767
:1031900000F5C3442DED048B00F580491C34054631
:1031A00009F57B632046D3ED008A0FF0C3FB05F5DC
:1031B00043563436002844D105F5C044D4F8D00134
:1031C0000368DB689847D4F860345B0221D5D4F8F3
:1031D000D03193ED447AD3ED0B7A67EE877A9FED89
:1031E000537AF4EEC77AF1EE10FA12DB05F540558A
:1031F00095ED3E7A67EE877AF7EE006A86EEA77A5B
:10320000B4EE667AF1EE10FAC8BFB0EE667A85EDDC
:10321000877A90ED250ADFED467AF0EE680A20EE17
:10322000270A304685F000FA3046B0EE408AFFF7B4
:103230008FFDBDEEC80ABDEC048BB8EEC00ABDE838
:10324000F087204605F500580DF0EEFE9FED399A07
:1032500098EDA18A28EE098A05F5A047BDEEC88A37
:10326000D7F8B43518EE102A1A4408EE102A824610
:10327000462067F0FBFDB8EEC88AD8ED8B7AD9F806
:10328000600FA0EE278A05F5974350339842FDEE74
:10329000C87A17EE904A45D1D8F86C3CB3F908804B
:1032A000B8F1000818BF4FF00108BAF1000F1ED1A5
:1032B00003685B699847D0B9D9F8600F03689B6BC6
:1032C0009847A0B905F5C043D3F8F434022B0ED1CA
:1032D000284612F015FB50B107F6CC73D3ED007AF7
:1032E00067EE897AFDEEE77A17EE903A1CB205F5A3
:1032F0008055D5F8BC34E41A97F8AC353BB10E488C
:103300004FF40061FFF7B8FB80F00100C3B2B0EEEC
:10331000680ABDEC048B424621463046BDE8F047C2
:1033200085F068BA4FF00008BFE700BF0000003426
:10333000E02E65420000C842402C002010B5044633
:1033400016F0E0F868B100B200EB4000C0EB0013EB
:1033500000EE103AB8EEC00ABDE81040132067F046
:1033600071BD2046FFF712FFF6E7000010B51048C8
:10337000FFF70AFED0B10F480FF002FDB0B10E4CBE
:10338000042067F073FDD4F8680C66F035FC042067
:1033900067F058FD132067F069FDD4F86C0C66F0F7
:1033A0002BFCBDE81040132067F04CBD10BD00BFE2
:1033B000402C0020DC8D0020404C0020F8B52DED85
:1033C000028B0446FFF7E0FD002800F0AB8004F517
:1033D000804704F59842D7F8603F0832934200F0E6
:1033E000A18004F598424432934200F09B8004F59A
:1033F00099422432934200F0958004F5984260325D
:10340000934200F08F8004F598427C32934200F0A2
:10341000898004F59A427C32934200F0838004F55F
:103420009B42183293427DD004F59B423432934242
:1034300078D004F59B425432934273D004F59C42F9
:10344000103293426ED004F5C3401C300FF098FC4C
:10345000002867D0D7F8602F04F597436C339A4261
:1034600060D004F50055F6EE008AD5F8680C66F0D9
:1034700083FAB4EEE80AF1EE10FA40DDB0EE087A15
:10348000FFEE007AE0EE077AB0EE670AD5F8802CFE
:1034900004F5A04607EE902AD6F8B035B8EEE77AE4
:1034A00007EE903AF8EEE77A5142E7EE007AFDEE49
:1034B000E77A17EE900AC6F8B00531F04BFAC6F875
:1034C000B005D7F8602F04F59A4308339A4222D00A
:1034D000D5F86C0C66F050FAB4EEE80AF1EE10FA8A
:1034E000B0EE408A21DCFEEE007AB4EEE70AF1EE9F
:1034F00010FA22D5B0EE087AF7EE007A19E0FEEE67
:10350000007AB4EEE70AF1EE10FABFD5B0EE087A11
:10351000F7EE007AB6E725484FF48051FFF7ACFA92
:103520000028D5D0BDEC028BF8BDB0EE087AFFEED6
:10353000007AE8EE077AB0EE678A204606F0E2FDF0
:1035400008B1B1EE488AD6F8B435D5ED806A9FED62
:10355000186A05F6844595ED007AB5EEC08A07EE47
:10356000903AF1EE10FACCBF28EE268A27EE488A70
:10357000F8EEE77A66EE866AE8EE067A27EE067AD5
:10358000FDEEE77AFDEEE66A17EE903ABDEEC77AF9
:1035900016EE902A17EE101A17EE900AC6F8B435F8
:1035A00031F0D8F9C6F8B405BCE700BF402C0020C4
:1035B0000000C842F8B5044604F5C04795F0E6FDA2
:1035C00097F8B032064653B1D7F8D802036804F52D
:1035D000AB4204F5AB411B6A30323431984704F5F5
:1035E0008045D5F8703FF31AB3F5FA6F03D9D5F8D3
:1035F000600F08F0AFF82C4BC5F8706FD3F8600F70
:103600000268136898470021204612F02FFBDFED77
:10361000277AB0EEC00AB4EEE70AF1EE10FA42D50E
:10362000D7ED207AB1EE047AF0EEE77AF4EEC77ABD
:10363000F1EE10FA37D504F586601CF039FDF6EE90
:10364000007AB0EEC00AB4EEE70AF1EE10FA2AD51D
:1036500004F5B65595ED017AF0EE087AB4EEE77A06
:10366000F1EE10FA05F104051DD504F53E501C30AD
:1036700085F0F4FB04F54350343085F06BF904F524
:1036800049500C3086F098F895ED007AF7EE007A04
:10369000B4EEE77AF1EE10FA05D504F54F50BDE827
:1036A000F84085F0DFBDF8BD406C0020000000341C
:1036B00000F5005090F9DF31012BC3BF00F6185020
:1036C00090ED290ADFED047A9FED040AC8BF20EED1
:1036D000270A462067F0B6BB0000C8420000000081
:1036E0002DE9F8432DED028B00F5804909F57B6348
:1036F000D3ED008A054611F007FF8046D9F8600F28
:1037000003681B6A984705F549560C3698B14F4C2B
:10371000D4F87C35002B0EDD95F038FDD4F87C35DF
:10372000C01A40F6B733984205D8B4F97045304610
:1037300086F04EF87AE005F5C04305F5005793F89A
:10374000E93443B1B7F97032002B04DD05F540537D
:1037500093F9623203BBD9F8603F05F597455035C0
:10376000AB426DD00021B0EE680A304685F0C8FD4E
:103770000546042067F07AFB2BB207EE903A97EDEE
:10378000897AF8EEE77AE0EE077AFDEEE77A17EE4F
:10379000904A444424B2CAE72846012112F0A6F810
:1037A0009FED2B7AB7F97032C0EE077A05F5A04588
:1037B00005F2BC5508EE103A55F80C3C9FED250A71
:1037C000B8EEC88A28EE278A07EE903AF8EEE77A34
:1037D00067EE807A9FED200A27EE800ABDF038FA66
:1037E000B7F9E831DFED1D7A95ED007A20EE270A72
:1037F00007EE903AF8EEE77A0021B4EEE77AF1EEC0
:1038000010FA58BFF0EE477A80EE277A3046DFEDA7
:10381000147AB0EE480AA7EE270AF0EE680A85F09F
:10382000CBFEBDEEC00A10EE103A1CB2BDEC028B0E
:1038300020460C49BDE8F84341F2941231F09AB8A1
:10384000B8F1000118BF01218DE700BF407C0020C6
:1038500000A08C450AD7233C35FA8E3C0AE81C416F
:10386000E02E65426CEEFFFF38B500F5405305468B
:10387000D3F844060368DB689847014605F54F50C6
:1038800085F0D2FC04B22846FFF77EFB70B107EE4C
:10389000904A05F50055B8EEE70AD5F8740C66F0C5
:1038A000ABF9BDEEC00A10EE103A1CB22046034937
:1038B000BDE8384041F2941231F05CB86CEEFFFF85
:1038C00038B590F8E433B02202FB030393ED777A26
:1038D000F7EE007AB4EEE77AF1EE10FA054600F55D
:1038E000A0441DD5002112F0C1F9DFED417AB0EE00
:1038F000C00AB4EEE70AF1EE10FA11D5D4F89C35FF
:10390000012B0DD0072B0BD0002384F8143504F5C0
:10391000A364002323602846BDE8384011F0F4BDBD
:1039200095F034FCD4F81C35C4F81C05C31AB3F563
:103930007A7F84BF002384F81435284611F0E4FD13
:10394000D4F89C35012B07EE100A2CD0072B2AD077
:10395000B8EEC77ADFED276AC7EE267A05F5005282
:10396000B2F9342200EE102AB8EEC00A27EE800A1F
:10397000DFED1F7AB0EEC07AB4EEE77AF1EE10FA1E
:1039800013D4002384F8143594F8143505F54F50FA
:10399000DBB985F031FBBDE83840174900B241F290
:1039A000941230F0E7BF9FED150A94F81425002A11
:1039B000EAD10122934284F81425E5D0072B1EBFDB
:1039C00004F5A36300221A60DEE704F5A36494ED16
:1039D000007ADFED0B7A67EEC77A9FED0A7A67EE21
:1039E000877AFDEEE77A17EE901A85F01DFCD2E794
:1039F0000000003400A08C456CEEFFFF00000000CA
:103A0000E02E65420000C84270B52DED028B00F536
:103A1000BE46743682B00446304691F0E3FB05465C
:103A2000D8B904F50053D3F8682CB2F9082072B95C
:103A300004F5C042D2ED207A93ED8C7AF0EEE77A6D
:103A4000F4EEC77AF1EE10FA4CBF0125002530469E
:103A500091F0DCFB002808BF0025304691F0C2FB46
:103A600050BB04F5A043D3F8103501331ED01DBB65
:103A70009FED1C8A2046FFF733FE07EE900AB8EE52
:103A8000E70A8DED010AFDB9152067F0DBF99DED20
:103A9000010A1A2067F0D6F904F5C440243002B0B8
:103AA000BDEC028BBDE8704003F016BC002DDFD0EA
:103AB0002046FFF705FF02E02046FFF7D5FE07EEA0
:103AC000900AB8EEE78AD5E71A2067F067FC9DED0B
:103AD000010A08B9B0EE480A152067F0B3F9B0EE54
:103AE000480AD6E70000000010B500F5005303F6C1
:103AF0008442D3ED806ADFED127A92ED007A9FED79
:103B0000116A03F6185366EEA76A27EE277AD3EDFB
:103B10002A7A67EE867AFDEEE66ABDEEC77AFDEE9A
:103B2000E77A044616EE902A17EE101A17EE900A5E
:103B300030F010FF04F5A044C4F8B40510BD00BF78
:103B40000000C842A00CB34510B5044613F092FE25
:103B5000031E2ADB04F5005191F9DF219A4224DD8E
:103B600004F5A040D0F89C45022C1ED0D1ED8E7AF1
:103B7000DFED0E6AD31A66EEE76A07EE102A07EE4B
:103B8000903AB8EEC77AF8EEE77AD0F8B43587EE17
:103B9000876A07EE903AF8EEE77AE6EE867AFDEE6F
:103BA000E77A17EE903AC0F8B43510BD0000C8426D
:103BB00070B52DED028B00F5A0459FED550AD5F8A7
:103BC000B0359FED547A07EE903AF8EEE77A044666
:103BD00067EE807A9FED500AF0EEE76AF4EE476AEE
:103BE000F1EE10FAC8BFF0EE477A27EE800ABCF07B
:103BF0009FFE30F031FDB7EE008AC8EE007A05F581
:103C0000B76304F50056C3ED007A04F5C04393F89A
:103C1000B0229AB1D3F8D802036804F532515B6A36
:103C2000984758B1D6F8802CD5F8B005514230F0FD
:103C300091FEC5F8B005BDEC028B70BD96F910324F
:103C4000002BF8D0204606F05DFA0028F3D104F5E9
:103C5000C740543014F00CF80028ECD1B6F9E83124
:103C6000012BB8BF012307EE903A05F2BC52F8EEE3
:103C7000E77AD2ED006A86EEA77AB4EEC87AF1EE62
:103C800010FA13D840F6C4122449D5F8B00530F024
:103C900061FEC5F8B005D6F8802C40F6C4139A42F0
:103CA000D4BFC6F8802CC6F8803CC4E705F5B763DE
:103CB000D3ED007AF4EEC77AF1EE10FABBDD88EEB0
:103CC000070A20EE000ABCF0EDFFDFED157AD5F80B
:103CD000B00520EE270ADFED137A20EE270A40F622
:103CE000C413FDEEC07A17EE904A9C42B8BF1C4642
:103CF0002246614230F02EFEC5F8B005D6F8803C71
:103D0000A342D4BFC6F8803CC6F8804C93E700BFFE
:103D10000AD7233C0000AA4235FA8E3C3CF6FFFF4E
:103D2000E02E65420000C84210B500F5405304463D
:103D3000D3F8440603681B68984704F50053D3F88A
:103D4000802C514230F006FE04F5A043C3F8B005C4
:103D50002046BDE81040FFF72BBF00007047000071
:103D6000012070470820704701207047014B93F8ED
:103D70001C027047404C0020034B93F9240A003882
:103D800018BF0120704700BF404C0020014B93F941
:103D90001E027047404C002013B5064BD3F8600F4D
:103DA0004B690468009308310EC9646CA04702B0E7
:103DB00010BD00BF406C002070470000704700003D
:103DC00038B5264DD5F8600F03685B689847192809
:103DD0003CD8DFE800F00D39370D0D373737373B6A
:103DE0003939393939393B37373737393B0D393973
:103DF00040241B4B93F8212412B193F820340BB9C3
:103E000044F01004174BD5F8602F9A42A3F11C031D
:103E100003D09A4218BF44F01004134991F991025B
:103E2000B0B19A4216D0032803D101F533518A422A
:103E300001D144F040040D4883F014F850B144F02F
:103E4000800407E01024D4E71824D2E70124D0E747
:103E50009A42F0D144F0010038BD00BF406C002010
:103E6000405C0020A0790020404C0020948D002070
:103E700008B5044806F010FF00280CBF01200220FE
:103E800008BD00BF402C0020F0B52DED028B8BB09B
:103E9000054619F007FF4FF48071D0F8047290EDD9
:103EA000828AD0F80C6204461948FEF7E5FD30B965
:103EB000184BDFED197A93EDA17AA7EE678A1748C0
:103EC0000DF0E6F930B1164BD3F850345F6893ED3E
:103ED000028ADE682D7C95F059F9D4F81823D4F8BD
:103EE0001C33D4F814130892099327221C23CDE91C
:103EF00000320390079103AA1E21284604978DEDF6
:103F0000058A06965EF076F90BB0BDEC028BF0BD2B
:103F1000402C0020404C002035FA8E3CDC8D0020E7
:103F2000408C002038B5C5780B46352D044628BF97
:103F30003525352200211846BFF016F92A4604F12E
:103F40000C01BDE83840BFF0C5B8000008B5024814
:103F500013F090FC00B208BD402C002037B50D4690
:103F6000134840F2EF2204F06BF92C7814F00404AB
:103F70000AD0696803220F481FF084FC0C4803B084
:103F8000BDE8304003F0BEBA01AA214628461FF022
:103F90004DFD0028F2D0DDED017A9FED077A67EE46
:103FA000877A2246FDEEE77A17EE901AE3E700BF24
:103FB000402C0020948C00200000C84210B5054C15
:103FC000012384F823345FF0D9FD002384F82334DF
:103FD00010BD00BF405C002062F0DEBF2DE9F04163
:103FE0002DED028B4FF0000882B0CDE900281E4F66
:103FF0009FED1E8A0C461546B0EE480AB1F9022024
:10400000D7F8681C4FF47A73064663F0ADFA0123C3
:10401000CDE90053B4F90020D7F86C1CB0EE480A83
:1040200030464FF47A7363F09FFAB4F90420D7F85E
:10403000701C9FED0F0A43463046CDE9005863F0EF
:1040400093FACDE90058B4F90620D7F8741CB0EE05
:10405000480A4FF47A73304663F086FA02B0BDEC3A
:10406000028BBDE8F08100BF404C00200000FA4404
:1040700000007A4410B5074B93F9D82640F24D342E
:1040800040F24D13002A08BF1C465FF03DFB204361
:1040900010BD00BF407C002010B5044620F026F87B
:1040A000204610BD10B50B4C002384F8533560F04A
:1040B0005FFA54F8A02CA4F550739A4208D194F8F2
:1040C000C4352BB904F5B860BDE8104037F08EB8A0
:1040D00010BD00BF407C002013B5124C94F8761040
:1040E000A4F1D80017F01CF978B194F87610A4F177
:1040F000D80017F083FB40B194F87610A4F1D800F3
:1041000002B0BDE8104017F0BBBB19F0CBFD01A910
:1041100019F098FB18B19DED010A02B010BD9FED9A
:10412000020AFAE7404C002000000000044B93F81C
:10413000B00220B1D3F8D80203681B6B1847704750
:10414000408C002008B5084BD3F8102C002A03DC63
:10415000BDE808405FF01CBB03F533605CF01EFC5B
:1041600090ED000A08BD00BF404C002008B5124881
:10417000D0F8602F00F644539A4216D0B0F9783F39
:10418000ABB900F5805393F8DD2482B990F8752F10
:104190006AB993F8893563B9A0F5804006F07CFDD3
:1041A00000280CBF0320042008BD0220FCE70520E6
:1041B000FAE70620F8E700BF406C002010B5214B5D
:1041C00003F55662D3F8603F934290B0044636D070
:1041D00000231D4802931FF03FFB014618B91A48FF
:1041E00002AA1FF085FB247C94F0D0FF174BDDED75
:1041F000027A9FED177AD3E9172305930023F8EE8F
:10420000E77A0793089309930A930B930C930D9302
:104210000E934FF6F853ADF83C300023CDE903027E
:1042200067EE877A96228DF83E303323CDE900324F
:10423000572103AA2046CDED067A5DF0DBFF10B0D2
:1042400010BD00BF406C0020948C0020408C0020EA
:104250000AD7233CF0B58DB0044694F097FF184A76
:10426000D2F8D432C31A642B28D8D2F8D0310290B5
:10427000D3F88C10D3F89020D3F88460D3F888500A
:10428000D3F8DC70D3F894E0D3F898C0D3F89C301E
:10429000099300238DF82C30069225231622CDE9B0
:1042A00000320591207CCDF81CE002AA5321CDF804
:1042B00020C00A97039604955DF09CFF0DB0F0BDF9
:1042C000408C002010B55FF09BFC044678B909488B
:1042D00050F8A02C80F85345A0F550739A4206D1AF
:1042E00090F8C4351BB900F5B86036F07FFF204662
:1042F00010BD00BF407C00202DE9F0472DED088B5C
:104300008B4CD4F8602F04F556639A4290B0054662
:1043100000F0E7808748DFED888ADFED889A9FED1F
:10432000889A0CF0B5FF002867D082480CF04EFE4A
:10433000002862D004F500589FED820AD8F8D00119
:104340006C3033F0B9FB08F5D470B0EE60AAB0EE73
:10435000418ACDED070A8DED081AF0EE40AA8DEDE9
:10436000060A87F083FFD8F8D4310146D3F85C23DE
:10437000D3F85833059204A8049333F07BF909A8C5
:104380008DED090AB0EE680ACDED0A0A33F082F924
:1043900028EE288A02A8BDEEC88A95F81090CDEDC7
:1043A000030A18EE103A8DED020A1EB233F0E6F958
:1043B000DFED657A20EE270A02A8BDEEC00A6AEE9C
:1043C000A8AA10EE103A1FB233F022FAB4EEE90AAE
:1043D000F1EE10FA58BFB0EE690ABCEEC00AD4F88C
:1043E000602F10EE103A9DB204F67C539A422AEEEA
:1043F00028AA7BD1DFED558A7EE0DFF854A195F83D
:104400001090DAF844760AF500583846D8F8B035F6
:1044100007EE903AD8F8B435B8EEE7BA07EE903A1E
:104420003B689B68F8EEE7AA984707EE900AF8EE1B
:10443000E77A384667EEA87A08F5A768FDEEE77ACE
:1044400004F69C7417EE903A1EB23B681B699847BD
:1044500007EE900AF8EEE77A98ED00AA67EEA87AE0
:10446000B4EEE9AAFDEEE77AF1EE10FA17EE903A13
:10447000DFED327AAAF5405058BFB0EE67AA1DB200
:1044800003F024F93B68D4ED007A5B6908EE100A6A
:10449000384627EE899A9847B8EEC88ABCEECAAA71
:1044A0002BEE28BA6AEEA8AA1AEE103A68EE288A0D
:1044B0008DED09BACDED0AAACDED0B8A8DED0C9AE2
:1044C0008DED0D0AADF83860ADF83A50ADF83C30DE
:1044D000B7221A23CDE900323E2109AA48465DF0F1
:1044E00089FE10B0BDEC088BBDE8F087D8F8D43158
:1044F000D3ED0F7A67EEA88AD8F8D83104F69C7409
:10450000D4ED007A186927EE899A8CF081FECDED02
:1045100009AA8DED0AAACDED0B8A8DED0C9A8DEDD1
:104520000D0AADF83860ADF83A70ADF83C50CFE701
:10453000406C0020DC8D00200AD7233C00FF7F4721
:104540000000C8429F0CB345E02E65420000000009
:10455000405C002001480CF04BBD00BFDC8D00200A
:1045600008B5034BD3F8600F03685B68984708BD34
:10457000406C002030B587B0054619F093FB044627
:104580002D7C94F0F7FDD4F88422D4F8883204927C
:10459000059300211023CD22CDE900320290039132
:1045A00002AA42F60C3128465DF024FE07B030BD69
:1045B00030B52DED028B89B0054619F073FB00F57F
:1045C0005A7393E8070002AC84E80700DDED020AA5
:1045D0009DED030A2D7CF1EE600AB1EE400ABCF0BD
:1045E000C9FB2046B0EE408A33F0EAFEDFED0B7ADD
:1045F000049B079328EE278A0C230122CDE9003281
:10460000A82105AA28468DED058A8DED060A5DF0E4
:10461000F1FD09B0BDEC028B30BD00BFE02E65425C
:10462000282938B5054623D007D824292BD0272997
:1046300011D01B2908D1012413E0432937D008D811
:104640004029F8D0422928D02846BDE8384063F0F8
:10465000F7BA5329EEE712215CF0CAFF044610B9FD
:104660000024204638BD297C134855F02BFFF8E77D
:1046700016215CF0BDFF04460028F1D0297C0E48CD
:1046800055F0FAFFEDE70C215CF0B2FF044600287C
:10469000E6D02846FFF78CFFE3E710215CF0A8FF87
:1046A00004460028DCD02846FFF764FFD9E7017CE8
:1046B000024890F095FDBEE718830020B48B0020DF
:1046C000F0B52DED028B05468DB01646B0EE408A52
:1046D0000C46002930D0007C5DF022FD0746287C86
:1046E0005EF022FC00F121039F4207D2287C0DB02E
:1046F000BDEC028BBDE8F0405CF068BF63690893D5
:10470000636A2269CDF82530236AA069E1680792BF
:10471000CDF829306222212327680590CDE90032A7
:104720000691287C0397192303AAC2218DED048AE0
:104730008DF824605DF05EFD0DB0BDEC028BF0BD28
:10474000F8B54B4CD4F8602F04F556639A420546F1
:1047500000F08C80A4F50056B6F8C232DF0713D5FE
:1047600044480DF0ADFF002879D004F50054D4F88A
:10477000D00103689B68984700F1940191ED010A0C
:1047800001222846FFF79CFFB6F8C2329C0712D5DB
:1047900038480DF095FF002864D0374BD3F8D0018E
:1047A0000368DB68984700F1940191ED010A022249
:1047B0002846FFF785FFB6F8C232580712D52D48B4
:1047C0000DF07EFF00284FD02B4BD3F8D0010368AB
:1047D0001B69984700F1940191ED010A03222846D4
:1047E000FFF76EFFB6F8C232190708D52349052234
:1047F00091EDFD0A284601F57C71FFF761FFB6F8DF
:10480000C232DA0616D51E4FD7F89C35042B11D1CB
:1048100019F048FA044607F6747090F011FD94ED13
:10482000C70ADFED187A014620EE270A062228463D
:10483000FFF746FFB6F8C2329B0617D50D480DF0BC
:104840003FFF98B10C4BD3F8D411284691EDAB0A39
:10485000BDE8F840042201F52A71FFF731BFA4F644
:104860003C718BE70849A0E70849B5E7F8BD00BFF0
:10487000406C0020DC8D0020408C0020405C00203B
:10488000407C0020E02E6542605E0020D45F002066
:1048900070B504460E4628F069FD90F8C412B023A6
:1048A00003FB0101AC31204603F02CFE0546C0B1EC
:1048B0003EB119F0F7F990F87C3243F0020380F82A
:1048C0007C3204F58043D3F8600F04F599436C33D0
:1048D000984204D004F59B447034A04201D106F004
:1048E0005DFE284670BD000073B516460191044672
:1048F00019F0D8F9019918F0EDFD0546C0B13EB1A7
:1049000019F0D0F990F87C3243F0020380F87C3241
:1049100004F58043D3F8600F04F599436C33984253
:1049200004D004F59B447034A04201D106F036FE59
:10493000284602B070BD000030B5054685B00C4673
:10494000D1E9040131F06AF840B168461EF094FFE5
:104950006A462146284662F077FD08B9022067E0E2
:10496000344840F24F32694603F06AFCD4ED037AD2
:10497000F4EE677AF1EE10FA22D69FED2F7AF0EE80
:10498000E77AF4EEC77AF1EE10FA54BF0122002262
:104990009DF80030294962F3410368468DF80030E4
:1049A0001FF0D4F80028D9D12548694671F07AF86B
:1049B00040B959F037FB0522162159F0EBF8CDE745
:1049C0000022E5E7D4ED017AFDEEE77A17EE903AA2
:1049D000DB0706D41B4B03F62452D3F8603F934207
:1049E00025D119491348022212F04CFD9DF8001000
:1049F00011F0040102D168461FF008F80D4869461D
:104A000003F0D0FC94ED020AB4EE400AF1EE10FA85
:104A10000BD6B5EEC00AF1EE10FA06DD9DF80010D7
:104A20000948C1F3400107F0A9FF002000E004207D
:104A300005B030BD402C002000000034848C0020E4
:104A4000204D0020406C00206479002010B52DED31
:104A5000028BD1ED017A91ED008AFCEEE77A8AB003
:104A6000CDED037A9DF80C1005AA044662F0D6FC41
:104A7000C8B1DFED0E7A059B009368EE277A00221D
:104A8000FDEEE77A114617EE903A06A81EF014FFE5
:104A900023682046D3F8CC3006A9984700200AB0F6
:104AA000BDEC028B10BD0220F9E700BF0000C84238
:104AB00037B5124DD5F8600F03681B6A0C4698474E
:104AC00040B9D5F8602F05F54C639A4202D0042016
:104AD00003B030BDD4ED007AD4ED020A94ED010AA2
:104AE0000748FCEEE77ACDED017A9DF8041004F05A
:104AF0009DF90028EBD00020EAE700BF406C0020C1
:104B0000402C0020134610B524220C4618460021E4
:104B1000BEF02AFBA27F8277E27FC277072280F86D
:104B20002020A28B8283D4ED067AF1EE677AC0ED65
:104B3000067A10BD10B48C8B162C03D15DF8044B93
:104B4000FFF7E0BF5DF8044B61F0F8BD08B591F8E0
:104B50002030072B0ED1094890F8B03243B191EDC7
:104B6000060A00F5CE70B1EE400A0DF071FB18B9DF
:104B7000042008BD0220FCE70020FAE7408C00205A
:104B800008B5D1ED007A9FED087A0848F0EEE77A93
:104B9000F4EEC77AF1EE10FA54BF0121002105F0BE
:104BA000ABFA002008BD00BF00000034402C0020FC
:104BB00010B5D1ED007AFCEEE77A17EE903A9CB290
:104BC000012C02D0022C06D084B9114821466BF08A
:104BD00073FE002010BD0F4890F8CC365B0707D558
:104BE00063F0D0FA0C4A05215CF0E6FA0420F1E704
:104BF00090F9B8361BB963F0C5FA084AF3E7A0F597
:104C0000A0400AF06DFE002814BF00200420E1E758
:104C1000F8820020407C002018800D0833800D08A9
:104C20001FB5D1ED017AFCEEE77A0B46CDED027AA5
:104C3000D1ED007A1A7C017C0192FCEEE77A0B48F8
:104C4000CDED037AD3ED027AFCEEE77A17EE902AE7
:104C500092B2009293ED030A9DF80C209DF8083063
:104C600009F0A4FF05B05DF804FB00BFDC8D002057
:104C700007B5D1ED007A0848FCEEE77ACDED017A70
:104C80009DF804100BF0BAFD00280CBF0420002092
:104C900003B05DF804FB00BFDC8D002070B58B8B8A
:104CA000C02B05460C4633D8B12B0DD8142B00F081
:104CB000AE80162B59D0112B00F0A6802146284635
:104CC000BDE8704063F080BEB23B0E2BF6D801A168
:104CD00051F823F0594D0108BD4C0108BD4C0108A5
:104CE000BD4C0108BD4C0108BD4C0108BD4C01087C
:104CF000BD4C01084F4D0108BD4C0108834D010812
:104D0000BF4D0108BD4C0108734D0108454D010818
:104D1000D42B13D007D8D02B23D0D12BCED1BDE8A4
:104D20007040FFF77DBFB3F5967F53D040F6B8369D
:104D3000B342C3D1BDE87040FFF79ABFBDE87040F1
:104D4000FFF71EBF2146BDE87040FFF7F5BD2146C5
:104D5000BDE87040FFF77ABE2146BDE87040FFF71E
:104D6000A7BEBDE87040FFF723BFBDE87040FFF766
:104D7000EDBE94ED000A2848FDF7B4FBE8B1002031
:104D80001CE0264C94F8913FBBB1254904F5AE5088
:104D900036F02AFB88B104F58053012283F8F92507
:104DA00004F54C610222A4F5804012F06BFB002850
:104DB000E5D11C4B002283F8F925042070BD174C67
:104DC00094F8913F002BF8D0154904F5AE5036F019
:104DD0008FFADFE7D1ED007A9FED137AF0EEE77AF4
:104DE000F4EEC77AF1EE10FA14D5D1ED017AF0EEB7
:104DF000E77AF4EEC77AF1EE10FA0BD50B490222EE
:104E0000054812F03FFBBAE709490222F8E70949D1
:104E10000222F5E70220D1E7402C0020406C002060
:104E2000848C0020407C00200000003400790020A9
:104E3000487900202C79002070B5434B03F62452AA
:104E4000D3F8603F93428EB00C467BD1CD78272DAE
:104E500028BF27252722002104A8BEF085F92A466D
:104E600004F10C0104A8BEF035F9059B9DF836400D
:104E70000093069B0193E443079B0293E4B2089BD3
:104E800003938DF8364094F081F914F0810F04F00B
:104E90008705064601D1802D13D1684632F054F9BA
:104EA000DFED2A7A2A4B20EE270ADFED2A7AC3F8B3
:104EB000746520EE270ABDEEC00A10EE102AC3F872
:104EC000682514F0820F01D1802D13D1684632F08D
:104ED00055F9DFED1E7A1E4B20EE270ADFED1D7A15
:104EE000C3F8786520EE270ABDEEC00A10EE102A3E
:104EF000C3F86C2514F0840F01D1802D13D16846BE
:104F000032F04CF9DFED117A114B20EE270ADFED7C
:104F1000117AC3F87C6520EE270ABDEEC00A10EEB8
:104F2000102AC3F8702563060CD5DDED0C7A9FEDD1
:104F3000097A074B67EE877A03F5B062C2ED007A13
:104F4000C3F884650EB070BD406C0020E02E654251
:104F5000407C00200000C84230B51E4C91B008468D
:104F600002A9FEF7DFFFD4F8602F04F624539A421B
:104F70002DD19DF83C30072B29D104F50054D4EDF8
:104F8000167ADDED056A9FED147AF8EEE77AE6EE23
:104F9000C77AFDEEE77AC4ED167A63F0F3F8226B78
:104FA000A36D52689FED0D7A9B1A07EE903AF8EECA
:104FB000E77A054667EE877A17EE900AFBF7A4FAC0
:104FC000074ACDE90001062128465CF0F5F811B04A
:104FD00030BD00BF406C00200000C8420AD7233C0F
:104FE0004C800D0810B51D4B03F62452D3F8603FDA
:104FF0009342044696B008460FD108A9FEF792FFE7
:105000009DF8541003AA204662F008FA38B963F0FC
:10501000B9F8134A04215CF0CFF816B010BDBDF802
:10502000503023F004039BB2002BF6D0DDED0B7A59
:105030009FED0C7A039B009367EE877A0022FDEECA
:10504000E77A114617EE903A04A81EF035FC236863
:1050500004A9D3F8CC3020469847DEE7406C002006
:1050600060800D080000C84230B48D7A4B7A43EA64
:105070000523CD7A43EA0543562B04460A461BD046
:1050800008D8522B12D0542B13D02046114630BCD6
:1050900062F0CCBA03F18073863B23F07F43012B8F
:1050A000F3D8017C064830BC55F0AEBB30BCFFF7EE
:1050B000C3BE30BCFFF750BF30BCFFF793BF00BF8B
:1050C0001883002000207047C820704701207047D7
:1050D000002070470020704790F890308B4286BFC8
:1050E00000EB8100D0F894000020704790F89030D9
:1050F0008B4286BF00EB8100D0F8940000207047FF
:1051000003207047014B93F81A027047404C00206F
:1051100070B504464C4810F0A3FD18B1236A43F45F
:1051200000032362484810F09BFD88B1462065F0DB
:105130009DFEDFED467AB4EEE70AF1EE10FA07D8ED
:10514000636A43F400036362A36A43F40003A36247
:10515000236A43F4F84323623D4BD3F8600F03689E
:105160005B6898470138182815D8DFE800F03B4302
:105170000D4543434343143B3B3B3B3B3B144343C1
:1051800043433B14453B3B00324A92F820348BB3F7
:1051900092F821248AB3304B93F8703F012B3DD015
:1051A000022B44D02D4B1D68DDB12D4E284696F8BC
:1051B0005A1C4FF029FAA0B1236A43F4807323628A
:1051C00096F9C0321BB1636A43F48073636296F848
:1051D0005A1C28464FF050FA18B1A36A43F4807362
:1051E000A36270BDD4E9092342F4E04243F4E043F2
:1051F0006262A362012300E00023616A41F48062DD
:105200006262A26A42F48060A062002BC3D041F4C3
:10521000406142F440626162A262BCE7236A43F4E7
:1052200080032362636A43F480036362BAE7236AFC
:1052300043F480032362636A43F480036362A36AD6
:1052400043F48003A362ADE7402C0020000000B4CB
:10525000406C0020405C0020407C002094920020A4
:10526000404C002013B54FF44470CDE900211EF0EE
:1052700035FF044628B1DDE9002162F0A1FF024BB1
:105280002360204602B010BD60820D0800207047E8
:1052900000207047002070470020704700F509503B
:1052A0003C30704700487047A4A80D0800F58040C6
:1052B000D0F8600F03685B681847000000F5804372
:1052C00000F59940D3F8603F40301B1A58425841CE
:1052D00070470000A22070472DE9F04100F5A0437F
:1052E00003F2B45353F8042CDFED666A07EE902AFC
:1052F000B8EEE77AD3ED007AF8EEE77A00F5C34826
:1053000090B027EE267A67EEA67A08F11C080446CC
:10531000002340468DED017ACDED027A03930BF028
:10532000B7FF04F5C046002800F0A680D6F8D031BB
:1053300084330FCB0CAF87E80F0008AD04AF87E8CC
:105340000F0085E80F0001A9384603AB02AA31F02F
:105350003FFF9FED4D0AD6F8507401A832F0ACFB28
:10536000294638468DED080ACDED090A8DED0A1A59
:1053700016F092FD93F00AFFD6F8D432C01A6328D3
:1053800004F57C652DD8D6F8D00103689B68984752
:10539000042100F19402284657F010FDD6F8D00100
:1053A0000368DB689847052100F19402284657F00E
:1053B00005FDD6F8D00103681B699847062100F166
:1053C0009402284657F0FAFCD6F8D421284602F574
:1053D0002A72072157F0F2FC04F5C740543013F04D
:1053E000AFFC40460DF06CF990B1D6F8D4018BF0CB
:1053F000EBFB68B1D6F8D4216E219032284657F0E5
:10540000DDFCD6F8D4216F21BC32284657F0D6FCFB
:1054100004F5435204326921284657F0CFFC04F5C5
:10542000485220326A21284657F0C8FC04F5405300
:1054300093F9622232B9D3ED967AF5EEC07AF1EEA5
:1054400010FA06DD04F54E5214326B21284657F04F
:10545000B5FC04F54F54204683F008FF28B104F151
:1054600030026D21284657F0A9FC18F01BFC18F0FB
:105470002DF910B0BDE8F08101A904F5965016F0A1
:10548000D3FB77E70AD7233CE02E654210B54FF4F3
:105490008011044612F0EAF910B12046FFF71CFF14
:1054A0004FF48001204612F0E1F928B12EF07AFC89
:1054B000BDE810402CF03ABE10BD000030B591B0F0
:1054C000002300F59655029302A9002304460DF12E
:1054D000070228468DF8073018F0BAF903A92846C4
:1054E00017F0AEF908B92E4B03933022002104A81F
:1054F000BDF03AFEA3238DF8103095238DF81130BE
:1055000093F04CFE04F5A042CDF81300D2F8B0356C
:10551000ADF81B3004F58053D2F8B425CDF8171040
:105520004620D3F8B814D3F8BC34ADF81D10ADF84C
:105530001F20ADF8213065F099FC10EE103A1520CF
:10554000CDF8233065F092FC10EE103ACDF82730FC
:1055500004F534539FED137AD3ED2F7A67EE877AF3
:10556000284617EE903ACDF82B30029BCDF82F301D
:105570009DF807308DF83330039B0D9318F06EFBC8
:1055800004F580433022D3F8A43F8DED0E0A04A920
:1055900004F57C600F9357F04DFD11B030BD00BF96
:1055A0002292CA7F0000C84230B58FB0352204462F
:1055B00000216846BDF0D8FDA3238DF80030952367
:1055C0008DF8013001238DF8023093F0E7FD04F5EA
:1055D000AA4304F540553833CDF803001B68D5F8CD
:1055E0004406CDF80710CDF80B3003681B699847C7
:1055F000ADF80F00D5F8440603689B689847ADF8EE
:1056000011001C4802F062F8ADF81300D5F844060A
:1056100003685B69984710EE103AD5F84406CDF858
:10562000153003689B69984710EE103A04F58041E5
:10563000CDF8193001F69C7335221B68CDF81D306A
:1056400004F5C043D86DCDF82100186ECDF82500C3
:10565000986DD3F8FC34CDF82900CDF82D3004F541
:105660007C60D1F8943FCDF83130694657F0E2FCC8
:105670000FB030BD402C002030B587B01622044654
:1056800000216846BDF070FDA3238DF800309523FE
:105690008DF8013002238DF8023093F07FFD04F580
:1056A000A045CDF803002046CDF8071005F0F4FA28
:1056B00005F5B4638DF80B001B680393124B1B6850
:1056C000D86A90F89C308DF810300368DB699847F1
:1056D00095F889358DF812308DF811002EF062FBA7
:1056E0002DF0B0FCD5F89C358DF813008DF81430F2
:1056F000162295F88A358DF81530694604F57C60D8
:1057000057F098FC07B030BD3C2C002010B58AB093
:105710002722044600216846BDF026FDA3238DF80C
:10572000003095238DF8013009238DF8023093F075
:1057300035FDCDF803000420CDF8071065F096FB89
:1057400010EE103A1320CDF80B3065F08FFB10EE01
:10575000103A4620CDF80F3065F088FB10EE103A75
:105760001520CDF8133065F081FB10EE103A0320C0
:10577000CDF8173065F08AFB10EE103A1A20CDF8FC
:105780001B3065F073FB10EE103ACDF81F3004F5B6
:105790009F43303327221B68CDF82330694604F538
:1057A0007C6057F047FC0AB010BD000013B50446FA
:1057B00000F57C60019056F06FFF019857F006F8F5
:1057C00004F58053019893F9D4300BB157F0A6F843
:1057D000204602B0BDE81040FFF798BF70470000B8
:1057E00030B500F5C04389B093F8B022044600F507
:1057F0007C6552B1D3F8C8011E2269468DF014FBB6
:105800000F496A46284657F0B1FD04F58043D3F8A6
:10581000600F03685B68984704F50053014693F8EE
:105820009C21284657F0C6FD04F5965018F0B4FCAC
:1058300004F5907009B0BDE8304026F001BE00BF0D
:1058400074830D089FED020A00224CF0C9BF00BF0F
:105850000AD7233C134B70B5044640F8043B63F071
:10586000DBFD114E114B63605425601963F08AFF14
:1058700066513035B5F5557FF7D104F5557065F0B3
:1058800043FF0B4A04F5EC6002F63C3190F034FB28
:1058900001232046074984F891394DF09FFB2046AB
:1058A00070BD00BF80380020FCD30D0810D40D0857
:1058B0001C4E0020BCC30D082DE9F04100F5085135
:1058C0009AB00D221831044655F0D2FF0022C0488C
:1058D00027214CF0FDFE0421002065F09FFE1321DE
:1058E000012065F09BFE4621022065F097FE152100
:1058F000032065F093FE65F009FC04F5C04393F9BD
:10590000683223B19FEDB30AB3484DF00FFF4DF05D
:105910006BFDB24AB24E138843F0040313804FF07C
:1059200000080AAF002110223846BDF01DFC0123FB
:105930008DF830303388ADF8283005A973680B93A3
:1059400038464CF0CDFDC8B19DF91430002B15DD63
:1059500063F0E2FE9DF81410036801391B68C9B2B8
:10596000984758B1051D28464CF058FD30B9B3682A
:10597000ADF8183006A928464EF0F2F908F10608ED
:10598000B8F12A0F06F10C06CCD1964800220DF191
:105990000B014CF02BFB06AD064620B34CF03EFD50
:1059A00008BB914B0FCB85E80F0004A928464CF0AB
:1059B00097FD002840F03B814FF004088B4B0FCB44
:1059C00087E80F0005A938464CF08AFD28B105A8E4
:1059D0004CF024FD08B148F0010803A930468DF8C9
:1059E0000C804EF06BF9824B0FCB85E80F0003A9BA
:1059F00028464CF075FD002846D00998002204A9DD
:105A00004CF0F4FA064600283ED04CF007FD05465F
:105A1000002839D19DF80C30013BDBB2032B96BF37
:105A2000744A0346D35C8DF82830304639464EF030
:105A300045F97148002205A94CF0D8FA064670F0E5
:105A400073FA78B170F06EFA90F8302090F8281060
:105A500090F84830114490F840200A44D34214BFD3
:105A60000125002586B130469DF90C804CF0D6FC0E
:105A700050B91DB1B8F1000518BF012539463046AF
:105A80008DF828504EF01AF904F50A500022B7EEAE
:105A9000000A012134304CF0A3FE04F50950002225
:105AA000B7EE000A022110304CF09AFE012304F5F3
:105AB000F9510093514A002308318E204CF00CFE1E
:105AC00094F974C9BCF1000F1AD14D4E0FCE3D466A
:105AD0000FC50FCE0FC50FCE0FC596E80F0085E896
:105AE0000F006246042138464CF0F2FD9FED450A56
:105AF00045484DF01BFE4548B7EE000A4DF016FE36
:105B0000012504F50351424A00950023203140F25B
:105B100005104CF0E1FD04F50A5002210430FFF7B6
:105B200091FE04F5075003212C30FFF78BFE04F59E
:105B3000075003213430FFF785FE032104F50A5096
:105B4000FFF780FE04F50A5002210830FFF77AFEC5
:105B5000022104F50850FFF775FE04F508500221F4
:105B60000430FFF76FFE04F5075002213C30FFF7C9
:105B700069FE04F5BE4074308FF0C6FC254A1368F8
:105B8000D90705D42449156004F5025308330B6086
:105B900004F50B5020490122083001254CF0EEFDA0
:105BA0001E4A0095002304F57C61FD204CF094FD15
:105BB0001B4B1A68D20705D41A4A1D6004F58F548E
:105BC00008341460174801214CF0F4FD2CE000BFAC
:105BD000F8C00D0800009643A4AE0E08789200208D
:105BE00068C30D08BCC00D08EC730D08FC730D08EC
:105BF0000C740D08F4C00D08C7C00D0864050E082C
:105C00001C740D0800000000D4C00D08E3C00D088E
:105C1000A80D0F08342C002000220020D8940E0874
:105C2000382C00200C2200201AB0BDE8F08104A816
:105C30004CF0F4FB00283FF4BFAE4FF00C08BDE67B
:105C40007047000000207047002070470020704718
:105C50000020704700207047704700000020704708
:105C60000020704784B001A880E80E0004B0002036
:105C70007047000000207047002070477047000008
:105C80001020704700487047F8CF0D080048704753
:105C900008D00D08002070477047000001207047B1
:105CA0000120704700207047002343608360C36079
:105CB00003614361002303767047000010B504467A
:105CC000FFF7F2FF0023637610BD0000027E531C35
:105CD000DBB2042B037600EB820288BF002382ED47
:105CE000010A88BF0376704710B50446FFF7EEFF40
:105CF000D4ED017A9FED107A94ED020A637E77EE7F
:105D0000877A042B77EE807A94ED030A94BF0133EF
:105D1000052377EE807A94ED040A637677EE807A35
:105D2000637E94ED050A77EE807A00EE103AB8EEC5
:105D3000C00A87EE800A10BD0000000010B50446BE
:105D40001EF0D4F9204610BD04F0BABC03F0E0BA4E
:105D500004F094B803F0EABA01F0B4BF01F01CBB40
:105D600001F09EBC01F0DEBCFCF7A2BFFCF74ABB11
:105D700070B51F4B036000F540530446D3F8D805B7
:105D80001C4AC3F8282408B11EF0B4F91A4B23604A
:105D900004F5805393F8C42E42B9D3F8C05E2DB1F8
:105DA00028462BF04BFA28461EF0A0F904F58E5039
:105DB0000C3080F09DFB04F58650143066F0A4FD95
:105DC00004F6C44504F66446B54204D0183D28469E
:105DD0002AF08AFEF8E7094BC4F8983804F69410C4
:105DE0005AF0B8FA04F510605AF0B4FA204670BDC3
:105DF0003CB70D08C0AF0E08BC8D0E089C530E08B2
:105E000038B5474B044640F8043B68F0FFFF04F107
:105E100010001BF0CBFA04F1680053F08BFC04F582
:105E2000907025F0EFFE04F586601AF017F904F281
:105E300054501EF061F904F698002CF063FA04F552
:105E4000446068F0C1FD04F551604EF003FB04F5B9
:105E50007C6057F023F804F58650143066F03CFD62
:105E600004F5885010301CF0BBFE04F58E500C3049
:105E700080F02AFB04F58F50083054F01DF804F52B
:105E800091501C306AF0A0F904F5805304F5935248
:105E90000025104683F86052224B10301A6049F0FA
:105EA00055FF294604F5965016F0ACF904F5C85094
:105EB000103079F05FF904F5EA5014307DF04AFBB8
:105EC00004F5F3500C307FF059FC04F5F650103017
:105ED00080F08EF804F5F950083015F0B5F804F5A7
:105EE0000250083079F04CFE04F5035020306FF07A
:105EF000F1FA04F5005304F5065083F89C510A4D5D
:105F0000343080F0B5FE2B6813B1084893F00CF9DB
:105F1000204607494DF062F82C60204638BD00BF8E
:105F2000BC8D0E08789B0020CC92002010D00D086C
:105F3000E48C0E082DE9F04F2DED028B04469FB046
:105F4000FFF75EFFE24B236004F50B500830FFF7CC
:105F500081FC04F53150203004F5005782F012FA2C
:105F600004F509532233C7F8883C04F53250062360
:105F700087F88C3C343066F0C1F804F5BE437433C6
:105F8000C7F8303D0E934FF40063C7F8343D5A23F1
:105F900087F8B43D04F5075807F6185308F11C08B4
:105FA000CC4AC7F82C8D04F5965BC7F828BDC3F81A
:105FB0006021C94AC3F86421B7EE008AC74AC3F812
:105FC000682104F53B50C3F8CC2183ED578A343067
:105FD0005AF0E0FC04F5345A04F53C505AF0DAFC6F
:105FE0000026BF4BC7F8103F0AF1180A87F8286F40
:105FF0000AF5FC70FFF758FEBA4BBB49C7F8103FD3
:1060000087F8296F50464CF0E9FFB84BC7F8303F8E
:1060100007F573630022C7F834BFC7F838AF04F53B
:106020003C555A63DA6304F53E50012387F8743F08
:10603000303508301DF020FC87F8986FAC492846B1
:106040004CF0CCFF04F53E5041461C3082F050FD30
:1060500004F543504146343082F0AEF904F549501E
:10606000414604F540570C3083F00CF92C223146A0
:1060700007F57C70BDF078F804F550569D4904F59D
:106080004F504CF0ABFF28369B4BC7F8283406F135
:10609000080091F02FFF04F5515904F5525309F10E
:1060A0001409383348460F935FF034FA0F9B09F117
:1060B00014094B45F6D10723C7F8DC350023A7F8B0
:1060C000E0354FF4CB701EF00FF8C7F8D80504F593
:1060D0005750243091F00EFF04F55850283091F0BD
:1060E00009FF864B1A6802B91E60854BC7F8283431
:1060F00004F559504FF48051C7F8445608301BF04E
:1061000057FA04F55B5008304DF0E0FE04F55B50A3
:106110001C3071F085FA04F5974004F58045343061
:1061200005F010FA774BC5F8B43B04F597405030B2
:1061300005F008FA744BC5F8D03B04F597406C3075
:1061400005F000FA714BC5F8EC3B04F598400830B7
:1061500005F0F8F96E4BC5F8083C05F543630022DD
:1061600004F59840DA609A605A6083ED008A443002
:1061700005F0E8F9674BC5F8443C04F598406030F9
:1061800005F0E0F9644BC5F8603C04F598407C30BC
:1061900005F0D8F9614BC5F87C3C04F599402430F2
:1061A00005F0D0F95E4BC5F8A43C04F599404030A9
:1061B00005F0C8F95B4BC5F8C03C04F599406C305C
:1061C00005F0C0F9584BC5F8EC3C04F59A4008308E
:1061D00005F0B8F9554BC5F8083D04F59A40243050
:1061E00004F59A4605F0AEF94436514BC5F8243D06
:1061F000304605F0A7F94F4BC5F8443D04F59A40E9
:10620000603005F09FF94C4BC5F8603D04F59A40AD
:106210007C3005F097F9494BC5F87C3D04F59B406F
:10622000183005F08FF9464BC5F8983D04F59B40B2
:10623000343005F087F9434BC5F8B43D04F59B4075
:10624000543005F07FF9404BC5F8D43D04F59B4030
:10625000703005F077F93D4BC5F8F03D04F59C40F2
:10626000103005F06FF93A4BC5F8103E04F59C402C
:106270002C3005F067F9374BC5F82C3E04F59C40EF
:10628000483008F0E5F904F59D40043005F05AF96E
:10629000314BC5F8843E314BC5F8A03E04F59D4016
:1062A0004FF4C053A5F8F43E2D4920304CF096FE33
:1062B000FE2385F86C3F052385F8903F4FF0FF33B0
:1062C000C5F8983F274BC5F8606FC5F8646F4BE081
:1062D0003CB70D08000080BF0000B4420000B4C20B
:1062E00048D00D0858D00D08CC470F0840450F087E
:1062F000E8440F0840430F08C0AF0E08E89500209F
:106300003C830D08B0DB0D08ACE20D08CCE50D08B0
:10631000ACD90D08C0DC0D0848DD0D0828DC0D08DF
:1063200030DB0D08ACDA0D083CE20D0838DE0D0854
:10633000C8DD0D0890D00D08B8DE0D08C4E10D08C9
:10634000B8DF0D08A8E00D0828E00D0840E10D08B1
:1063500038DF0D083CD90D0848E50D0880D00D0840
:106360008C680F08495D0108119305F57B65934B17
:1063700085ED008A04F59F4004F5A0454FF40071B7
:10638000009322468E4B109434301AF067FB4FF086
:10639000FF33C5F8103505F5A4638A4ADA60032394
:1063A0000026C5F89C3505F5B763C5F86865C5F8DE
:1063B0006C65C5F87065C5F87465C5F87865C5F88D
:1063C0007C6583ED008A804BC5F8E0357F4BC5F8CE
:1063D000E83504F5AC407E4BC5F8F035C5F8DC4532
:1063E000C5F8E445C5F8EC4504301DF045FA04F560
:1063F000AC4020301DF040FA04F5AC403C301DF0BC
:106400003BFA04F5AB49734BC5F8503609F1400926
:106410004FF0FF33A5F8543609F198001DF02CFA1F
:106420004FF0FF326C4BC5F8B4266C49C3F80090AE
:1064300048464CF0D3FD4FF6FF73A5F8FC354FF0FE
:10644000FF33A5F8183604F5AD40654B6549383083
:1064500018604CF0C3FD04F5AD40583054F0FCFD1D
:10646000614BD7F844261294CDE913345F4BCDE944
:1064700015345F4BCDE917345E4BCDE919345E4BD3
:10648000CDE91B345D4B1D931EA911E903000CAB34
:1064900083E80300DDE91A010AAB83E80300DDE9C4
:1064A000180108AB83E80300DDE9160106AB83E8B9
:1064B0000300DDE9140104AB83E80300DDE9120108
:1064C00002AB83E8030004F5C0474946CDE9002844
:1064D00053465A460E988EF021FE0BF51B73384634
:1064E0003B6334301DF0C8F9384644301DF0C4F920
:1064F000384654301DF0C0F91C22314607F16400C3
:10650000BCF032FE04F5C24804F5C14008F154085D
:10651000503066F01DFB404680F064FC384B394932
:10652000C7F8543140464CF059FD374A374911609D
:1065300004F5C3430C334FF0140CB0B20CFB001243
:106540000136127C002AF8D1314A1080314A16688F
:1065500016B1314892F0E8FD04F5C34010301360E5
:1065600080F02AFC2D4BC7F8903104F5C340594602
:106570001C3009F07DFB2A4BC7F89034642387F860
:106580009434284BC7F8C83404F5C940264BC7F8E3
:10659000CC34264910304CF021FD254BC7F89034FF
:1065A00020460123C7F8F06487F8F86485F8503571
:1065B0001FB0BDEC028BBDE8F08F00BF10800D084E
:1065C000495D01080000B4424D5D0108515D0108BC
:1065D000555D01080000FFFFC0910020D4610E0846
:1065E0007C9B00203CC10E08595D01085D5D0108DF
:1065F000615D0108655D0108695D01086D5D010867
:10660000CC790D08A4790D08889200206CC50D087E
:10661000869200204492002024D00D080C7A0D08A8
:1066200068D00D08B8010E0810020E08D8B60E0882
:1066300090030E0810B592F0A7F8064C064B1860B0
:106640002046FFF777FC2046044A0549BDE8104084
:10665000BAF048B8402C00203C2C002058F4002010
:10666000715D01080069C0F3401070470F299DBF9C
:10667000302303FB0100503000207047014B93F999
:1066800061027047404C0020014BD3F8740C7047F6
:10669000404C002008B503689B68984730B9044B0C
:1066A00093F87A0FB0FA80F0400908BD0020FCE7AB
:1066B000406C002008B504480FF042F810B9034BB5
:1066C00093F8740F08BD00BF402C0020406C0020E0
:1066D000022A10B50C4605D1BDE810400948352204
:1066E00010F0A8BF084BD3F8600F03685B689847A9
:1066F000A04205D163F010F8BDE8104062F096BFEB
:1067000010BD00BF402C0020406C0020012910B5B6
:106710000C4610D0022904D061B961F033FD084A5B
:1067200002E061F02FFD074A06215AF045FD064BB5
:10673000C3F8344210BD61F025FD044AF4E700BF00
:10674000A8D10D0880D10D08408C002097D10D08EC
:10675000012910B50C4614D0022907D0D1B90E4B2F
:10676000C3F8F01461F00EFD0C4A05E00A4BC3F8C3
:10677000F01461F007FD0A4ABDE8104006215AF006
:106780001BBD61F0FFFC074A06215AF015FD024BC4
:10679000C3F8F04410BD00BF408C0020E7D10D08C5
:1067A000BCD10D08D0D10D08012903D0022914BF96
:1067B00000210221014BC3F8141C7047404C0020FB
:1067C000012902D0022900D011B9024BC3F8F414F8
:1067D000704700BF408C00206C2910B400F3A680E5
:1067E0003F290FDC162900F39980032940F39A8092
:1067F0007E4B01248C402340002B00F093805DF8F9
:10680000044B7047A1F140032C2B00F28B8001A4B4
:1068100054F823F0CD6901082569010825690108AC
:10682000256901082569010825690108256901080C
:1068300025690108FF670108256901082569010824
:106840002569010825690108FF6701082569010814
:10685000256901082569010825690108C36901083E
:1068600025690108C369010825690108C369010890
:10687000C3690108C3690108FF67010825690108A8
:10688000C3690108FF670108256901082569010836
:10689000FF670108FF67010825690108FF67010814
:1068A000256901082569010825690108256901088C
:1068B000256901082569010825690108256901087C
:1068C000FF670108FF670108112B2BD801A454F8BA
:1068D00023F000BFFF670108256901082569010849
:1068E00025690108FF670108256901082569010874
:1068F000256901082569010825690108256901083C
:1069000025690108FF670108FF670108256901087B
:1069100025690108FF670108FF670108A1F1270346
:10692000112BD1D95DF8044B63F078BDA0291FDC91
:106930009529F7DDA1F196030A2BF3D801A454F8A9
:1069400023F000BFFF6701082569010825690108D8
:1069500025690108FF670108FF670108256901082B
:10696000FF6701082569010825690108C369010855
:10697000B52921DCA929D5DDA1F1AA030B2BD1D89A
:1069800001A454F823F000BFFF670108256901083E
:1069900025690108FF6701082569010825690108C3
:1069A000FF670108256901082569010825690108B3
:1069B00025690108FF670108A1F1D003022BB1D8B6
:1069C0001DE75DF8044B002363F0FABC084B01227D
:1069D00083F8EC24A3F58043D3F8700C00283FF42F
:1069E0000EAF5DF8044B642162F0DCBE1000410084
:1069F000408C00206C2938B50346154600F3A28070
:106A00003F2912DC38290ADC26296FDC102900F026
:106A10000581162900F08A81042900F016812A4692
:106A20001846BDE8384063F069BAA1F140022C2A4B
:106A3000F5D801A050F822F0F56B01081F6A010893
:106A40001F6A01081F6A01081F6A01081F6A0108FE
:106A50001F6A01081F6A0108256C01081F6A0108E6
:106A60001F6A01081F6A01081F6A01084F6C0108AC
:106A70001F6A01081F6A01081F6A01081F6A0108CE
:106A8000976C01081F6A0108EB6C01081F6A010876
:106A9000A16C0108E16C01088D6C0108236D0108EF
:106AA0001F6A01080B6D0108556C01081F6A010877
:106AB0001F6A0108E36B01083B6D01081F6A0108AA
:106AC000336C01081F6A01081F6A01081F6A010868
:106AD0001F6A01081F6A01081F6A01081F6A01086E
:106AE0001F6A0108C36D01085B6C0108A1F1270250
:106AF000112A94D801A050F822F000BFE36B0108DE
:106B00001F6A01081F6A01081F6A0108E76B010874
:106B10001F6A01081F6A01081F6A01081F6A01082D
:106B20001F6A01081F6A01081F6A0108456C0108F5
:106B30002D6C01081F6A01081F6A01083F6C0108DB
:106B4000396C0108A02921DC95297FF768AFA1F1F4
:106B500096020A2A3FF663AF01A050F822F000BF68
:106B6000456D01081F6A01081F6A01081F6A0108B4
:106B70004B6D01089D6D01081F6A0108AB6D01088E
:106B80001F6A01081F6A01086B6D0108B52923DC23
:106B9000A9297FF744AFA1F1AA020B2A3FF63FAF24
:106BA00001A050F822F000BF616C01081F6A0108C3
:106BB0001F6A01088B6D01081F6A01081F6A01081E
:106BC000676C01081F6A01081F6A01081F6A010833
:106BD0001F6A0108E36D0108A1F1D002022A3FF605
:106BE0001EAF01248FE0A91E864B4D424D4183F814
:106BF0006D5FF6E7AA1E5542834C554184F8EB546D
:106C000061F0C0FA814A94F8EB14814B002908BF67
:106C10001346804A06215AF0CFFAE2E70A21FFF72D
:106C200057FDDEE72A4601211846F8E72A460421E7
:106C3000FAE72A460321F7E72A460C21F4E72A4619
:106C40000F21F1E72A460021EEE70B21E7E72A466C
:106C50000D21E9E72A460521E6E72A461521E3E763
:106C60002A461121E0E7AB1E5A425A41664B93F87F
:106C700094129142B5D083F8942261F083FA664A67
:106C8000664B022D08BF1346654AC3E729461846DE
:106C9000FFF78AFDA5E729461846FFF737FDA0E76D
:106CA000594CD5B1022D0DD1012384F8E834A4F557
:106CB0000053D3F8600F03685B6A984710B15948D6
:106CC00000F096FF61F05EFA534A94F8E814534BD3
:106CD000002908BF1346544A9CE784F8E854E6E7C5
:106CE00029461846FFF734FD7BE7012445B1022D04
:106CF00009D1454BC3F8EC41002283F8DC2202E0C5
:106D0000414BC3F8EC51204638BD01242DB1022D72
:106D1000F9D1464B83F87440F5E7444B83F874503F
:106D2000F1E729461846FFF74BFD5AE7022A7FF4A0
:106D300058AF3C4808F0D4FD53E762F0EDFC62F038
:106D400075FC4EE72A4607216EE71846294662F091
:106D5000EDFF374880F086F8044600283FF441AF45
:106D6000294B0122C3F8EC21C6E7274BD3F8AC32FC
:106D7000002B3FF436AF012425B1022DC3D183F897
:106D80002C40C0E783F82C50BDE7022D7FF429AFDB
:106D90009FED280A2348FBF7A5FB22E7022D7FF48D
:106DA00020AF20480EF0DAFB1BE701242DB1022DA5
:106DB000A9D1154B83F8EA44A5E7134B83F8EA54AD
:106DC000A1E7022D12D10F4DD5F8600F0368DB6BE0
:106DD0009847044678B10121A5F5804003F08CF96D
:106DE00091E71548294690F017FAFAE60D48002178
:106DF00003F082F9F5E661F0C5F9104A04215AF072
:106E0000DBF9EEE6406C0020408C0020FCD10D0840
:106E1000CFB90D0804D20D08DFA30D0818E30D0843
:106E200014D20D08402C002020D20D08404C002028
:106E3000948D002000000000E07A002033D20D087D
:106E400010B599B104681168416004B90160126815
:106E500001681B68521A9A4202D80021084610BDE8
:106E6000017A012381F001010372F7E7037A3BB154
:106E700044682CB11368029A12681B1B9342ECD928
:106E80000023C0E90033EFE70023C0E90533C0E980
:106E900008338385037780F828307047F0B52DEDEF
:106EA000028B044687B09F48B0EE408A0E467FF0C2
:106EB000E3FF40B1236933B1206B00F50E7010F091
:106EC000B9FE054638B12046FFF7DEFF002007B0C7
:106ED000BDEC028BF0BD236B93F93C22002A1EDD32
:106EE00093F8A032DBB1904BD3F8F424002AEAD116
:106EF0002369D4ED007A991E4842F5EEC07A4841E4
:106F0000F1EE10FA84F82C0027D8C4E90822C4E96D
:106F1000052284F82D2084F828202277D7E7834F94
:106F2000D7F8600F03689B6B984728B107F5805727
:106F300097F89835002BD6D07D4800210EF096FEAC
:106F4000DFED7C7AB4EEE70AF1EE10FACBDA78489E
:106F500003F0A2FE0028C6D1B5E76EB1F4EEC87A00
:106F6000F1EE10FA3CDD236BD3F8C432DB0403D519
:106F7000714815F015FC064684F82D6092F006F96C
:106F8000D4ED027A9FED6D7A039067EE877AFCEE7E
:106F9000E77A17EE903A5B000593B4F90630CDED31
:106FA000047A002B1EDC0023C4E9083384F828305F
:106FB00094F90430002B41DC0023C4E90533237726
:106FC00094F82C00002882D194F82D0000287FF43A
:106FD0007EAF94F8280000287FF479AF207F76E711
:106FE0001646C9E70421524800F0AEFCB4F9063059
:106FF00007EE903AF8EEE77A05ABF4EEC07AF1EEE0
:1070000010FA0093CCBF0121002104AB03AA04F1C4
:107010002000B0EE408AFFF713FF0028C8D061F0CF
:10702000B1F8064618EE100AF9F76EFA444ACDE9AF
:107030000001042130465AF0BFF8B9E7414E9FEDF8
:10704000427AD6F8B824DFED416A06F58051D1EDD9
:107050007F7A82EAE270B0EE476AA0EBE270A7EEB8
:10706000A66A07EE900AF8EEE77AF4EEC67AF1EE39
:1070700010FA53D8D6F8BC0491ED806A07EE900A56
:10708000A6EE267AF8EEE77AF4EEC77AF1EE10FA79
:1070900044D591ED816A9FED2E7AA6EE267AF4EE24
:1070A000C77AF1EE10FACCBF01270027642113FB49
:1070B00001F1284BD3F8B005121A002AB8BF52428A
:1070C0008A422DDAD6F8BC24D3F8B435D31A002B73
:1070D000B8BF5B428B42ACBF0023012304F1140014
:1070E0000FB983F0010505AB009303AA04AB294651
:1070F000FFF7A6FE00283FF463AF61F043F8D6F82F
:10710000B814D6F8BC24642392FBF3F291FBF3F39A
:1071100000920421104A5AF04FF851E70027C5E7C2
:107120000023DBE7948D0020408C0020406C002081
:10713000402C002000000034003F002000007A4472
:107140002CD40D08403C00200000FA430000C84247
:107150000000FAC3407C00203DD40D0873B582893D
:10716000036BD20704466CD493F93C22002A03DD5A
:1071700093F8A022002A64D1524DD5F8601F05F57E
:10718000616291425DD0A5F54055B3F90860D5F82C
:10719000B83407EE903AD5F8BC34B8EEE77A07EE8B
:1071A000903AF8EEE77A6846CDED017A8DED007AF7
:1071B00030F02EFB730007EE903AF8EEE77AB0EE6F
:1071C000C00AF4EEC07AF1EE10FA42D4236B93F8C1
:1071D000F1223AB307EE906AF8EEE77AF4EEC07A5D
:1071E000F1EE10FA1EDB002183F8F112236B586BCD
:1071F00088F0E6FB236B9FED347ADA6BD2ED067AEA
:1072000005F2C46267EE877A92ED007AF4EEC77AEF
:10721000F1EE10FA06D5986B8AF032FE236B986B6C
:107220008AF0C8FBA389226B13F0020302D192F803
:10723000F11299B9002382F8F232236B93F8F1022C
:1072400005E0002083F8F102236B83F8F20202B01C
:1072500070BD236B012283F8F122B7E705F2DC5100
:10726000D1ED007A9FED197AF0EEE76AF4EEC76A85
:10727000F1EE10FADFDD05F2D451D1ED006A9FED99
:10728000146AB0EEE67AB4EEC67AF1EE10FAD2DD08
:1072900005F5BB6191ED007AB0EEC77AB4EEC67A1F
:1072A000F1EE10FAC7DD67EEA67AF5EEC07AF1EEE0
:1072B00010FAC0D5D5F8BC3406498B42ACBF0023C8
:1072C0000123B8E7406C00200AD7233CC2B8323E05
:1072D000920A063F6CEEFFFF08B5036B93F8F222AB
:1072E0003AB1DA6A92F8A020022A03D0002283F889
:1072F000F22208BD0B4B9FED0C0AD3ED007AF5EEA0
:10730000C07ADFED0A7AF1EE10FAD8BFB0EE670A64
:10731000152063F097FDBDE808409FED050A132096
:1073200063F090BD1C42002000A08CC500A08C45DD
:107330000000000000F58040D0F8600F03681B6C6F
:107340001847000000F5005393EDA07A00F5C04007
:10735000B5EEC07AF1EE10FA5DBF036BDFED076AA0
:10736000D3ED017A806C5FBFF8EEE77AE7EE267A1C
:10737000FDEEE77A17EE900A704700BF0000C842A2
:1073800000F5005090F8C00228B141F00101084218
:1073900014BF01200020704710B54B68516800F5FC
:1073A000C0448B42D8BF0A46606ECCBF1A4619460D
:1073B0002DF0D0FA606610BD10B504464D486EF051
:1073C000E5F910F0080217BF4B4BDFED4C7A93ED57
:1073D0003B7AD3ED3D7A1FBF77EE877A9FED487AEF
:1073E000012267EE877A10F0010317BF424B9FED31
:1073F000437AD3ED3D6A93ED3A7A1CBF37EE667A55
:10740000DFED3F6A04F5005118BF27EE267AD1ED73
:10741000A26AF5EEC06A18BF0123F1EE10FA34DD5E
:10742000354A9FED376AD2EDA26A66EE866A01227E
:10743000F4EE676AF1EE10FA58BFF0EE667A04F5E2
:10744000C04090F86C1029B373B1D0ED1C6AF8EE0F
:10745000E66AF4EEC76AF1EE10FA58BFF0EE476A3A
:10746000FDEEE66AC0ED1C6A9AB190ED1C7AB8EEAA
:10747000C77AB4EEE77AF1EE10FAD8BFB0EE677AC9
:10748000BDEEC77A80ED1C7A03E0002AD7D1002B2D
:10749000D5D110BDABB1036BD3ED016AF8EEE66A4E
:1074A00076EE876A90ED197AB8EEC77AF4EEC76A7D
:1074B000F1EE10FAD8BFB0EE667ABDEEC77A80ED75
:1074C000197A002AE5D0036B93ED017AB8EEC77AFA
:1074D00077EE277A90ED197AB8EEC77AF4EEC77A8C
:1074E000F1EE10FA58BFB0EE677ABDEEC77A80EDC4
:1074F000197ACEE7204D0020404C0020000000000B
:107500000000C84200F5C0400023836670470000B9
:1075100073B51646044600236A46304600931CF0B5
:1075200099FA48B1DDED007A9FED267A67EE877A09
:10753000FDEEE77A17EE900A04F5C045A8663378A9
:107540005B0718D595F86C30ABB104F5AD4001225E
:1075500001A9583053F006FF68B1D5ED1C7ADDED76
:10756000016A9FED187AF8EEE77AE6EEC77AFDEE4B
:10757000E77AC5ED1A7A04F5A043D3F89C35042BBD
:107580001DD004F50054B4F9BA22002A15DDAB6E03
:107590009FED0D7A83EAE371A1EBE37107EE901A98
:1075A000F8EEE77A67EE877A07EE102AB8EEC77A28
:1075B000F4EEC77AF1EE10FA01D50023AB6602B003
:1075C00070BD00BF0000C8420AD7233C37B50B7816
:1075D0005A0704460D461DD500F5AD40012201A90C
:1075E000583053F0BFFEA8B1D5ED017A2B78DFED0E
:1075F0001A6AF8EEE77ADB0767EEA67A19D59DEDF1
:10760000017AB4EEE77AF1EE10FACCBF0120002047
:1076100003B030BD2B78D5ED017A13F0010FF8EEF1
:10762000E77A04F5C0440ED194ED127AB8EEC77A29
:10763000E7E704F5C044236B93ED017AB8EEC77A0F
:10764000E7EE667ADBE7236B93ED017AB8EEC77A53
:1076500077EE877AE8E700BF0AD7233C00F50053AE
:1076600000F58042B3F96A32D2F8602F00EE103A8A
:1076700000F5994340339A42B8EEC00A0ED100F5A6
:10768000A040D0F89C35042B02D090F851352BB196
:1076900000F67470D0ED007A30EE270A70470000D3
:1076A000014608B501F5C041FFF7D8FFD1ED127AC8
:1076B0009FED057AF8EEE77AE0EE477AFDEEE77A9D
:1076C00017EE900A08BD00BF0000C84237B500F5AC
:1076D000C045044695F86C30DBB100F5AD400122A1
:1076E00001A9583053F03EFE98B1D5ED1C7AD5ED86
:1076F0001D6A9FED0B7AF8EEE77AE6EE877ADDED0C
:10770000016AE6EEC77AFDEEE77A17EE900A03B05B
:1077100030BD2046FFF7C4FF6B6E181AF7E700BFB5
:107720000000C842014608B5FFF798FF01F5C041C7
:10773000D1ED207A37EEC00ADFED047A20EE270A79
:10774000FDEEC07A17EE900A08BD00BF0000C842E7
:107750002DE9F04100F5C04800F5C04508F14408A6
:1077600054350446294640461CF0E8FB04F5A04782
:1077700004F5C04607F5A76334362A46314683ED43
:10778000000A40461CF010FB07F23C57DFED220ACE
:1077900087ED000AB7EE001A76202DF03BF804F5CD
:1077A000345383ED770A2046FAF72CFE04F5804324
:1077B000D3F8600F03685B6898470B280CD007D894
:1077C0000A2810D004F5C0440023A366BDE8F08168
:1077D0000E38C0B20128F5D829462046FFF7F6FE3C
:1077E0000028EFD011E029462046FFF7EFFE30B920
:1077F0000A484FF48041FBF73FF90028E2D12046C8
:10780000FFF790FFB0F5FA6FE6DD2A4631462046D5
:10781000BDE8F041FFF77CBE00000000402C0020D6
:1078200010B52DED028B00F5C043D3ED167A93F819
:107830005430DFED1D8AB8EEE78ADA0728EE288A91
:1078400082B0044609D400F5805202F5A662D2ED5A
:10785000007AF8EEE77AA7EEE88A5B070FD504F521
:10786000AD40012201A9583053F07CFD38B19DEDA7
:10787000010A30EE480A02B0BDEC028B10BD204672
:1078800004F58054FFF70CFF04F5A66393ED000A9E
:1078900007EE900AB8EEC00AF8EEE77A28EEC00AC2
:1078A000A7EEA80AE5E700BF0AD7233C73B5044654
:1078B0001646FFF765FD78B966BB04F5C3451C3570
:1078C00028460AF031FDB8B328460AF0D5F898BB2F
:1078D0002046FFF7A5FF09E004F5005595F8903C18
:1078E000DB0705D505F6AC4595ED000A02B070BD85
:1078F00004F5C3401C300AF03DFD0028DCD095F8AB
:107900005A1C04F551604CF075FE0228D4D19FED4D
:107910000D0AEBE704F5A04393F8703F022BCCD19E
:1079200004F5AD40012201A9583053F01BFD002899
:10793000C3D09DED010AD9E704F5C04494ED200AB7
:10794000D4E700BF0000000000F5C04393F86C20AE
:10795000FFF7ACBF38B52DED028B00F5804200F586
:107960009843D2F8602F60339A4204464CD100F518
:107970008053D3F8C05400F50053B3F9B832002B4C
:1079800065DD04F5B65292ED017AF7EE007AB4EEB9
:10799000E77AF1EE10FA5AD404F53552D2ED007AB6
:1079A000F6EE006A67EEA67A87EE871AB5EEC01A81
:1079B000F1EE10FA4BD907EE905A9FED278AB8EEF8
:1079C000E70A07EE903A04F5AD4004F5C044F8EE3E
:1079D000E70A20EE080A583053F0D0FDA36E9FED61
:1079E0001F1ADFED1F0A002BBCBF07EE903AF8EE1E
:1079F000E77A4FF42970B8BFA7EE880ABDEC028B76
:107A0000BDE838402CF006BF07F000FEF8B904F5D9
:107A10004053D3F8440603681B69984704F50053A4
:107A2000DFED0F0AB3F9B83201EE103A04F5AA43BC
:107A300093ED0E0AB8EEC11A054640F27F202CF0F5
:107A4000E9FEBDEEC00A10EE103A1BB297E7BDEC9E
:107A5000028B9FED030A38BD0AD7233C00007A440D
:107A60000000000010B5044691F090FB04F50053AF
:107A7000D3F8A42C801A41F2883290420FD8022108
:107A80002046FFF77DFC50B104F5A044D4F89C25B6
:107A9000042A04D103F6984393ED000A10BD9FED2C
:107AA000010AFBE70000000030B52DED028B00F568
:107AB000C045DFED268A95F86C3083B004465BB391
:107AC000D5ED1C7A9FED220AF8EEE77A00F5AD407D
:107AD00027EE800A012201A9583053F07BFCD8B16F
:107AE0002046FFF737FFDDED017A85ED1D0A37EE01
:107AF000800A20468DED010AFFF7B4FFDDED017A23
:107B000030EE270A20EE280ABDEEC00A10EE100A59
:107B100003B0BDEC028B30BD2A6B6B6E52689B1AB2
:107B200008EE103A2046FFF799FDB8EEC88A2046C5
:107B3000A0EE288AFFF796FFBDEEC88AB8EEC88A85
:107B4000A0EE288ABDEEC80AE0E700BF0000C842E8
:107B50000AD7233C10B500F580430446D3F8600FE4
:107B600003685B6A984718B104F5C04494F8E804C8
:107B700010BD000038B500F5C0440D46636E0B44DF
:107B8000636694F86C302BB1FFF7E4FF10B9216FF6
:107B90002944216738BD000030B500F50050D0F809
:107BA000B422D3070FD4094B0B201D785C688D429B
:107BB00004D1224214BF0120002030BD013803F15E
:107BC0000803F2D1F9E70120F7E700BF94D40D08CC
:107BD00010B500F580430446D3F8600F03685B6876
:107BE000984701462046BDE81040FFF7D5BF00008A
:107BF00037B500F5C0440546A36C63660023A36651
:107C0000FFF7E6FFD0B105F5AD40012201A95830DC
:107C100053F0A8FB90B12846FFF79CFF70B9DDED4B
:107C2000017A9FED087A67EE877A0123FDEEE77A05
:107C300084F86C30C4ED1C7A03B030BD002384F8A6
:107C40006C30F9E70000C84238B504460D46FFF72E
:107C5000BFFF30B1032128461BF0D8FE80F001039E
:107C6000D8B204F5C04484F86D0038BD73B500F592
:107C7000C0444A6862660B780D46D90741BF236B42
:107C80005B689B18636694F86D30064623B100F577
:107C9000C0415431FFF7D8FF2B785B070ED506F5AE
:107CA000AD40012201A9583053F05CFB30B10123F3
:107CB00084F86C306B68236702B070BD002384F8D1
:107CC0006C30F9E7F0B52DED028B044683B004F576
:107CD000C0450E468DED010AFFF7C8FFDFED320A01
:107CE0009DED010A40F24310B7EE001A2CF092FD10
:107CF000AB6E5B4207EE903AF8EEE77A204667EE0D
:107D0000807A04F50057FDEEE77AB0EE408A17EE70
:107D1000901AFFF72FFFD7EDAF7AF5EEC07AF1EEAC
:107D200010FA3CDDAB6E002B39DD2046FFF7CEFCB0
:107D300007EE900ADFED1D6AB8EEE77AD7EDAF7A6D
:107D400067EEA67AB4EEE77AF1EE10FA27D531465F
:107D50002046FFF78BFF2946324644312046FFF785
:107D6000D7FBAB6E5B4207EE903AF8EEE77A20461F
:107D700067EE887AFDEEE77A17EE901AFFF7FAFEC3
:107D8000B5EEC08AF1EE10FA09DDD5ED1A7AB8EE3B
:107D9000E77AC7EE087AFDEEE77AC5ED1A7A03B006
:107DA000BDEC028BF0BD00BF000000000000C8C2A7
:107DB000F0B500F5C04487B094F8543003F00503E3
:107DC000052B07460BD054F01BFB4FF4AE724FF45B
:107DD000801154F0CDFA0025284607B0F0BD1E48AA
:107DE0006A4603211BF022FE0028F4D01B4801AA9A
:107DF00003211BF01BFE05460028ECD0184BDFEDDD
:107E0000190A93ED000A40F26D10B7EE001A2CF03B
:107E100001FD04F154030FCBB0EE401A02AEDFEDCA
:107E2000111ADDED010A9DED000AB7EE002A86E881
:107E30000F002CF021FCDFED0C7A20EE270A3046F3
:107E4000FDEEC07A032217EE901A1BF01BFD31469F
:107E50003846FFF70BFFBFE7748C0020948C00209E
:107E60007C810020000000000000C842F7B50E46EB
:107E700002210446FFF784FA70B304F5A045D5F853
:107E80009C35042B28D12046FFF7A2FE20B304F531
:107E9000AD47583704F5C04101236A46443138469E
:107EA00053F04AF9C0B104F5C041012301AA54318D
:107EB000384653F041F978B19DED017ADDED007A55
:107EC00077EEC77A96ED007A37EE277A05F25C55A1
:107ED00086ED007AC5ED007A03B0F0BDF0B52DED6A
:107EE000048B00F5005489B000F5516694F85A1CD3
:107EF0000391054630464CF07DFB0399074630461A
:107F00004CF08AFB042F0399B0EE408A20D1002365
:107F100005A88DED050A069307932FF01BFF05A911
:107F200005F5AF502DF0A0FDDFEDAD7A8DED050A22
:107F3000B4EEE71AF1EE10FACDED060A8DED071A50
:107F400006DB05F5805393F83C7517F001070CD15B
:107F500094F8903C002262F3000384F8A82C84F883
:107F6000903C09B0BDEC048BF0BD94F8903C9A07AE
:107F70005FBF43F0020384F8903C04F6944383ED22
:107F8000008A05F5325104F6AC4383ED001A2C311A
:107F90002846FFF76BFF94F8A83C092B00F28A8073
:107FA00004F54B63D3ED000A9FED8E9AB0EE480ABC
:107FB0002CF01EFB00BB04F6944394F85A1CD3ED3E
:107FC000008A30464CF046FB07EE900A9FED867A19
:107FD000F8EEE77A78EEC88A67EE877AF0EEE88AFC
:107FE00067EE897AF4EEE78AF1EE10FAC2BF94F8F0
:107FF000A83C013384F8A83C04F54B6394F85A1C60
:10800000D3ED008A30464CF025FB07EE900AF8EEDF
:10801000E77A9FED767A67EE897A78EEC88A67EE1E
:10802000877AF0EEE88AF4EEE78AF1EE10FA02DDE4
:10803000002384F8A83C04F54B6383ED008A94F890
:10804000903CDA078DD52846FFF7EAFB04F6AC43EF
:1080500093ED008A05F5C04330EE488A93F86C3002
:10806000002B72D005F5AD40012205A9583053F020
:1080700079F900286FD191F089F8D4F8A42C41F255
:108080008831821A8A42034604F6984204F69C41DB
:108090006AD982ED008A284681ED008A0221FFF725
:1080A0006FF920B105F5BE45D5F88020EA67C4F820
:1080B000A43C56E794F8903C43F0010384F8903CCC
:1080C00005F5A043D3F89C6505F58043301FD3F830
:1080D000602F05F59B43464203F1540346419A4203
:1080E00012D005F59B4370339A420DD005F59943A4
:1080F00040339A4209D13E4B05F5C340B3F8FE1513
:108100001C3009F0D5FC00B13E4694F8903C59076C
:1081100091D4002E8FD002212846FFF731F9002894
:1081200089D043F0040384F8903C04F6AC4305F591
:1081300050561868F8F7E8F92836CDE900012D4ABD
:108140000621304659F038F875E72846FFF740FD1C
:10815000002887D18FE704F6AC4393ED000A9DED2C
:10816000058A38EE408A86E79FED200A92ED007A74
:10817000DFED217A28EE008AA7EE278A82ED008AB9
:10818000C4F8A40CD1ED007A38EE678AF3EE0E7ACB
:10819000B0EEC88AB4EEE78AF1EE10FA7FF7E1AEEE
:1081A00094F8903C5B070ED504F6AC4405F55056A8
:1081B0002068F8F7A9F92836CDE900010F4A062111
:1081C000304658F0F9FF05F53250242200211030D6
:1081D00009B0BDEC048BBDE8F040BAF0C5BF00BFEC
:1081E000000000340AD7233CCDCC4C3DCDCC4C3ED6
:1081F000407C002054D40D08CDCC4C3F71D40D08E8
:1082000038B52DED028B0D460446FFF709FB002320
:1082100020462B70B0EE408AFFF724FC0221204656
:1082200038EE400AFFF7ACF828B104F5005494F892
:10823000900C00F00100BDEC028B287038BD0000EE
:1082400070B50B7803F00503042B05460C46164663
:1082500014D105F5C04554F0D3F8B2B24FF48011F3
:1082600054F086F82A6B636852689B1A13F5FA7FFC
:10827000C8BF6360237843F00103237070BD000022
:10828000F8B500F5805300F5A047D3F83065D7F86E
:108290006055B542044619D00E4A1268D26A92F867
:1082A0009C209AB100F5C041751B25225431FFF77F
:1082B000C7FF07EE905AB8EEE70ADFED077A04F53C
:1082C000345020EE270A183083F012FDC7F860659D
:1082D000F8BD00BF3C2C00200AD7233CF8B500F5C0
:1082E000A04C00F5C0449CF853E505460F4604F148
:1082F0003406BEF1000F4AD004F154030FCB86E8D8
:108300000F0001238CF8543597E80F0004F1540650
:1083100086E80F00E36D05F5C04654365BB9236E61
:108320004BB9E36CA26DE365236D23661AB9A16CAA
:1083300030461BF0A7FA314628222846FFF780FF77
:1083400094F8541011F0040102D130461BF05EFB8A
:1083500005F5C04105F5C0403246343144301BF0CC
:1083600059FD30B104F13406443494E80F0086E836
:108370000F00284606F022FD2846FFF7E9F92846B7
:1083800007F008F92846BDE8F840FEF7D3BF04F12E
:1083900044030FCB86E80F0001238CF853358CF88B
:1083A00054E5B1E7F8B500F500530446B3F91232CD
:1083B000002B0D4632DB0B7813F0020F14BF4FF089
:1083C000FF33012304F5C04606F13407337306F189
:1083D00044030FCB87E80F0095E80F0006F1540720
:1083E00087E80F00572239462046FFF729FF20462D
:1083F000FFF7FEFB2046FFF7ABF9204607F0CAF86F
:1084000004F5A043002583F854552046356183F8D0
:10841000595506F0D3FC86F8DE52F8BD4FF0FF3315
:10842000D0E700002DE9F043354B1B6885B00546C9
:10843000D86AF9F779F800285FD105F5005393F968
:10844000283C5A1C52D0002B05F5866611DD95F8A4
:108450004124242107EE903A01FB026292ED0B7A4F
:10846000F8EEE77AB0EEC77AB4EEE77AF1EE10FAFA
:108470003CDC05F5805305F5965793F83C3513F031
:10848000010429D0C3F340089B0732D495F8E413C4
:1084900095F828444FF0B00909FB015191F8C1311A
:1084A0004CBB022B18D968461BF0E6F969463846E2
:1084B00015F022F9044678B195F8E43309FB03532B
:1084C0004246D3F8D01168461BF0DCF915F0EAFB00
:1084D000694614F0FFFF0446304617F093FE384615
:1084E00014F016FF2846FAF79BFA204605B0BDE8BF
:1084F000F0830024F0E74446EEE70020F6E700BFF3
:108500003C2C002038B50C4B1B680546D86A0C463D
:10851000F9F70AF810B10024204638BD15F0C2FB67
:10852000214614F0D7FF04460028F4D005F5AB40EF
:10853000403030F029FAEFE73C2C0020F0B500F590
:10854000A04300F5C046002283F8532583F8542544
:1085500006F14403044600EE101A0FCB87B006F173
:10856000340585E80F0002AD3246B8EEC00A284651
:10857000154944324BF0B2FD95E80F0006F154075F
:1085800087E80F0040F25712394620460197FFF75F
:1085900057FE01992046FFF757FB01992046FFF748
:1085A00065FB04F500532046B3F91232002BB4BF2B
:1085B0004FF0FF3301233373FFF7CAF8204607B0AB
:1085C000BDE8F04006F0E6BF0863002010B503499F
:1085D00004464BF083FD204610BD00BF0863002019
:1085E000F8B500F5C04505F1440304460E460FCB2F
:1085F00005F1340787E80F0006F108012046FFF770
:108600006DFEB28802EB820202EB8202920012B28D
:1086100004F5A043002AD8BF4FF4C872A3F84E2532
:108620002A6BA96D5068091AC3F8201591680A31A0
:10863000E965D2680A322A660022C3F8342583F835
:10864000502583F86425C3F8242503F5A36200218F
:1086500011604FF0FF32C3F8102594F8411404F56F
:108660008662242000FB012203F5A963D26A1A6006
:10867000F8BD000070B50E4608310446FFF72EFE27
:10868000B38804F5A04543B3642213FB02F3C5F895
:108690002035B5F94E35002BD8BF4FF47A7304F569
:1086A0003250D8BFA5F84E35242200211030BAF040
:1086B0005BFD04F5C04304F5BE4093ED200A31464E
:1086C00074308CF021FED5F89C35072B0CD1204658
:1086D0000421BDE87040F9F763BED5F82035002BC2
:1086E000D7DC40F6B833D2E770BD000030B50831B2
:1086F00004460FC985B06D4685E80F0004F5C041FA
:10870000443128461BF022FA20462946FFF7E6FDB1
:1087100004F580440123C4F8883F05B030BD000053
:108720000B7A00F5C04013F0020F14BF4FF0FF3377
:1087300001230373704700007FB501F1080305466C
:108740000E460FCB6C4684E80F0005F5C04144315E
:1087500020461BF0FBF921462846FFF7BFFD3146B6
:108760002846FFF7DDFF04B070BD00007FB501F1C2
:10877000080304460E460FCB6D4685E80F0004F54E
:10878000C041443128461BF0E1F929462046FFF755
:10879000A5FD20463146FFF7C3FF337907EE903A37
:1087A000337E9B0748BF9FED0A7AF8EE677A04F59F
:1087B000C04448BF67EE877A9FED067A67EE877AF6
:1087C0000123FCEEE77A6362C4ED017A04B070BD68
:1087D0000000803B00A00C477FB501F10803044670
:1087E0000E460FCB6D4685E80F0004F5C0414431BD
:1087F00028461BF0ABF929462046FFF76FFD2046BF
:108800003146FFF78DFFB38804F5C0444FF47A7208
:108810005343E3610123636204B070BD2DE9F3416A
:1088200000F5C0450446543500F5C0400E463430CE
:1088300029461BF04BF904F5A047C8B94FF0FF33A8
:10884000C7F8103506F1080738461BF045F803282D
:1088500002463BD1F16828461BF014F8B28804F5B3
:10886000C04320465A6202B0BDE8F041FEF74ABE5E
:1088700024F07CFDF9F7E0FA012812D94FF0FF331C
:10888000C7F8103524F072FD90F8C432DFED140AF9
:10889000B02202FB030090ED300A28461BF0F4FBE7
:1088A000D0E704F58058D8F8C0042BF087FF04F512
:1088B000A653C7F81005D3ED007A9FED0A0ADFED45
:1088C000080AF8EEE77A27EE800AE6E701AA002117
:1088D00038461BF00DF80028C0D001990022BAE7F5
:1088E00000007A440AD7233C7FB501F1080304460F
:1088F0000E460FCB6D4685E80F0004F5C0414431AC
:1089000028461BF023F929462046FFF7E7FC2046BE
:108910003146FFF705FF04F5C0440023636204B04D
:1089200070BD000037B504460D4690F02FFC206264
:10893000D5ED027AF5EEC07AF1EE10FA15DD9FED75
:10894000127A67EE877AFCEEE77AC4ED077A5FF079
:1089500019FCE2694FF47A73B2FBF3F30B4A062178
:1089600003B0BDE8304058F027BC6CF05DFD00233B
:10897000009395F90D2095F90E3095F90C106CF0D7
:10898000EFFCE061E3E700BF00007A44ECD40D089F
:108990002DE9F0432DED028B85B0044615F082F9E8
:1089A00014F068FA04F5805304F5A04693F8B8373C
:1089B0000BB9002877D0D6F81035013373D1D6F82B
:1089C0003435002B4BD090F0E1FBD6F83435C01A8B
:1089D000B0F5FA6F67D394F8E423DFED607A9FED8A
:1089E000608A4FF0B00808FB024292ED780A20EE50
:1089F000270A2BF0FBFE06F5A369D9ED007A30EECD
:108A0000670A2BF0F3FEDFED577A20EE080A04F533
:108A1000505720EE270A2BF091FEFDEEC07A283742
:108A200017EE905AC6F81055D9ED007A67EE887A9D
:108A300017EE900AF7F768FDCDE9020194F8E433E8
:108A400008FB0343D3F8DC01F7F75EFD464ACDE9A6
:108A500000012B460621384658F0AEFB23E004F512
:108A60009070F9F7E9F902281DD994F8E433B0229F
:108A700002FB034393ED777AF1EE047AB4EEE77AE2
:108A8000F1EE10FA0FDD394B1B68D86A0368DB6919
:108A90009847012803D090F079FBC6F83405D6F842
:108AA0003435002B8FD104F54053D6F81015D3F888
:108AB00044064A1C036847D01B6B98472C4810F0AB
:108AC00087FD20B104F5AB40403032F0BDF92046BF
:108AD000FEF728FED6F820358342054637DA07EE42
:108AE000905A9FED247AF8EEE77A04F5505767EE36
:108AF000877A283717EE900AF7F706FD1E4ACDE968
:108B000000013846062158F057FB04F5C0444FF0E9
:108B1000FF330125C6F8103586F8505504F144039B
:108B20000FCB04F13407543487E80F0084E80F00BA
:108B300012486CF0F5FD002386F85335284605B041
:108B4000BDEC028BBDE8F0835B6B9847B6E7084845
:108B500010F01EFD0028C2D1F1E700BF35FA8E3CAF
:108B6000E02E65420000C842FCD40D083C2C0020D9
:108B7000402C00200AD7233C20D50D08204D002092
:108B8000F8B500F5C04600F5C04534365435044606
:108B9000294630461AF09AFF04F5405730B304F5E1
:108BA000A043D3F810154B1C20D0D7F84406036817
:108BB0001B6B984704F5C0456B6A012B44D06B6A68
:108BC000022B05D12046FEF76BFDAB6D984241DDCF
:108BD0002046FEF765FDAB6DC01A0028B8BF4042C5
:108BE000B0F5FA7FCCBF0020012034E004F5C0408E
:108BF000294644301BF0A2F9DFED177AB4EEE70AFC
:108C0000F1EE10FA16D5304629461BF067F89FEDB5
:108C1000137ADFED130AF6EE007AE0EE077A2846C3
:108C20009FED100AFDEEE77AF8EEE77A27EE800A6C
:108C30001BF02AFAD7F844069FED0B0A03682A4670
:108C40009B6A31469847B5E72046FEF729FDAB6D94
:108C50009842B4DB0120F8BD00004843A00CB345A6
:108C6000000096430AD7233C0000000073B5384C3F
:108C7000D1ED026AD4ED127A9FED367AF8EEE77AFA
:108C80000546D7EE876A0E46F5EEC06AF1EE10FA99
:108C900008DD5FF077FA304A062158F08DFA01209E
:108CA00002B070BDD1ED037AF5EEC07AA4F52D6463
:108CB000F1EE10FA94ED006A12DDF4EEC67AF1EEF0
:108CC00010FA0DD55FF05EFA05462068F7F71CFC38
:108CD000224ACDE900010621284658F06DFADEE768
:108CE000DFED1F7A337CB4EEE76AF1EE10FA54BF81
:108CF000B0EE677AB0EE467A0BB90020D0E7B5EE59
:108D0000C06AF1EE10FA0CDC86EE876A03EB83038F
:108D100007EE903AF8EEE77AF4EEC67AF1EE10FA42
:108D2000EBD595F82440002CE7D190F02FFAAB6AF0
:108D3000C01A337C4FF47A7253439842DDD9012331
:108D400085F8243090F022FAA8622046A8E700BFF8
:108D5000408C00200AD7233C3CD50D084DD50D088A
:108D60000AD723BC38B505467FF006FB7EF084F8B1
:108D7000044640B990F00AFA2B6AC01AEB6998428F
:108D800084BFEC610124204638BD000038B504469C
:108D90000D4690F0FBF904F5C0439FED067A98620A
:108DA000D5ED027A67EE877AFDEEE77AC3ED097AB0
:108DB00038BD00BF00007A4410B5044690F0E6F9D3
:108DC00004F5C0439A6A801A5A6A90424FF0000034
:108DD00084BF5862012010BD00F5C04300F5AA41D0
:108DE0005A6A91ED0E7A22EAE27207EE902AF8EEC4
:108DF000E77A0020B4EEE77AF1EE10FA44BF586249
:108E00000120704710B500F5005300F5C040B3F9DC
:108E10001232002BB4BF4FF0FF330123037300F174
:108E2000540444300FC884E80F0010BD38B5044620
:108E30002DED028BF0EE408AB0EE608A09B3012975
:108E40005ED0B5EEC08AF1EE10FA69DDDFED357A5D
:108E5000B4EEE78AF1EE10FA62D8FCEEC87A04F5B7
:108E6000505017EE903A304A0621283058F0A4F9B5
:108E7000FDEEC87A04F5005417EE903A84F8DF311D
:108E80003CE0F8EE000A2BF0B3FB40B104F580445F
:108E90004FF0FF33C4F8983FBDEC028B38BD04F5AA
:108EA0000053B3F9E82107EE902AF8EEE77AF4EEE2
:108EB000E87AF1EE10FAC4D8B3F9EA3107EE903A45
:108EC000F8EEE77AF4EEE87AF1EE10FAB9DBDFEDCE
:108ED000157A68EEA77A04F58043FDEEE77A04F58B
:108EE000505017EE902AFCEEE87AC3F8982F06212E
:108EF00017EE903A0D4A283058F05EF90120CBE782
:108F0000FCEEC07A00F5505017EE903A084A062160
:108F1000283004F5005458F04FF9C4ED7D8AEDE790
:108F20000020B9E70000C84293D50D086CD50D08A4
:108F300080D50D08D1F80D3000EE903AD1F8093007
:108F4000097A00EE103AFFF771BF000070B58B8808
:108F5000012B04460D4611D100F590763046F8F706
:108F60006BFF02280AD994F8E413B02303FB0161D4
:108F70002046AC31BDE87040FFF7C4BA14F092FE51
:108F800005F10801BDE8704014F0A4BAF0B500F591
:108F9000A0470024BF4B87F8594589B005460846CD
:108FA0000E4683F86D402FF001FB002835D00123D9
:108FB00087F8503505F54053D3F844060368DB6B5A
:108FC000984705F5C04387F8574503A81C611AF078
:108FD00053FCB7F8FC154FF6FF73994208BF2146C2
:108FE000013105F5AB4001AA89B2403031F0AEFA4B
:108FF000F0B1BDF80630A3F115025342534187F892
:10900000513550B105F5C340BDF806101C3008F0CD
:109010004FFD10B1002387F8513574885E2C77D846
:10902000522C31D8103CA3B20F2B4BD900248DE029
:109030000346E4E7C33C112CF8D801A353F824F00D
:10904000A19201082D900108A19201082D9001081C
:109050002D9001082D900108A19201082D90010882
:109060002D9001082D900108DF9201082D90010834
:109070002D9001082D9001082D900108659201089E
:109080002D90010885920108533C0B2CCED801A3EA
:1090900053F824F01192010819920108299201084D
:1090A0002D9001082D9001082D9001082D900108A8
:1090B0002D9001082D9001082D90010801930108C1
:1090C000299201080F2CB1D801A353F824F000BF56
:1090D00095910108CF910108D9910108E391010808
:1090E000F7910108A1910108679101082D900108ED
:1090F0002D9001082D9001082D9001082D90010858
:109100002D9001082D90010807920108ED910108AA
:10911000D42C1ED8C22C8DD8B22C00F099800DD83A
:10912000702C00F09080722C80D1D6ED027AFDEE8A
:10913000E77A05F5C045C5ED097A29E0B32C00F0C2
:109140008C80BC3C012C8CBF00240124204609B03B
:10915000F0BD40F6B8339C427FF468AF317A4E4898
:1091600007F04CFB14E0002305F5C34487F889356C
:109170001C347188204607F043FF314628B1204651
:1091800009B0BDE8F04008F03DB92846FFF728FADD
:109190000124DBE706F108012846FFF79FF8F7E70F
:1091A00005F5C3441C341521204608F081FC48B164
:1091B000002387F889353146204609B0BDE8F040E4
:1091C00008F024B831462846FFF754FAE0E7314664
:1091D0002846FFF7B1FADBE731462846FFF7C6FA23
:1091E000D6E731462846FFF7F7FAD1E73146284659
:1091F000FFF77AFBCCE705F5994129226C31284627
:109200000EF040F9C4E731462846FFF707FBBFE7F9
:10921000012487F8574599E7002305F5C34087F8EF
:10922000893531461C30ABE705F5C3471C37384656
:1092300008F022FC3146044618B12846FFF756FADA
:1092400084E73846B9E731462846FFF79FFD9FE798
:1092500031462846FFF76EFE9AE731462846FFF76B
:1092600075FE95E7B388012B92D803F0010387F8C8
:10927000523505F55050B388084A0621283057F07A
:109280009BFF85E7B188003918BF0121284600F00F
:1092900033FF7DE7408C0020DC8D0020A4D50D0835
:1092A00005F5C144F36805F5C045503495F84911FA
:1092B0007BB933696BB973695BB9204663F076FC9F
:1092C00004287FF465AF95F84911204663F078FCD7
:1092D0005EE706F10802204663F0B0FD58E705F5A9
:1092E000C04305F5C14096ED041AD6ED020A96ED8D
:1092F000030A93F849110022503063F083FC47E7DA
:1093000005F5994031464030FFF70CFB40E700BFC0
:1093100000F5804200F59943D2F8602F40339A421D
:1093200001D1FFF733BE01207047000010B500F5F2
:10933000804200F59943D2F8602F40339A420446A8
:109340000ED100F5994108226C310EF09BF804F51E
:109350005050044ABDE810400621283057F02CBF79
:1093600010BD00BFB4D50D082DE9F04F2DED048BD5
:1093700000F5C04898ED878ADFEDD87AB0EEC87A5C
:10938000B4EEE77AF1EE10FA48BF00F50053DFEDD6
:10939000D47A42BFB3F9123208EE103AB8EEC88A56
:1093A00000F58045B4EEE78AF1EE10FA94BF4FF075
:1093B000FF37012788F80C70D5F8883F9BB004462A
:1093C0000E46F0EEC88A052B16D8DFE813F006002B
:1093D0002B0068008700C4005E0100F540543A4647
:1093E000D4F844060368B0EE680ADB6A083198478F
:1093F000BC4806F00BF908B9002047E1BA4C236BD2
:10940000B4F95C125B68642201FB0231A4F5C04030
:10941000FFF794F8A4F5C04005F0D0FC0123C5F88F
:10942000883FE9E700F540533A46D3F8440603681D
:10943000B0EE680ADB6A08319847D8F80830002B8C
:10944000B8BF5B42012BD7DD98F80D301BB998F8F7
:109450000E30002BD0D004F5B153D3ED020A93EDBA
:10946000030AF1EE600AB1EE400AB7F083FCDFEDCB
:109470009F7A20EE270A05F68C7383ED000A10EE22
:10948000100AF7F741F804F550542834CDE90001EB
:10949000974A0621204657F08FFE0223BFE700F5CA
:1094A000C04901F1080A09F14409494650461AF039
:1094B00045FD30EE680AF1EE047AB0EEC00AB4EE73
:1094C000E70AF1EE10FA00F3E680D8F8083001332D
:1094D000022B40F2EA800323C5F8883F04F540538D
:1094E00006F10808D3F8440603683A46DB6AB0EE92
:1094F000480A41469847DFED7F6A9FED7F7A05F67F
:109500008C73D3ED007A012F18BFB0EE667A04F5A4
:10951000A65377EE877A93ED030A9FED787AA7EE4C
:10952000C70A2BF063F9DFED767AB0EEC00AB4EE2D
:10953000E70AF1EE10FA7FF55FAF04F5505006210F
:109540002830704A57F038FE0423C5F8883F41465A
:109550002046FEF7C3FE06F1080595E80F000AAFA6
:109560000DF1380887E80F0088E80F0004F5804304
:1095700003F68C7A9FED649A9AED000ADFED630A98
:109580000393384630EE090A1AF07EFDDFED5F0ADC
:109590009AED000A9FED5E8A40461AF075FD04F5CB
:1095A00040534246D3F84406036839469B6AB0EEFE
:1095B000480A984795E80F0004F5C3490DF1480B98
:1095C00009F11C098BE80F00DAED009A484607F014
:1095D0003DFD79EE899A04F5C048F0EE400A584600
:1095E000B0EE690A08F144081AF04EFD5A463946B1
:1095F00040461AF00FFC834695E80F009AED000AEA
:1096000016AF87E80F00F0EE680A30EE090A384618
:109610001AF03AFD394640462A461AF0C5FB07A91A
:1096200004F59650F0EE408A8DED078A8DED088A9C
:109630008DED098A14F034F900284AD029464046B5
:109640001AF088FB05A907A8CDED060A8DED050ADD
:109650002EF0F2F8DFED257A20EE270A2BF05AF8EB
:10966000B0EEC00ABBF1000F3FF4C6AEF3EE0E7AC7
:10967000B4EEE70AF1EE10FA23D5039A0523C2F8F7
:10968000883F3146484607F0C1FD01201BB0BDECC4
:10969000048BBDE8F08F494650461AF04FFCB4EEFB
:1096A000E80AF1EE10FA7FF510AF04F540543A469F
:1096B000D4F844060368B0EE680ADB6A514698475E
:1096C0009AE6F6EE007AF4EEE78AF1EE10FAD4DCD0
:1096D00092E6BBF1000F3FF48FAECEE700000034FE
:1096E000000000B4402C0020408C0020E02E654299
:1096F000DCD50D080000B4420000874335FA8E3CEB
:10970000C2B8B23DFED50D080000344300007A44D3
:1097100000000000F0B5044600F5C3408FB01C30D7
:109720000F4608F0E9F9054638BB09AE30461AF095
:10973000A3F804F5A0434FF6FF72B3F8FC3593424B
:1097400008BF0023013304F5AB4007AA99B24030AB
:1097500030F0FCFEA0B104F5C04407B1A56096E866
:109760000F0001AD85E80F00236E0093543494E898
:109770000E00044803F0C8F9054628460FB0F0BDB6
:109780000125FAE74879002070B5054605F5C04681
:10979000002106F023F834696CB9284605F036FF3D
:1097A00010B90024204670BDB368012BF9DD8FF09D
:1097B000EDFC3061F6E7716A49B18FF0E7FC33697F
:1097C000C01AF3699842ECD900237362012128463C
:1097D000FFF7A0FF04460028E3D005F55050054AE6
:1097E0000621283005F5A04557F0E6FC002385F852
:1097F0005935D7E720D60D0838B50A468B88190A9F
:10980000137EDB0748BF01EB8101044648BF4900D6
:1098100005F0E4FF04F5A043002583F859552046E0
:1098200005F0F4FE10B90025284638BD04F5C04304
:10983000596A39B1D3E901128A42F4DD012AF2DD15
:109840005D6201212046FFF765FF05460028EAD04A
:1098500004F55050024A0621283057F0ADFCE3E7EA
:1098600038D60D0838B5054605F5C044898805F099
:10987000B5FF636A5BBBA368002BB8BF5B42012BDB
:1098800002DC0024204638BD627BA37B6AB9002B32
:10989000F7D005F55050A26C6423062192FBF3F338
:1098A00028300C4A57F088FC01E0002BF1D101214F
:1098B00061622846FFF72EFF04460028E1D005F537
:1098C0005050054A0621283057F076FCDAE700218F
:1098D000EFE700BF50D60D086ED60D0810B5044650
:1098E0000B4808F0EDFE48B10A4BDFED0B7AD3F8D8
:1098F000D83193ED090A20EE270A10BD04F5005473
:10990000B4F9403200EE103AB8EEC00AF5E700BFF5
:10991000DC8D0020408C00200AD7233C10B52DEDB3
:10992000028B00F500530446B3F944120029ACBF82
:1099300001224FF0FF3200F5C0430029B8BF494271
:109940001A7389B205F04AFF04F5AA43204693ED45
:109950000E8AFFF7C3FFB5EEC00AF1EE10FAD8BFCA
:109960009FED0D0ABCEEC00AB8EE400AB4EEC08A04
:10997000F1EE10FA0AD804F550502830074A0621B3
:1099800057F01AFC0120BDEC028B10BD204605F0FB
:109990003DFE0028EFD1F6E70000000088D60D0854
:1099A0002DE9F04F00F5A0492DED028B4FF0FF336C
:1099B00000F5C04AC9F810350AF154030F460546B0
:1099C0000FCBBC8897F8048089B004AE240A86E8DF
:1099D0000F001ED057463437314638461AF0AEFADB
:1099E00031463846B0EE408A1AF078F9DFED567A03
:1099F000B4EEE78AF1EE10FA0BDBE3B200EE903A38
:109A0000DFED527AF8EE600A20EE270A30461AF0AF
:109A10003BFB05F5405B99F85425DBF844069FEDC8
:109A20004C0A036805F5C0479B6A443732B305F515
:109A3000C04132463431984705F50053B3F94232FC
:109A4000002B1EDD07EE903A09F5A762F8EEE77AE3
:109A500092ED007AB4EEE77AF1EE10FA11DD05F539
:109A6000C0413246343138461AF0D4F9F8B90024EE
:109A7000204609B0BDEC028BBDE8F08F3246394676
:109A8000D9E7B8F1000F1CD1002C3CD1DBF84446DB
:109A900023682846D3F82080FFF720FF09F22C53D3
:109AA000D3ED000A2046C047B0EE408A0DE0002CFE
:109AB000DDD10AF144030FCB0AF1340585E80F002C
:109AC000D6E707EE908AB8EE678A314638461AF034
:109AD00035FAB4EEC08AF1EE10FA17DBB9F8FC35AE
:109AE0000393314638461AF029FABCEEC00A05F550
:109AF0005050039B174A8DED000A0621283057F07D
:109B00005BFB0124B4E79FED128ADEE705F5C04157
:109B10003246343138461AF07DF904460028A6D082
:109B2000B9F8FC350393314638461AF007FABCEE13
:109B3000C00A05F55050039B074A8DED000A062127
:109B4000283057F039FB93E700000034E02E6542DF
:109B500000000000A0D60D08BED60D082DE9F04784
:109B60004B881F2B8AB004460D466BD80F2B41D86B
:109B700004F55050BF4A0421283057F01DFB9BE0EC
:109B8000A3F1BC02182AF3D801A151F822F000BFBA
:109B9000B99C0108B99C0108719B0108719B0108DF
:109BA000719B0108719B0108719B0108B99C010818
:109BB000719B0108B99C0108719B0108719B010808
:109BC000719B0108B99C0108719B0108719B0108F8
:109BD000719B0108B99C0108B99C0108B99C010856
:109BE000719B0108719B0108B99C0108719B0108D8
:109BF000B99C0108A3F110020F2AB9D801A151F8AC
:109C000022F000BFF59C0108DB9D0108E59D0108DD
:109C1000F19D0108079E0108019D0108CB9C0108E8
:109C2000719B0108719B0108719B0108719B0108E0
:109C3000719B0108719B0108719B0108119E01082D
:109C4000FB9D01085E2B21D8522B91D9A3F1530221
:109C50000B2A8DD801A151F822F000BF1B9E0108EC
:109C60002D9E0108379E0108719B0108719B010818
:109C7000719B0108719B0108719B0108719B010890
:109C8000719B0108619E0108379E0108722B00F04C
:109C9000E28007D8702B7FF46BAF0AB0BDE8F047C5
:109CA000FFF78AB8D42B09D8BB2B3FF669AFA3F1D5
:109CB000B202012A3FF65CAF012052E0DF2BFBD05D
:109CC00040F6B8329342F7D052E700F5C3461C364F
:109CD0001621304607F094F930B1294630460AB0D3
:109CE000BDE8F04707F07ABC20460AB0BDE8F0476F
:109CF000FEF74EBE29460AB0BDE8F047FFF750BE5A
:109D000000F5C3451C351521284607F0D1FE28B1C2
:109D100028460AB0BDE8F0470BF0C2B904F5A045EB
:109D200004F5BE46D5F89C3504F5C04704F5C04897
:109D300004F5C049072B06F1740607F1340708F152
:109D4000540809F144090FD104F5AB4418340194C7
:109D5000D5F82035009342464B46394630468BF0C5
:109D600097FB0AB0BDE8F0870DF127018DF82700B9
:109D70004148FEF745FA05F25C53D3ED007AD5F879
:109D800040A505F5A663D3ED000A05F23C5330EE7D
:109D9000670A93ED001A8DED070A04F5C2405430AE
:109DA000CDED060A8DED051A7DF05CF805462046DE
:109DB00000F072FF9DF827309DED051ADDED060AD3
:109DC0009DED070ACDE90203CDE900A54B464246C9
:109DD000394630468BF0B2FAC3E7A98805F0FEFC9D
:109DE0000020BEE729460AB0BDE8F047FFF704BDF2
:109DF0000AB0BDE8F047FFF7C7BC29460AB0BDE886
:109E0000F047FFF72FBD0AB0BDE8F047FFF786BD6A
:109E10000AB0BDE8F047FEF7B3BE04F59940294605
:109E200040300AB0BDE8F047FEF720BF04F5C3405C
:109E300029461C3053E704F5C3461C36304607F06C
:109E40001BFE08B9304664E729462046FFF78CFA26
:109E50000028F7D185E70AB0BDE8F047FEF7BCBFA0
:109E600004F59940294640300AB0BDE8F047FEF7B6
:109E700079BF00BFDCD60D08402C002070B500F57E
:109E8000804200F59943D2F8602F40339A4205464C
:109E90000E4602D00024204670BDFFF75FFE044648
:109EA0000028F7D005F55050318828305BF014FBBE
:109EB000F1E7000021F04003152B04D0A1F15E036F
:109EC00058425841704701207047000000F5804219
:109ED00000F59943D2F8602F40339A4207D100F53C
:109EE000A040B0F8FE355B1A584258417047002038
:109EF00070470000192963D8DFE801F00D1115192A
:109F00001D2125282C62303437563A3A3D404347CC
:109F10004A4E62525A5E00F59A406030704700F532
:109F200097403430704700F597405030704700F547
:109F300097406C30704700F598400830704700F546
:109F400098404430704700F59840E6E700F59840A7
:109F50007C30704700F599402430704700F59940F7
:109F60004030704700F59940E3E700F59A40E4E798
:109F700000F59A40F0E700F59A40E2E700F59A40D4
:109F8000E6E700F59B401830704700F59B40C8E7B6
:109F900000F59B405430704700F59B40703070478F
:109FA00000F59C401030704700F59C4048307047E9
:109FB00000F59D400430704700F59C402C30704700
:109FC0000020704700290DDB074890F88C2CCBB29D
:109FD0009A4207D3D0F8883C0122595CA0F5005082
:109FE0000DF028BB704700BF404C00202DE9F34125
:109FF00000F5005300F5505593F8583C03F0010666
:10A0000003F0020803F004075B07044605F1280586
:10A0100035D01F4A0621284657F0CEF826B104F560
:10A020003E501C307EF0B6FFB8F1000F04D004F5AE
:10A03000435034307EF02AFD27B104F549500C30EE
:10A040007FF0D2FB04F5C044012384F8E934114ABF
:10A05000114B1249B8F1000F08BF1A46002F08BF74
:10A060001946CDE900210E4A0621002E18BF1346DD
:10A0700028460C4A57F0A0F802B0BDE8F0810A4A21
:10A080000621284602B0BDE8F04157F095B800BF60
:10A0900009D70D08FED60D084CC80E0805D70D08C7
:10A0A000F8D60D081AD70D082CD70D0810B50446A0
:10A0B00000F53E501C307EF099FF04F543503430DB
:10A0C0007EF010FD04F549500C307FF0C7FB04F51D
:10A0D000C04393F8E9245AB1002283F8E92404F537
:10A0E0005050044ABDE810400621283057F064B8AB
:10A0F00010BD00BF4CD70D0809B1FFF777BFFFF7C0
:10A10000D5BF000000F580430A4AD3F8601F914292
:10A110000DD093F86D3F43B900F59942403291421A
:10A1200003D100F5A04090F852351846704700233F
:10A13000FBE700BFA079002010B504468FF026F899
:10A14000054BD3F8803FC01A642804D82046BDE8E8
:10A1500010405FF05BBA10BD406C002010B500F5F8
:10A160003154D4ED027AF5EEC07AF1EE10FA8AB0ED
:10A170004FF0000304F1080444D9079308930993AE
:10A1800006AB019307AB009303AA05AB04A900F546
:10A19000965013F025FA30B3DDED080A9DED070A5D
:10A1A000B6F04CFCDDED090AB6F048FCD4ED007ABF
:10A1B0009DED047A77EEA76AB4EEE70AF1EE10FAA5
:10A1C000F4EEC76AACBF01200020F1EE10FA0CD803
:10A1D00002309DED037AF4EEC77AF1EE10FA0CD856
:10A1E000003818BF01200AB010BDF4EEC77AF1EEB6
:10A1F00010FA9CBF0130C0B2EBE7012894BF0020E9
:10A200000120F0E70020EEE738B5114B1A7A04463A
:10A21000EAB901251D7253F005FF2A4604F5C3452E
:10A2200011211C3553F0B6FC284607F0A9FC70B18B
:10A23000284607F061FC062204F59B4128B1543101
:10A24000BDE8384003480DF01DB91831F8E738BDB6
:10A2500040910020402C002010B5074B1A7A4AB1DB
:10A2600000241C7253F0DEFE22461121BDE810408E
:10A2700053F090BC10BD00BF409100202DE9FF417C
:10A28000054605F59658684619F0F6FA69464046BF
:10A2900013F0FAFA0646E8B137487CF0E3FD50B116
:10A2A00005F53153D3ED027AF5EEC07AF1EE10FAEE
:10A2B00094BF0126002605F5C3401C3007F060FC62
:10A2C0002E4C2F4F00B146B1002328462380FB734C
:10A2D000FFF7C2FF04B0BDE8F0812846FFF73EFF5C
:10A2E000A0B363787BBB23780133DBB2082B2370E8
:10A2F00002D1404613F0E0F92378092B02D1404601
:10A3000013F0D2F92378092B1DD94FF485732380DC
:10A3100053F088FE0222102153F03CFC8EF036FFF1
:10A320006368C01A47F23053984209D905F5505076
:10A33000144A0221283056F03FFF8EF027FF60605C
:10A340002846FFF761FF6378FB73C3E72378002B90
:10A35000F9D0013B6278DBB22370002AF3D0002BE6
:10A36000F1D1667053F05EFE3246102153F012FCBC
:10A370002846FFF771FFE6E7948D0020409100200A
:10A38000ED91002060D70D0810B500F5A044D4F879
:10A390009C35042B01D1012010BD00F5C3401C30B9
:10A3A00008F074F90028F6D194F8C805F4E7000025
:10A3B00073B500F580450192A5F8781F04468EF02C
:10A3C000E5FEC5F87C0FD5F8600F03685B68984719
:10A3D00085F8760FD5F8600F03685B689847019A97
:10A3E000182818D8DFE800F00D170D0D0D0D0D0D14
:10A3F0000D1752175917595917414141171717414E
:10A400005900334B93F8EA3403B304F598414431CF
:10A4100020460DF037F8D5F8600F95F8766F036891
:10A420005B68984704F55054864204F1280447D0ED
:10A43000D5F8600F03689B689847264A03460421B5
:10A44000204602B0BDE8704056F0B6BE04F5005399
:10A4500093F95432022BD8D0042B0BBF04F598414A
:10A4600004F5974160313431D2E704F5C043D3F8A5
:10A470006034D90203D504F599416C31C8E704F57D
:10A480009B419B064CBF70315431C1E7204601927D
:10A49000FFF77AFF019A0028BDD104F5005601921A
:10A4A00096F95432002BB6D0D5F8600F03685B687C
:10A4B000984785F8760F96F95432019A022BCAE72D
:10A4C000054A0421204602B0BDE8704056F074BE33
:10A4D000408C002070D70D0892D70D08F0B50446C7
:10A4E00004F5804685B00F4615465FF015F8D6F89E
:10A4F000600FA6F8787F03685B68984718281ED815
:10A50000DFE800F00D0D0D0D0D0D0D0D0D1D65821B
:10A510000D0D71711D5353531D1D1D530D003E4BE9
:10A52000D3F89C25012A21D104F5005393F8553224
:10A53000023B012B1AD904F5405383F82424D6F8A2
:10A54000600F364A364B052D18BF13460268039339
:10A550009268904704F5505428340090039B314A88
:10A560000421204656F028FE05B0F0BD2E4B93F88E
:10A57000EA343BB104F598412A46443120460CF0B8
:10A5800081FFDCE704F5005393F95532032B03D127
:10A59000204605F085F9D2E7022BEBD0042B2ED113
:10A5A00004F599412A464031E8E704F5C043D3F861
:10A5B0006034DA0223D49B0604D504F59B412A4675
:10A5C0007031DBE704F59B412A465431D6E720463B
:10A5D000FFF7DAFE0028B2D104F5C3401C3007F0C3
:10A5E000F9FA0028EED104F5005393F95532032B04
:10A5F000CED0022BBED0042BD2D0012B9FD104F59C
:10A6000099412A466C31B9E704F5005393F9553264
:10A61000042B94D1C4E700BF407C0020A8D70D08CC
:10A6200054BB0D08B0D70D08408C002070B500F564
:10A63000505504462835124A0421284604F5804620
:10A6400056F0BAFD0023A6F8783F04F5005393F8BE
:10A650009C31032B12D196F8761F302220460CF045
:10A66000E9FFD6F8600F03689B689847054A0346E0
:10A6700006212846BDE8704056F09EBD70BD00BF63
:10A68000C4D70D08DBD70D0800F5405310B50022E4
:10A690000529044600F5505083F8242400F12800D1
:10A6A0000CBF054A054A042104F5804456F084FD98
:10A6B0000023A4F8783F10BDF4D70D0805D80D0885
:10A6C000013A38B50446052A3ED8DFE802F04B1BB4
:10A6D0008711900300F5C04393F8B03243B100F501
:10A6E0009C4104222C314448BDE838400CF0CABEDD
:10A6F00004F5C04393F8B03223B104F59B41042222
:10A700005431F0E704F58043D3F8602F04F59B4300
:10A7100054339A4226D004F59C432C339A4221D0DC
:10A7200004F5A043D3F89C35042B1BD0334D95F88A
:10A73000913FBBB1324905F5AE5030F0D9FA20B1A6
:10A74000304B012283F8C82538BD2D4905F5AE50A0
:10A7500030F0CEFD30B104F5994104224031A5F529
:10A760008040C1E704F58043D3F8602F04F59B4394
:10A7700054339A42E8D004F59C432C339A42E3D0F8
:10A7800004F5A04304F5C3401C30D3F89C5507F0F2
:10A790007DFF0028D8D1042DD6D004F5005393F9BD
:10A7A0001F32022B0DD004F59941204604226C3152
:10A7B0000CF068FE04F507501F30BDE8384048F043
:10A7C000E3BC0E4890F8913F002BECD00C4900F50B
:10A7D000AE5030F08DFA0028B2D1E4E700F5C24067
:10A7E000BDE83840012214215430F7F7D1B9BDE853
:10A7F000384005F055B800BF402C0020406C0020C8
:10A80000848C0020407C002070B52DED068B044622
:10A810008EF0B0FC414BB4F8BE101A88404E8A420C
:10A820000546404A06D01980002330601370BDEC05
:10A83000068B70BD33683C49C31A8B4265D901232E
:10A8400013705EF069FF5EF021FE35605EF064FF1C
:10A850005EF01CFE5EF042FE0428E8D95EF05CFE6D
:10A86000204600210BF02EF820460021B0EE40AA31
:10A870000BF032F820460121F0EE409A0BF0F6F989
:10A8800000212046B0EE408A0BF030F804F5C240BB
:10A890005430F0EE408A7CF0EFFA9FED249A0028C5
:10A8A000B0EE4A0A4FF0040008BFB0EE498A60F0EB
:10A8B000C9FAB0EE690A132060F0C4FAB0EE680A73
:10A8C000152060F0BFFAB0EE680A1A2060F0BAFAFC
:10A8D000B0EE480A462060F0B5FA0121084660F063
:10A8E000BDFDB0EE490A022060F0ACFAB0EE490AB4
:10A8F000032060F0A7FA20460BF0FAFBBDEC068BB4
:10A900002046BDE870400CF049BB1278002A8ED07A
:10A9100044F6206293428AD993E700BF4C9100200D
:10A92000509100204E910020400D030000000000D7
:10A9300000F5804200F59943D2F8602F40339A42E7
:10A9400004D100F5A04090F8C805E8B10F4B93F88A
:10A950009C0103F58043A0F12702012A93F8F83403
:10A960000FD92C2809D00A2809D0A0F13102504271
:10A9700050410A2B18BF002070470120F9E7012041
:10A9800070470A3B58425841704700BF404C002076
:10A9900008B500F5005393F8E02042B193F81C315C
:10A9A0002BB1FFF7C5FF80F00100C0B208BD012048
:10A9B000FCE700002DE9F04700F50055B04F95F891
:10A9C0001C81044600F5C2408AB054307CF04AFA3B
:10A9D000D7F89C35042B064642D1012104F50357D4
:10A9E000DFF8B0A2203738466BF000FA9AF8F83456
:10A9F0000A2B814604D1002E54D100238AF8F83462
:10AA000095F8E030002B59D195F9E6309D4D012B9A
:10AA100003D0063BDBB2012B11D895F89C310A2BF1
:10AA20000DD104F58046D6F8600F03681B6A98477D
:10AA300028B1D6F8641F2B2220460CF023FD9AF88B
:10AA4000F8340A2B04BF37238AF8F83495F89C3180
:10AA50000A2B02D1372385F89C310AB0BDE8F08774
:10AA60000028BAD004F58043B7F8FE95D3F8600FFC
:10AA700003685B6898471428AFD004F5C3401C30C6
:10AA800007F052FC0028A8D14946A7F5A040FFF7DF
:10AA900011FA01460028A1D097F8C4154B1E59425F
:10AAA00059419BE740EA0803DBB2002BA8D1AAF585
:10AAB000C04000F0F1F800289FD0A1E7002ECCD0D4
:10AAC00004F5BE4074308AF0AFFB0028C5D12046A3
:10AAD000FFF72EFF0028C0D1B9F1000F00F0BF80B2
:10AAE00069494A4638466AF059FD95F9E680B8F159
:10AAF000010F07D040F38780A8F10603DBB2012BDA
:10AB000000F281805FFA88F8B8F1010F4ED104F5A8
:10AB1000804204F59943D2F8602F40339A4209D11C
:10AB200004F5A04393F8C83523B195F81F32013BD3
:10AB3000012B92D904F599410A226C31204606AEC8
:10AB40000CF0A0FC304618F097FE95F9F92092BB66
:10AB5000B8F1010F2FD004F5C048B5F9FA30D8F894
:10AB60003010DFED4A5AD1ED017A002BF8EEE77A8A
:10AB700052DD07EE103AF8EEC76AE6EEA57A3046E7
:10AB8000FDEEE77A17EE901A18F07CFE00233846A7
:10AB9000CDE904336BF0C6F904A96BF007FF002878
:10ABA00057D0049B0893059B099317E004F59A413D
:10ABB0000A222431C2E72046FCF7C4FB07EE900AC4
:10ABC0006F4604F5C042443221463846B8EEE70AE3
:10ABD000FDF7FCFC97E80F0086E80F0095F9E630DA
:10ABE000012B10D031462046FDF72EF83146204685
:10ABF000FDF7D8FB95F9E630072B04D104F5405456
:10AC0000012384F8223453F00DFA4A4609210AB090
:10AC1000BDE8F04752F0BEBFD5ED3A6A95ED3D5A1A
:10AC200095ED3B7A35EE076A36EEC57AB4EEC67A14
:10AC3000F1EE10FA89BF37EE067A95EDA07A27EE8D
:10AC4000257AF6EE006A94BFE7EE257AE7EE267ADB
:10AC500095E7D8F830309A680892DB68A4E7B8F135
:10AC6000000F3FF4FAAE95F81C31002B7FF4F5AEDF
:10AC700004F55050064A0521283056F09DFAC2E7E7
:10AC8000407C0020404C002020D80D080000C84225
:10AC900029D80D08408C002010B5044600F5C240AC
:10ACA00054307CF0E9F898B104F5C3401C3008F04A
:10ACB000E3F960B904F5AB4494ED087ADFED087A66
:10ACC000B4EEE77AF1EE10FAACBF0120002010BD1F
:10ACD00004F5AB4494ED087ADFED027AF0E700BFAB
:10ACE000CDCCCC3D6666663F70B500F5804600F57C
:10ACF0009C43D6F8602F48339A42044600F5A0459D
:10AD000002D195F89805D8B904F5C340B5F8FE15F9
:10AD10001C3006F075F9A0B9D6F8603F04F59944E7
:10AD20004034A3420CD195F898354BB1D5F89C35F9
:10AD3000032B05D1B5F8FE05A0F116035842584182
:10AD400070BD0020FCE700002DE9F74F00F58042C0
:10AD500000F59943D2F8602F40339A42044600F53B
:10AD6000A04504D100F5005B9BF9F8313BB9002305
:10AD7000C5F88C3585F8893503B0BDE8F08F8EF0C5
:10AD800005FAD5F84465804636B1861B40F6C313F4
:10AD90009E4294BF002601262046FFF77DFF0190CA
:10ADA00028B1002785F888754FF0000A46E004F5C1
:10ADB000C24054307CF056F881460028F1D004F5AA
:10ADC000BE4A0AF1740A50468AF02EFA0746002855
:10ADD00045D095F888A5BAF1000F3BD156B304F5DC
:10ADE000805041F27071D0F8B824002AB8BF5242A6
:10ADF0008A4206DCD0F8BC24002AB8BF52428A42FC
:10AE00002BDD04F5AC4104F5C0400431443019F0A9
:10AE100095F8DFED487AC5F88C85B4EEE70AF1EED7
:10AE200010FA4FF000024CBF4FF0010A4FF0000A39
:10AE3000C5F89025012285F88825374604F59070DD
:10AE4000F6F7FAFF022832D9002F44D10023C5F8C3
:10AE50008C3591E7019EB246ECE75646EAE750464C
:10AE60008AF0CAF9824648B1002E9DD04FF4FA7399
:10AE7000C5F890354FF0000A4F46DFE7D5F89C251E
:10AE8000012A07D0032AD9D12046FFF72DFF002839
:10AE90008AD1E9E7DBEDA67AF5EEC07AF1EE10FA99
:10AEA00082DD95F89835002B7FF47EAFDEE704F560
:10AEB000F95604F50059083699F87610304610F026
:10AEC000A5FB0028C2D099F87610304610F096FC09
:10AED0000028B9D1BAE7D5F88C0510B9C5F88C852A
:10AEE0004AE7D5F89025A8EB00089045FFF444AF59
:10AEF00095F88925002A7FF43FAF012285F889253E
:10AF00009BF8F811CB0705D504F5C2400C2154304D
:10AF1000F6F73EFE04F550502830BAF1000F06D087
:10AF2000054A022103B0BDE8F04F56F045B9034A87
:10AF30005146F7E70000964240D80D0856D80D0854
:10AF40002DE9F04F2DED028B044685B0002304F56A
:10AF5000005903938EF01AF9D9ED7D7AF5EEC07A97
:10AF6000F1EE10FAC4BF9FEDC37A67EE877A04F55D
:10AF7000907BC8BFFCEEE77A80465846CCBF17EE00
:10AF8000907A9627F6F758FF022840F20B8194F842
:10AF9000E4339FEDB97AB02202FB0343D3ED777A15
:10AFA00067EE877AFCEEE77A17EE903A9F428CBF05
:10AFB00000270127B9F9E831022BB8BF022307EEB9
:10AFC000903AB8EEE78A03A9F6EE087A04F59650AF
:10AFD00028EE278A12F036FC054640B1DDED037AF3
:10AFE000F4EEC87AF1EE10FAACBF01250025584600
:10AFF000F6F722FF012804F5A0461AD804F5C2404E
:10B0000054307BF02FFFA0B19DB906F5B46393EDEA
:10B01000007ADFED9A7AB4EEE77AF1EE10FA08DD05
:10B02000DDED037AF4EEC87AF1EE10FAACBF01253B
:10B03000002504F5C3401C3005F03AFA824600288A
:10B0400040F0018104F5C24054307BF00BFF002832
:10B0500000F0078194F8E43304EB0313D3F8903144
:10B060007BB158460193F6F7E7FE012800F29C8079
:10B07000019BA8EB030041F2873398428CBF002369
:10B080000123D6F8402502B11BB9002D40F08E8077
:10B090003D4604F5804204F59943D2F8602F4033D1
:10B0A0009A421AD199F92032002B40F08780002370
:10B0B00086F88A35D6F89C35042B00F0B080072B33
:10B0C00000F0C380032B08D12046FFF70DFE20B10E
:10B0D000002586F88955C6F8445596F88A3503B197
:10B0E0008DB907EE905A9FED667AF8EE677A06F50D
:10B0F000B46367EE877AD3ED006A9FED627AE6EE7D
:10B10000877AC3ED007A2046FFF7C6FD0546A8B151
:10B1100096F8A415C6F8408509B9C6F8A88504F5BF
:10B12000804204F59943D2F8602F40339A4205D10A
:10B13000D6F8443503B109B9C6F8448596F8CC363B
:10B1400086F8A45565F3C30386F8CC3674F01CFE6C
:10B15000294674F0F5FD4C4B20465D71FFF7F4FD78
:10B160002046FAF789FA35B199F89E311BB98EF06D
:10B170000DF8C9F8A00189F89E512046FFF78CFD13
:10B18000002840F08D8004F5C24054307BF074FEFE
:10B1900080F00100C0B286F8AC0505B0BDEC028BB2
:10B1A000BDE8F08F002705E753466AE728F0FAFD6F
:10B1B00027F048FF00287FF46BAF6AE75B4207EE99
:10B1C000903A04F69803F8EEE77A93EDDB7AF4EE22
:10B1D000C77AF1EE10FA13DD012386F88A35C6F836
:10B1E000948506F5B463DFED297A93ED007AB4EE29
:10B1F000E77AF1EE10FA7FF75DAFC3ED007A59E719
:10B2000096F88A35002B3FF455AFD6F8943540F6C2
:10B21000B832A8EB030393423FF649AF4AE704F57F
:10B22000BE40743089F0E8FF00283FF456AF06F5C1
:10B23000A66393ED007ADFED157AB4EEE77AF1EECE
:10B2400010FA7FF74AAF012547E706F5A66393EDAD
:10B25000007AFEEE007AB4EEE77AF1EE10FAF2D45C
:10B260003BE7D6F89C35002D18BF3D46012B0FD18A
:10B27000002532E70000B4420000C8429A99993E86
:10B280009A99193E9A99593FED910020CDCC4C3EA8
:10B2900004F5BE40743089F0A5FF0028E8D11CE712
:10B2A000002078E700207047002070470120704799
:10B2B000034BD3F89C05431E58425841704700BFCA
:10B2C000407C002030B587B002A818F0D5FA3A4883
:10B2D00089F088FF20B139493948FCF7C7FC1FE0E5
:10B2E000354889F089FFE8B1364C04F1240523463E
:10B2F00004F11002A4F11001A4F1D000009589F02E
:10B30000A1FFCDE90045A4F60C3292ED000A2E49CA
:10B3100004F11003A4F11002A4F1D00089F054FF4D
:10B3200007B030BD244802A989F0A4FF08B102A9E2
:10B33000D2E7264CD4F8103C002B0CDD94F8B03B3F
:10B340004BB1A4F500501F49FCF790FCA4F5005048
:10B35000FCF7D8F8E4E71A4804F058F90028BAD105
:10B360001B4C94F854305B071FD4A36E002BB2D053
:10B37000124AA2F12001A2F1100018F04BFD0028A2
:10B38000A9D1144C0E48D4ED007AB7EE000A04F6A9
:10B39000183130EE670AFCF795FC094804F6F822EC
:10B3A00004F61831FBF7F8FFBAE7A4F5C040FCF744
:10B3B000FFFC0028B4D1D8E7B48B0020948C002087
:10B3C000402C0020848C0020D0580020404C0020CD
:10B3D000408C00207C81002008B50A4890F891320A
:10B3E000013B012B03D8A0F50050F7F7E7FF064813
:10B3F000F7F7AAFE0448F7F7A1FFBDE808400248A6
:10B40000F8F702BB404C0020402C002010B5044649
:10B4100007480CF033FF50B1064B93F8DD0230B112
:10B42000236820469B6B984780F00100C0B210BD96
:10B4300014900020408C0020124B984210B5044616
:10B4400001D1002010BD03F11C029042F9D003F19C
:10B4500038029042F5D003F174029042F1D0D43317
:10B460009842EED003681B6A984720B1064B93F8C8
:10B470002234002BE5D1206907F022F980F0010089
:10B48000C0B2DFE710780020405C0020174B9842E4
:10B4900010B504460ED003F11C0290420AD003F10D
:10B4A0003802904206D003F17402904202D0D433A5
:10B4B000984206D10E4B93F94902B0FA80F0400948
:10B4C00010BD03681B6A984718B10A4B93F82234E1
:10B4D00043B9206907F0F4F830B12069BDE81040A5
:10B4E00009F094BC0020EBE70120E9E71078002088
:10B4F000404C0020405C002073B50F4E0D461146B5
:10B5000096F968221AB90124204602B070BD03687A
:10B5100001915B69984704460028F4D1D6F860345D
:10B52000019913F4802FEED00448054B00682A4699
:10B53000C06A25F01DFEE7E7408C00203C2C00206F
:10B5400068D80D08084A0260084A4260111F8160ED
:10B5500002F10801C160A2F1380102F59C7242615A
:10B56000034A016182617047B4D80D08148E00202F
:10B57000003F002008B503681B6E98470648D0F8C6
:10B58000602F00F6A4439A4205D0BDE80840A0F51C
:10B590008040FEF78BBD08BD406C00202DE9F743CD
:10B5A0005C4C04F5A36300221A60A4F55073C11A21
:10B5B0004B42A4F500594B4189F8B83604F5A56310
:10B5C000002584F8FC54A4F8525584F8565584F8A4
:10B5D000145584F8895584F88A55C4F87C55C4F804
:10B5E0007855C4F87455C4F884551A60836904F515
:10B5F0008058D3F8FC31A4F84C3508F144030646D2
:10B600000FCB08F1340787E80F0084F8555584F80C
:10B610006455C8F810508DF0B9FD44F8980C3368A3
:10B6200030465B6998474FF0FF3384F8595589F8E5
:10B63000245444F8683C84F85805306906F0D4F97D
:10B6400088F86D5084F8575533683046DB6D98475D
:10B65000A4F580570546002858D0336830469B6BC8
:10B66000984784F89805D9F844060368DB6B984737
:10B67000A4F5E2507DF0F6FDA4F5A0400AF074F8C0
:10B68000A7F5F9506AF018FC94F8C835CBB1A4F5C9
:10B69000A040FFF701FBA0B908F5AA707BF0ECFB16
:10B6A00078B9D7F8600F03685B6B984748B95CF0CE
:10B6B00069FD194A062155F07FFD04F5B8602FF0A9
:10B6C000C3FB1648F6F79EFE336993F9CC206AB1A6
:10B6D000586801A912F0B6F834699DED010A0146D7
:10B6E00004F18800FBF7DAFB84F841013368304647
:10B6F0005B69984750B1336993F93C22002A02DD17
:10B7000093F8A03213B9002387F86D3F284603B0A1
:10B71000BDE8F083407C002074D80D08402C002048
:10B7200070B503685B6E0E4615469847044650B9DF
:10B7300095F900303BB90548054B00683246C06AB0
:10B74000294625F015FD204670BD00BF3C2C002089
:10B7500098D80D0810B50E4C20467DF07FFB04F5FF
:10B76000AC707DF0F7F804F52C707EF025F8094BED
:10B7700003F5A042002182F8141502F5A36200210E
:10B7800003F500531160012283F8E82E10BD00BFBD
:10B79000DC5B0020402C002008B52DED028B15202D
:10B7A000B0EE408A5FF04EFBB0EE480ABDEC028B73
:10B7B0001A20BDE808405FF045BB000008B5084806
:10B7C00090F949320121A0F5005033B10AF04EFA48
:10B7D000BDE8084046205FF035BB0AF06FFAF7E796
:10B7E000404C002001207047012070470120704725
:10B7F00001207047012070471920704700487047AA
:10B800001CD90D08004870472CD90D0884B038B5F4
:10B8100005AC84E80E00054614210C48FCF7BCF981
:10B820002A696423B2F9C01068B103225943204643
:10B8300018F028F805482146FCF7B4FDBDE838406B
:10B84000012004B070470122F0E700BF402C002027
:10B8500013B50F4901AAA1F1100018F0FBF840B18F
:10B86000DFED0C7A9DED017AB4EEE77AF1EE10FA95
:10B870000CD8094CD4F8440603689B6B984728B150
:10B8800006492E22A4F540500BF0FCFD02B010BD7D
:10B89000948C0020000000B4405C0020147A00204A
:10B8A00030B51D4C0546D4F8640F036887B05B695A
:10B8B000984738B119491A482F220BF0E3FD0120AF
:10B8C00007B030BD174806F0FBFE0028F2D1A4F502
:10B8D0008054D4F8440603689B6B984728B1D4F889
:10B8E000440603681B6C984798B10F4B0FCB02AC12
:10B8F00084E80F00284601F06BF82868059B009348
:10B9000094E80E00446C2846A0472846FFF7A0FFA5
:10B91000D5E7064BEAE700BF406C0020147A002010
:10B92000402C0020DC8D0020848C0020948C002092
:10B9300010B50446FFF78CFF2046BDE8104001F02B
:10B9400083B80000042070470048704721DF0D08CD
:10B950000048704721DF0D08037F73B1D0ED087AEE
:10B96000FDEEE77A17EE903A084AC2F8B035437F09
:10B970003BB1436AC2F8B43570478369D3F8F831F4
:10B98000F2E78369D3F8FC31F4E700BF407C002084
:10B9900008B50023838300F12801806911F068FF56
:10B9A000012008BD70B56E4E2DED048B06F59F434A
:10B9B00004460121304693ED0C9ADFED6A9A09F0B6
:10B9C00081FF0121B0EE408A304609F085FFC8EEC4
:10B9D000297A06F50055A069B5F96C3204F1280101
:10B9E00008EE903AF8EEE88AB5F96E3268EEA78A6A
:10B9F000C0EE297A08EE103AB8EEC88A28EE278AF7
:10BA000011F036FF95F9723263B39FED577AF0EE7D
:10BA1000E87AF4EEC77AF1EE10FA23D5227FA36913
:10BA2000002A55D1012222770022226294ED087A61
:10BA3000DFED4E7AD3F8F8314D4A4E4867EEC77ABB
:10BA40009FED4D7A67EE877AB0EE490AFDEEE77A10
:10BA500017EE901A0B44C2F8B035002301227DF096
:10BA60008DF908E0002343482377F0EE490AB0EE51
:10BA7000680A7DF07FF904205FF0E4F995F97232ED
:10BA800043B19FED397AF0EEC87AF4EEC77AF1EE61
:10BA900010FA28D4002339486377F0EE490AB0EE53
:10BAA000480A7CF0C1FD13205FF0CCF9B5F9703283
:10BAB000002B03DD324E96F9623263BB2848202109
:10BAC000F6F7DAFF002843D1254809F01DFD42E0D2
:10BAD000D3EDC56A96ED467AD4ED087AE6EE877A1C
:10BAE000C4ED087AA2E7637F2BB901236377A369CA
:10BAF000D3F8FC3163621E4B616AC3F8B415A369C5
:10BB0000D3F8FC010023091A1A461C48B0EE490A72
:10BB10007CF070FEC7E70121A6F5405009F0E6FE73
:10BB200080EE297AB5F97032002106F5137007EE20
:10BB3000903AF8EEE77AF0EE490A27EE870A7DF0B0
:10BB40003BFDBDEC048B2046BDE87040FFF724BEF2
:10BB50000348F7F7C5FD07EE900AB8EEE70AF0E7ED
:10BB6000402C002000A08C4500000034E02E6542EF
:10BB7000407C0020DC5B00200000C842345D0020D7
:10BB8000405C00202DE9F04F2DED0C8BDFF8A8A3D1
:10BB90009FEDDEDA9FEDDE9A97B00AF59F4300F144
:10BBA000280504460121504693ED0CBA09F08AFE9F
:10BBB00001215046F0EE408A09F08EFE01215046E8
:10BBC000B0EE408A09F092FEDFEDD27A88EEA77AD5
:10BBD0000AF5005601A8B6F96C320AF5A04B0AEE38
:10BBE000903AF8EEEAAAB6F96E32DFEDCB8A6AEE49
:10BBF00087AA88EE277A0AEE103AB8EECAAAB6F9F2
:10BC000070329FEDC68A2AEE07AA80EE277A09EEE7
:10BC1000903AF8EEE99A6AEE8D7A69EE879AF0EE3C
:10BC2000EACAF4EEC8CACDED017AB0EECACA6AEE2D
:10BC30000D7AF1EE10FAF0EEE9BAB4EEC8CACDED25
:10BC4000027A58BF4FF0010969EE8D7A48BF4FF074
:10BC50000009F1EE10FAF4EEC8BA9AED460ACDEDFD
:10BC6000037A54BF4FF001084FF00008F1EE10FACC
:10BC700054BF012700272BF073FF01A928462BF0A2
:10BC8000F7F928462BF0EEFA28462BF05DFA20EE65
:10BC9000090A284620EE280ABDEEC00A10EE103A26
:10BCA000CBF8B0352BF06AFA20EE090A20EE280A0C
:10BCB000DFED9B8ABDEEC00ACDED0D8A10EE103A85
:10BCC000CBF8B4350DF1280B4FF07E535946A069DF
:10BCD0000A93CDED0C8ACDED0B8A11F0C9FD002140
:10BCE000504609F0C3FFB0EEC00AB4EEC80AF1EE48
:10BCF00010FA16D55046FEF7CFFF90B9F4EEC8CA39
:10BD0000F1EE10FA0DD5B4EEC8CAF1EE10FA08D56E
:10BD1000F4EEC8BAF1EE10FA44BF9BE80F0085E8D4
:10BD20000F000AA82BF002FB294612A88DED141A69
:10BD30008DED120ACDED130ACDED151A2BF008FB8F
:10BD40000DF1100A51460EA88DED101ACDED048AA2
:10BD5000CDED058ACDED068A8DED0E0ACDED0F0AEB
:10BD6000CDED111A2BF0BEF8B6F96C32DFED6D7A1D
:10BD700001EE103AB6F96E3209EE103AB6F97032A9
:10BD800008EE903AB8EEC11AB8EEC99AF8EEE88A11
:10BD900021EE271A29EE279A68EEA78AF4EEC8CA80
:10BDA000F1EE10FA21EE0D1A29EE0D9A68EE8D8A49
:10BDB00007D594F83830DFED5A7A002B18BFB0EE73
:10BDC000671AB4EEC8CAF1EE10FA07D594F8393004
:10BDD000DFED537A002B18BFB0EE679AF4EEC8BAC5
:10BDE000F1EE10FA07D594F83A30DFED4D7A002BDA
:10BDF00018BFF0EE678A9AE807000DF11C0B8BE87C
:10BE00000700F1EE410AC2209DED070A28F002FD6D
:10BE1000C3208DED070AB0EE491AF1EE490A9DEDF7
:10BE2000080A28F0F7FCB0EE681AF1EE680A8DED0A
:10BE3000080AC4209DED090A28F0ECFC514658463A
:10BE40008DED090A2BF022FE12A928468DED120A6B
:10BE5000CDED130A8DED141A06F57A662BF008F96C
:10BE600028462BF0FFF9DDED076A96ED007A2E4BA0
:10BE70009FED270AC6EE877A5846DDED086ACDEDBC
:10BE8000077AD3ED3E7A86EEA77ADDED096A8DED6D
:10BE9000087A86EEA77A8DED097A2BF061FEB9F16A
:10BEA000000F01D0CDED07AAB8F1000F01D08DED44
:10BEB00008AA0FB1CDED099AF0EE4B0A9DED070AE5
:10BEC0001A487CF057FF04205EF0BCFFF0EE4B0AEE
:10BED0009DED080A16487CF0A7FB13205EF0B2FF28
:10BEE0000021F0EE4B0A9DED090A12487DF064FB3B
:10BEF0002046FFF751FC84F8389084F8398084F8A4
:10BF00003A7017B0BDEC0C8BBDE8F08F35FA8E3C63
:10BF1000E02E654200A08C450000C84200000034BD
:10BF200000000000CDCC4C3E405C0020DC5B0020DB
:10BF3000345D00208C5E0020402C002010B50446AB
:10BF4000FFF73CFC0B4B93F97222022A0DD1B3F997
:10BF50007022002A09DD03F5805393F9623223B180
:10BF60002046BDE81040FFF70DBE2046BDE810405A
:10BF7000FFF718BD404C00200A207047004870476A
:10BF80002EFF0D08004870472EFF0D080120704756
:10BF9000012070470120704701207047034BD3F800
:10BFA0009C05031F58425841704700BF407C002049
:10BFB00070B505462D48D0F8642F00F624539A42F8
:10BFC00015D12B6993F844318BB100F5AE502EF0AA
:10BFD00005FB044658B95CF0D5F8254A032155F015
:10BFE000EBF82B69012283F84321204670BD214CD8
:10BFF00094F8B03223B194F968329A1E53425341F7
:10C000001D4E86F8583504F144030FCB04F1340576
:10C01000543485E80F0084E80F0006F5B8602FF06F
:10C0200053F9164B1C68E56A2B6828465B689847ED
:10C03000B0B195F84D309BB1E36A9B8F83B15CF052
:10C04000A1F8E36A0E4A9B8F062155F0B5F8E36A22
:10C0500006F5B860998F2EF023FFE36A00229A87D5
:10C0600008488AF041F80124BFE700BF406C002077
:10C0700014DA0D08408C0020407C00203C2C00206D
:10C080002EDA0D086856002038B50D4C94F8C435EA
:10C09000012B10D104F5B8602CF0FCF9B4F8FE5572
:10C0A0000848294605F004FD28B9152D03D104F6EA
:10C0B000747089F077F90023C4F8443538BD00BFA7
:10C0C000407C0020DC8D002008B511F0EBFD90F8DD
:10C0D0007C32DB0704D5BDE8084002482EF090BF53
:10C0E00008BD00BF0082002038B5344C94F8C43538
:10C0F000012B0ED0A4F545710822A4F5A0400BF049
:10C10000C1F95CF03FF8BDE838402D4A062155F0F2
:10C1100053B82C48B4F8FE5505F0EEFC20B1BDE84C
:10C120003840284808F01CBE162D05D0152D36D1F4
:10C13000D4F89C35072B0AD123480CF0C1FF2248C4
:10C140000DF006F9BDE838401F480DF01BB8A4F506
:10C15000A040F7F7E9FDA4F5A040F7F7C5FCA4F56A
:10C160004053D4F8B01593F9B02264235A4304F62F
:10C17000747089F073F8C4F8B00504F6747089F02F
:10C18000AFF930B1BDE838409FED100A46205EF0AF
:10C1900059BEA4F5A040BDE83840F7F789BA1E2D76
:10C1A00018BF4FF0FF33084818BFC4F81035F7F731
:10C1B000BBFD0548F7F798FC0348ECE7407C0020FE
:10C1C00048DA0D08DC8D0020402C00200000000023
:10C1D00070B5144890F968320E46154613B901241B
:10C1E000204670BDD0F860345B0312D5A0F58053B3
:10C1F00000F5CE70B3F8FE1504F002FF044640B916
:10C20000094B0A48006832462946C06A24F0B0FF4C
:10C21000E6E707482EF0E2F904460028DFD1054B97
:10C22000EFE700BF408C002074DA0D083C2C0020A2
:10C230000082002088DA0D0810B5144BB3F8FE35E3
:10C24000532B04461ED10AF029F99FED110A46200E
:10C250005EF0F8FD9FED0E0A49205EF0F3FD9FEDC4
:10C260000C0A4A205EF0EEFD46205EF0CBFE49202F
:10C270005EF0C8FE4A205EF0C5FE2046BDE81040D4
:10C28000FFF768BABDE81040FFF7A6B8407C002071
:10C2900000000000082070470048704714DB0D08BC
:10C2A0000048704720DB0D080120704708B50248A0
:10C2B000FDF79CFE012008BD402C0020014800F045
:10C2C0005FB900BF8478002010B50446FFF784F8FA
:10C2D0002046BDE81040FFF771BA0000012070470A
:10C2E0000048704798DB0D0800487047A0DB0D0838
:10C2F000012070470120704710B5044B03F154042E
:10C3000044330FCB84E80F00012010BD408C002087
:10C3100008B50B4800F5A04200F500530321D3F8FF
:10C32000803C93FBF1F3C2F8B035F7F741FC0448C9
:10C33000F7F7DAFBBDE808400148F7F7B9B900BFE5
:10C34000402C0020072070470048704711BD0D08A1
:10C350000048704718DC0D08012070470120704725
:10C36000012070477047000008B50023037743623F
:10C37000034889F0B9FE0348FBF73AFC012008BDE9
:10C3800068560020402C002010B5194CD4F8683CA9
:10C39000B3F9083023B9D4F8743CB3F90830F3B1D9
:10C3A000002303774362D4F8680C5DF0A5FA04F526
:10C3B0004863D3ED007A0F48F8EEE77A27EE800A5B
:10C3C000BDEEC00A10EE103AC0F8B035A0F5A0409E
:10C3D000F7F7EEFBBDE81040074803F015B8037F00
:10C3E000002BE0D0A4F50050F7F79EFCF2E700BF69
:10C3F000404C0020407C0020402C002070B54E4D69
:10C40000DFED4E7A95F8E4339FED4D7A2DED048BF8
:10C41000B02606FB035393ED788A9FED4A9A28EEE7
:10C42000278A05F5A653BDEEC88A93ED030AF8EEF8
:10C43000C87A044667EE897A97EE870A28F0D6F91B
:10C44000237FF0EE408A002B62D105F50053D3F82C
:10C45000683CB3F90830002B5AD1284609F054F84B
:10C46000002855D195F8E43395F8281406FB0353BA
:10C4700093F8C12100294BD1012A49D993ED777A4C
:10C48000F0EE087AB4EEE77AF1EE10FA40DBDFED79
:10C490002E7AB0EEE80AB4EEE70AF1EE10FA37D5DC
:10C4A000636A93B38CF072FE636AC01AB0F5FA7FC8
:10C4B00032D8237F002B3CD0244DA5F1200696E8EE
:10C4C0000F0085E80F0094ED088AA5F110013046B1
:10C4D000B8EEC88A17F032FD28EE098ADFED1C0A93
:10C4E000284670EE200AB0EE480A17F0CDFD194B31
:10C4F0009FED190AD3F84406BDEC048B03682A4665
:10C5000031469B6ABDE8704018478CF03FFE606280
:10C51000636A002BCDD0C5E7104D84ED088A012356
:10C5200023770023636205F110030FCB85E80F002A
:10C53000BFE7BDEC048B70BD402C00200000C8425A
:10C5400035FA8E3C0AD7233CDB0FC93F948C002080
:10C5500000007A44405C002000000000748C002041
:10C56000036A0B60007F70470520704700487047E2
:10C5700090DC0D0800487047A0DC0D0801207047D2
:10C5800038B54B4D2DED028BD5F8680C9FED498ADF
:10C590005DF0B2F9D5F8803C07EE903AF8EEE77A14
:10C5A00005F5405427EE800AA5F50050BDEEC00AFF
:10C5B00010EE103AC4F8B035F7F7FAFAD5F86C0C6B
:10C5C0005DF09AF9B5EEC00AF1EE10FADABF05F6A1
:10C5D0008443D3ED007AD5ED807A3748CBBF20EE87
:10C5E000270A20EE270A20EE080A28EE400ABDEEB0
:10C5F000C00A10EE103AC4F8B435F7F7A5FA95ED75
:10C60000807AD4F8B40505F6844327EE087AD3ED92
:10C61000007A27EE888AFDEEC77A17EE902AFDEEA3
:10C62000C87A17EE901A28F095F9C4F8B405224894
:10C63000FDF768FD20B1D4F8B4355B42C4F8B435D9
:10C640001E4B93F8743F63B195F95432022B08D115
:10C65000002301214620C4F8B035C4F8B4355EF09B
:10C6600055FF5DF059F85F215EF09EF8E8B15EF08D
:10C670006BF8022819D194F85535B3B904F5A563C0
:10C6800093ED007AD5EDA87AB4EEE77AF1EE10FAE0
:10C690000BD5012384F85535BDEC028B084A0948B7
:10C6A000BDE83840042154F087BDBDEC028B38BD95
:10C6B000404C00200000C842402C0020406C00206C
:10C6C000A8DC0D086860002010B50446FEF784FE63
:10C6D0002046BDE81040FFF771B800000620704703
:10C6E0000048704728DD0D080048704738DD0D0808
:10C6F00001207047012070470120704701207047DA
:10C700007047000008B5044889F0EEFC0348FBF7C9
:10C710006FFA012008BD00BF68560020402C0020A1
:10C7200038B50F4C04F50055D5F8680C5DF0E4F809
:10C7300004F53252D2ED007AF8EEE77A04F5A04320
:10C7400027EE800A2046BDEEC00A10EE102AC3F87C
:10C75000B025F7F72DFA2046BDE8384002F054BE68
:10C76000402C00200F20704700487047B0DD0D08B6
:10C7700000487047B8DD0D08012070470120704760
:10C780000120704701207047012070470120704749
:10C7900030B5184B2DED028B002283F8222403F5CF
:10C7A0004153043305460FCB85B06C4684E80F0037
:10C7B000114804F0E3FB90B1A86900F57F702AF0FE
:10C7C000DDFF0D48B0EE408A04F040FCF0EE400A78
:10C7D0009FED0A0A204628EE000A17F055FC0023B8
:10C7E0000748EB612146FBF7DDFD012005B0BDECFC
:10C7F000028B30BD405C0020DC8D0020E02E6542C5
:10C80000402C002038B5424C94F859354BB104F512
:10C81000805393F8B03223B1BDE838403D4808F06A
:10C8200071BAD4F87435002B18DC3B48F7F77CFA62
:10C83000D4F87835002B29DC3748F7F755F9374D10
:10C8400095F82234002B46D00121A5F5405009F07F
:10C850000DFABDE8384046205EF0F4BA8CF096FC44
:10C86000D4F87435C01A40F6B7339842DDD82C4D51
:10C87000D4F86805D5F8802C514228F06BF8C4F83C
:10C88000B005A5F50050F7F793F9D1E78CF07EFCE1
:10C89000D4F87835C01A40F6B7339842CCD8204B3C
:10C8A000DFED206A93ED807AD4F86C0503F68443BB
:10C8B000D3ED007A27EE267A67EEA67ABDEEC77A28
:10C8C000FDEEE77A17EE102A17EE901A28F042F8DC
:10C8D000C4F8B405B3E7A5F5805393F9DF31012B14
:10C8E00004DCBDE838400C48F6F7E2BED4F88435E5
:10C8F000002BF6D08CF04AFCD4F88435C01A40F6F0
:10C90000B7339842EDD805F5165595ED000AA0E726
:10C91000407C0020DC8D0020402C0020405C00206A
:10C92000404C00200000C842D0ED077A0348FCEEDE
:10C93000E77A17EE903A99B202F050BF402C0020EF
:10C9400084B010B503AC84E80E000B4821466F227A
:10C95000FBF776FC9DF80C1011F0040102D1204683
:10C9600017F054F804482146FBF71CFDBDE81040C1
:10C97000012004B0704700BF402C0020B0EEC00A78
:10C98000FDEEC07A38B54FF6FF7205460C4617EE3D
:10C99000900A002127F0DEFF07EE900A002CF8EE47
:10C9A000E77A044BC5ED077A14BF4FF0FF3201223E
:10C9B0001A7338BD408C0020FEF784BC0C207047F1
:10C9C0000048704791E00D08004870475E1B0F0853
:10C9D00008B50C48FCF716FA0A480B49FBF734F97E
:10C9E0000848F6F7D1FA40B106484FF48051F6F7FF
:10C9F00043F810B10348FBF7FBF8024802F0DEF9F8
:10CA0000012008BD402C0020948C002008B50D4862
:10CA1000F7F78AF90B48F6F7B7FA50B109484FF41F
:10CA20008051F6F729F820B1BDE80840054802F02A
:10CA3000EBBC0448F7F758F8BDE808400148F6F7A2
:10CA400037BE00BF402C002008B509484FF4805184
:10CA5000F6F712F828B107480022416E543016F05C
:10CA600011FFBDE808400248002102F0B7BE00BF38
:10CA7000402C0020408C0020881A10B527F092FE30
:10CA80000F4B9A680028B8BF4042002AB8BF5242F4
:10CA900048F6A041B2FBF1F24FF47A7102FB0111AA
:10CAA00088420BDC93F85420D20605D503F15404D8
:10CAB00044330FCB84E80F00012000E0002010BDBC
:10CAC000408C002013B504468069019100F57F7009
:10CAD0002AF054FEDFED0A7A20EE270A27F004FE42
:10CAE000DFED087A019920EE270A2046FDEEC07A94
:10CAF00017EE902A02B0BDE81040FFF7BDBF00BF9F
:10CB0000E02E65420000C84284B070B52DED048B64
:10CB100086B00FAD85E80E004D4CDFED4E8A06461F
:10CB2000D4F8440604F5405494ED080A0368B0EEC6
:10CB3000C00A5B6A9847B4EEE80AF1EE10FAB0EE6C
:10CB4000408A07DA012006B0BDEC048BBDE87040D6
:10CB500004B070474049284617F0FCF802A8CDED14
:10CB6000030A8DED020A2AF0D9FE04A88DED040A0D
:10CB7000B0EE480ACDED050A2AF08CFD13A928462F
:10CB80008DED000ACDED010A17F0E4F802A88DED55
:10CB9000020ACDED030A2AF03BFEB4EEE80AF1EEFC
:10CBA00010FACFDBB4EEC08AF1EE10FA9FED2B9AAB
:10CBB000DFED2B8ADFED2B9A2BD802A869462AF0ED
:10CBC00059FD04A88DED040ACDED050A2AF0D6FD25
:10CBD000684620EE098A2AF0D1FD94F90C3007EE60
:10CBE000903AF8EEE77A28EE288AA7EEA90A27F00D
:10CBF000FDFD20EE090ABDEEC88A20EE280A18EED7
:10CC0000101AFDEEC07A304617EE902AFFF734FF77
:10CC100099E738EE400A38EE088A80EE080AB4F048
:10CC200075F802A8B0EE408A2AF0A8FD94F90C30FD
:10CC3000F0EE007AB0EE697AA8EE677A07EE903AE5
:10CC4000F8EEE77AA7EE270A27F0D0FDC0E700BF8D
:10CC5000405C002000000034848C0020E02E6542FF
:10CC60000000C842DB0FC93F10B504460848F6F77C
:10CC70008BF920B92046BDE81040FEF723BB0448DD
:10CC80004FF48051F5F7F8FE0028F3D010BD00BF37
:10CC9000402C00200020704700487047A0DE0D089F
:10CCA00000487047A8DE0D0800207047036993F81C
:10CCB000140118B1D3F8C402C0F38010704700000B
:10CCC00038B5154C05460021204608F0FBFD042030
:10CCD0005EF0B8F80021204608F0FEFD13205EF05B
:10CCE000B1F80021204608F001FE2846FEF754FD69
:10CCF0002046012108F0BAFF46205EF0A3F8AB6998
:10CD000004F5A044D3F8F831C4F8B035AB69D3F8D2
:10CD1000FC31C4F8B43538BD402C0020FEF71ABDF4
:10CD2000172070470048704720DF0D080048704703
:10CD300028DF0D080120704701207047012070474F
:10CD400010B50369002283F8402103690446D3F833
:10CD50003C0103689B689847A368186882F088FDC7
:10CD6000206904F083FE0349A06910F081FD0120D1
:10CD700010BD00BF707800201FB50D4C9FED0D0A4F
:10CD800004F5C04304F5A044D3F8D0016C302AF078
:10CD900093FEFDEEE00ABDEEC00A10EE903AC4F834
:10CDA000B43510EE103AC4F8B03504B010BD00BF71
:10CDB000402C00209F0CB34530B52DED028B83B085
:10CDC00004468CF0E3F90146206900F50E700BF083
:10CDD0009FF938B1204603B0BDEC028BBDE830406E
:10CDE000FEF7FABA206990F84031BBB1012104F096
:10CDF000C3FDA368DFED400A1868036801215B6E7C
:10CE0000B0EE600A9847206903F016FA3B4803B079
:10CE1000BDEC028BBDE83040FFF790B8384DDFED38
:10CE2000398A022104F0A8FDD5F86C0C5CF064FD91
:10CE30002369D3ED390A93F93C2220EE200A002A17
:10CE400060EE280A3FDD93F8A032002B3BD0D5F8E6
:10CE5000740CCDED000A5CF04FFD2369D5F8680C29
:10CE600093ED3A8A20EE080A20EE288A5CF044FD11
:10CE7000236993ED381A20EE410A20EE281ADDEDE1
:10CE8000000A2069CDED010A8DED001A03F010FAB9
:10CE9000A36895F9722218689DED001ADDED010A6C
:10CEA0000368F0EE408A2AB31B6CB0EE480A98473C
:10CEB000A36818680368F2EE040A5B6E0021B0EE06
:10CEC000680A9847A2E7D5F8680CCDED000A5CF037
:10CED00013FD2369D5F8740C93ED388A20EE080A07
:10CEE00020EE288A5CF008FD236993ED3A1A20EEC3
:10CEF000010AC2E7DB6BD8E7000000004878002099
:10CF0000404C00200000C842122070470048704783
:10CF1000A0DF0D0800487047A8DF0D08012070470A
:10CF2000012070470120704738B52DED028B436812
:10CF30009FED1C8A1D680446006904F0BDF9236951
:10CF400093ED131AD3ED110A434200EE103A21EE8D
:10CF5000081A60EE880AB8EEC00A284683F042FE3E
:10CF6000636820691D6804F0A7F9236993ED131A1B
:10CF7000D3ED110A434200EE103A21EE081A60EE9A
:10CF8000880AB8EEC00A284683F0A6FE9FED060A7E
:10CF9000206903F07DF9206905F022FFBDEC028BCA
:10CFA000012038BD0000C84200000000014800F028
:10CFB00073BE00BFBC79002013B5044600698830F9
:10CFC000FAF7CCF88CF0E2F80146206900F50E7013
:10CFD0000BF09EF828B1204602B0BDE81040FEF7E5
:10CFE000FBB9206990F840313BB3012104F0C4FC47
:10CFF000A368DFED170A18680368B0EE600A5B6E7D
:10D0000001219847206903F017F963689FED100A22
:10D01000186885F011F80F48F6F796F80D48F6F7FE
:10D020008DF920469FED0A0AFEF7B6FB206988308D
:10D0300002B0BDE81040FAF74FB9074804F000FE0F
:10D040002069019004F09EF9019806F0D5FAE2E714
:10D0500000000000402C0020DC8D002014207047D0
:10D060000048704726D90D0800487047711B0F080B
:10D07000012070470020704770B504460E4800F04C
:10D080003BF82369002583F84051206904F0B6FF7E
:10D090006069052103F072FD084826690221FAF74C
:10D0A00053FC86EDB70A2369C3F848512369C3F8D6
:10D0B0004C51012070BD00BFF4790020402C0020AD
:10D0C000014800F0E9BD00BFBC790020014800F034
:10D0D00069B800BFF47900201320704700487047FA
:10D0E00090E00D080048704798E00D080120704757
:10D0F000012070470120704738B52DED028BDFED20
:10D10000240AC3689FED238A0446B0EE600A1868BB
:10D110007FF030FFE368186880F00AF863682069E0
:10D120001D6804F0C9F8236993ED131AD3ED110AB1
:10D13000434200EE103A21EE081A60EE880AB8EE7B
:10D14000C00A284683F04EFD636820691D6804F01C
:10D15000B3F8236993ED131AD3ED110A434200EE9D
:10D16000103A21EE081A60EE880AB8EEC00A284686
:10D1700083F0B2FD206905F033FE25698CF006F8D6
:10D18000C5F86C01BDEC028B00230120E36138BDC2
:10D19000000000000000C842014800F07DBD00BF53
:10D1A000BC79002030B52DED048B0446006985B0B4
:10D1B0008830F9F7D3FF38B1B64805B0BDEC048B21
:10D1C000BDE83040FFF7F8BE8BF0E0FF0546206970
:10D1D000294600F50E700AF09BFF38B1204605B0D5
:10D1E000BDEC048BBDE83040FEF7F6B8206990F83E
:10D1F000403163B3012104F0BFFBA368DFEDA60A51
:10D20000186803680121B0EE600A5B6E98472069D8
:10D2100003F012F863689FEDA00A186884F00CFF11
:10D22000DFED9D0AE368B0EE600A18687FF0A2FEA9
:10D23000E36818687FF07CFF9848F5F785FF97480A
:10D2400005B0BDEC048BBDE83040F6F777B8C36A93
:10D2500093F8CB3013B99248FFF74EFF206903F0E3
:10D2600051F918B1E36818687FF080FE2369D3F89C
:10D270006C31EB1AB3F5FA7F0BD9E368DFED860A60
:10D280001868B0EE600A7FF075FEE36818687FF0FA
:10D290004FFF23699FED838AC3F86C5102212069F7
:10D2A00004F06AFB636820691D6804F005F82369CF
:10D2B00093ED131AD3ED110A434200EE103A21EE1A
:10D2C000081A60EE880A2846B8EEC00A83F08AFC85
:10D2D000D4E9033518687FF0B7FEA36818680368BF
:10D2E0009B6EF0EE408A984703AAF0EE400A02A92E
:10D2F000B0EE680A284603F01FF8E368DDED030A84
:10D3000018689DED020A7FF035FE6368186883F0A7
:10D310005BFC18B96368186884F04CFBE368624DE5
:10D320001868012180F070F8E36860481B689B680A
:10D33000D3EDCF7AFDEEE77A17EE903AC5F8B03527
:10D34000E3681B689B68D3EDD07AFDEEE77A17EEB1
:10D35000903AC5F8B43504F073FC2369D3F83C0166
:10D36000036805F2B4525B6B05F5B661984748B1A6
:10D3700063681B68D3F88823C3F89423D3F88C23FD
:10D38000C3F898232069DFED4A9A04F069FBD5F8C9
:10D39000B035206907EE903A012105F2B453F8EE5A
:10D3A000E78A93ED009A06F0C1F8A368B8EEC99A2F
:10D3B000186820EE290A036868EEA98A29EE299ADE
:10D3C000DB6A20EE081A69EE080A28EE880A9847F8
:10D3D000384BD3F8602F03F6D4518A4248D16369A1
:10D3E00093F86430062B0AD8206903F0D9FC30B1D9
:10D3F0006069072103F0C2FB206904F0FFFD2748A4
:10D400000221FAF7A1FA206903F0A8F8636993F8FA
:10D410006430072BB0EE408A08D12369D3F8C432B8
:10D420009B0403D4A069012110F0E8FE6368B5EE07
:10D43000C08AF1EE10FA1868CCBF01210021B1EECC
:10D44000480A83F055FC206907F0EAFD206903F0E3
:10D4500051FF1248F5F778FE1048F5F76FFF9FED82
:10D460000E0A2046FEF798F905B0BDEC048B30BDDE
:10D4700003F624539A42206907D190F8423123B130
:10D480009FED050A02F004FFE0E7019003F07AFF48
:10D490000198F7E7D879002000000000402C002018
:10D4A000F47900200000C842407C0020DC8D002080
:10D4B0000AD7233C406C0020152070470048704775
:10D4C00010E10D080048704710E10D080120704779
:10D4D0000120704700207047C369012B06D1044B1F
:10D4E00093F87003431E584258417047002070471C
:10D4F000408C00200E4BB3F91222B3F9443207EEF0
:10D50000102A07EE903AB8EEC77AF8EEE77AB0EE56
:10D51000C77AF0EEE77AB4EE677AF1EE10FAC8BF98
:10D52000F0EE477AB7EE080A27EE800A704700BF90
:10D53000404C00202DE9F043844D2DED048B95F8EF
:10D54000E0928BB00446B9F1000F0BD08049312234
:10D55000A5F5C04009F096FF01200BB0BDEC048B8F
:10D56000BDE8F0830123C36105F1440696E80F008E
:10D5700005F1340787E80F0023692A6BB3F8C07000
:10D58000DB6A526893F8A0306421022B17FB012755
:10D5900040F0B68007EE907A3246B8EEE70AA5F57D
:10D5A000C04106A8FBF712F806A9304616F0C6FCE3
:10D5B0002046F0EE408AFFF79DFF2369B3F9C020B3
:10D5C000D3ED310A01EE102AB3F9C220B0EE409A31
:10D5D00000EE102AB8EEC11A1A20B8EEC00A27F0E1
:10D5E00019F92369B3F9C030F4EEC98A07EE903A0D
:10D5F000F1EE10FA54BFF0EE686AF0EE496AB8EE48
:10D60000E77AC8EEA67A236820465B68B0EE408AC7
:10D6100067EE877AB4EE670AF1EE10FA48BFB0EE13
:10D62000678A98470146A5F5C040FAF7B5FA082180
:10D6300002468046A5F5C040FAF738F9DFED457A95
:10D6400038EE408AB4EEE78AF1EE10FA31DBC4F826
:10D650001C9096E80F0005F1540484E80F009FED3C
:10D660003E9AB8F1000F14D005AA0321304616F0F7
:10D670003FF970B1DDED057AF8EEE77A0322E8EEC6
:10D68000097A2046FDEEE77A17EE901A16F0FAF8BE
:10D6900062E7D5ED128A3148F8EEE88A16F01CF9F7
:10D6A000E8EE098A02462E48FDEEE87A17EE901A57
:10D6B000ECE7F4EEC98AF1EE10FA21D505AA494645
:10D6C000304616F015F918B1059B9F42A8BF1F46BA
:10D6D0005AF058FD064619EE100AF2F715FFCDE98B
:10D6E000020118EE900AF2F70FFF1E4ACDE9000181
:10D6F0000621304653F060FD6069032103F03EFAD5
:10D7000039461948FAF71AFF206903F0BFFC13489D
:10D7100005AA002116F0ECF868B96269AB6CA96D36
:10D720008B4292F82010D4BF0023012363F3000141
:10D7300082F8201010E70A4806AA002116F0D8F84F
:10D740000028EAD0DDE905316269E9E7408C002074
:10D75000147A0020000000340000C842848C0020AD
:10D76000948C002018E10D08402C0020014800F0A6
:10D7700093BA00BFBC790020F0B52DED028B99B0B3
:10D7800004468BF003FD0146206900F50E700AF097
:10D79000BFFC054638B1204619B0BDEC028BBDE890
:10D7A000F040FDF719BEE36983B1012B00F01E8143
:10D7B0009F48F5F7C9FC9E48F5F7C0FD9C4819B095
:10D7C000BDEC028BBDE8F040F6F71EB99FED998ADB
:10D7D00060688DED098A8DED0A8A8DED0B8A8DEDDD
:10D7E0000C8A0BAA09A901230068934D83F010F954
:10D7F0002069B0EE480A03F00BF963688F481B6894
:10D80000D3EDCF7AFDEEE77A17EE903AC5F8B03552
:10D8100063681B68D3EDD07AFDEEE77A17EE903A95
:10D82000C5F8B43504F00CFA2369D3F83C01036859
:10D8300005F2B4525B6B05F5B661984748B1636871
:10D840001B68D3F88823C3F89423D3F88C23C3F838
:10D850009823206904F00AF9A36820691E683368D8
:10D86000DF6AD5F8B03507EE903A05F2B453D3ED40
:10D87000000AF8EEE00AF8EEE78ACDED050A05F0B9
:10D88000C9F8DDED050AB0EE401A3046B0EE680A80
:10D89000B8472069C36B93ED070A02F0F9FC2069D1
:10D8A00003F028FD63688DED0D8A8DED0E8A8DEDF8
:10D8B0000F8A18680FA983F0FDFB0D9B14930E9B34
:10D8C000159302220F9B169314A910A816F0ACFB17
:10D8D0005B4907AA10A816F0BDF848B1DFED597AE8
:10D8E0009DED077AB4EEE77AF1EE10FAFFF660AF3D
:10D8F000554D0123E36105F1440797E80F0005F159
:10D90000340686E80F002B6B22695B68B2F8C060B2
:10D91000642216FB023607EE906A3A46B8EEE70A32
:10D92000A5F5C04114A8FAF751FE384614A916F01F
:10D9300005FB2046B0EE408AFFF7DCFDB4EEC08A5E
:10D94000F1EE10FAF0EE408A22D508AA002105F186
:10D95000540015F0CDFF18B1089B9E42A8BF1E468B
:10D960005AF010FC074618EE900AF2F7CDFDCDE90B
:10D97000020118EE100AF2F7C7FD344ACDE90001A2
:10D980000621384653F018FC6069032103F0F6F8CD
:10D9900031462748FAF7D2FD206903F077FB284982
:10D9A00007AAA1F1100016F055F8636988B19DED42
:10D9B000077ADFED247A93F82020B4EEE77AF1EECF
:10D9C00010FAACBF0121002161F3000283F820208E
:10D9D000EEE6AA6CA96D8A4293F82010D4BF00220B
:10D9E000012262F3000183F82010E1E6206906F0CD
:10D9F0006DF8636993F86430042B06D91248036B01
:10DA00002A465968543015F03DFF636993F8643035
:10DA1000032B02D9206907F043FB236993F8D43123
:10DA2000013B012B3FF6C4AE0148F5F7C7FCBFE64A
:10DA3000402C002000000000407C0020DC8D0020F5
:10DA4000948C002000000034408C002018E10D0868
:10DA500030B5C369012B85B004D1404C94F87033C4
:10DA6000012B04D005B0BDE83040FDF72BBCA4F578
:10DA70008043DFED3B6AB3F912229FED3A0A07EECD
:10DA8000102AB3F9442207EE902AB8EEC77AF8EECE
:10DA9000E77AB4F95C22B0EEC77AF0EEE77AB4EE3A
:10DAA000677A00EE902AF1EE10FAC8BFF0EE477ADE
:10DAB000B8EEE07AD3EDA00A03F6485270EEC70A3A
:10DAC00092ED007A27EE267AF5EEC00AF7EE006AAC
:10DAD000F1EE10FAB4EEE67A48BFDFED220AF1EE7D
:10DAE00010FAD8BFB0EE667AF3EE046A77EEA71AA2
:10DAF00067EEA67AC0EE876A54346D4693ED7B7A62
:10DB0000194BB0EE612AA6EE872A93ED001AF4EEC7
:10DB1000427AF1EE10FA48BFB0EE672AF4EE421AEC
:10DB2000F1EE10FAC8BFB0EE612A26F0A5FD94E828
:10DB30000F0007EE901A9FED0D7AF8EEE77A85E870
:10DB40000F00E0EE077A0A482946FDEEE77ACDEDB0
:10DB5000017AFAF78BF805B030BD00BF408C002089
:10DB60009A99193F00000000788100200000C84207
:10DB7000402C00201120704700487047A8E10D0894
:10DB800000487047B4E10D0801207047012070473C
:10DB900001207047012070470369002283F840216B
:10DBA00001207047184B1949D3F8D80203F20442F8
:10DBB00092ED007AB3F9A421B5EEC07AF1EE10FA35
:10DBC00007EE902AC8BFDFED126AF8EEE77ACABF07
:10DBD00027EE267A20EE270A27EE000A67EEA07AC3
:10DBE000BDEEC00AFDEEE77A10EE102AC1F8B025AE
:10DBF00017EE902AC1F8B425036801F2B4525B6BAA
:10DC000001F5B661184700BF408C0020407C002021
:10DC10000000C8421E4BDFED1F6AB3F9A411A3F543
:10DC20008050A3F58043F5EEC00AD3F8802C8A42D9
:10DC3000A8BF0A4607EE902AF1EE10FAF8EEE77A4E
:10DC4000D6BF03F6844393ED807A93ED007A27EEF6
:10DC5000800A07EE901ACCBF27EE267A27EE667A66
:10DC6000F8EEE77ABDEEC00AB4EEE77AF1EE10FA0C
:10DC700058BFB0EE677A60EE870A10EE102AFDEE0C
:10DC8000E00AC0F8B02510EE903AC0F8B4357047FD
:10DC9000408C00200000C84237B52C4CD4F8683CBA
:10DCA000B3F908201B8B07EE102A07EE903AD4F840
:10DCB0006C3CB8EEC77AB3F908201B8BF8EEE77A14
:10DCC000054687EE270A224807EE102A07EE903A0B
:10DCD000B8EEC77AF8EEE77A8DED010AC7EE270AAB
:10DCE000CDED000A09F0C4FFDDED000A9DED010A4B
:10DCF00028B1284603B0BDE83040FFF753BF04F514
:10DD00008043D3F86024520405D4284603B0BDE80C
:10DD10003040FFF77FBFB3F9A43107EE903AF8EE39
:10DD2000E77A04F5405427EE800A67EEA00ABDEEBC
:10DD3000C00AFDEEE00A10EE103AC4F8B03510EE5D
:10DD4000903AC4F8B43503B030BD00BF404C002059
:10DD50001490002010B504468BF018FA0146206993
:10DD600000F50E700AF0D4F920B12046BDE810404D
:10DD7000FDF732BB114803F063FF206990F9D03002
:10DD80004BB102F01FFA0E48F5F7DEF9BDE810407E
:10DD90000B48F5F7D3BA02F08BFA206905F0E6FBE1
:10DDA0000748F5F7D1F90648F5F7C8FA20469FED80
:10DDB000050ABDE81040FDF7EFBC00BFDC8D002078
:10DDC000402C0020000000000B20704700487047E6
:10DDD000CEE40D08004870472CE20D080120704782
:10DDE00001207047012070470020704738B52F4848
:10DDF000F5F79AFF2D48F5F777FE2C48F5F758FC14
:10DE00002A481021F4F738FED0B1294A936C926D5C
:10DE10009342D4BF00230123254C94F8C82072B943
:10DE200063B304F144030FCB04F1340585E80F001C
:10DE3000A4F5C040F9F78CFC012384F8C83038BD44
:10DE40001C4AB2F94C1C0029F9DD02F580429FED15
:10DE50001A7A936C926B9B1A07EE903AF8EEE77A77
:10DE600067EE877A07EE101AB8EEC77AF4EEC77A33
:10DE7000F1EE10FACCBF01230023CDE7A4F58043D7
:10DE8000642193F9B02212FB01F2D3F8801CA4F5AF
:10DE900080548A42A8BF0A46D4F8B005C3F8802C43
:10DEA000514226F057FDC4F8B005C8E7402C0020C9
:10DEB000408C0020404C00200AD7233CF0B52F4C6A
:10DEC0002DED028B04F14405074695E80F0004F19F
:10DED000340686E80F0083B0A4F5C040F9F732FAA3
:10DEE0000146A4F5C040FAF729FBA4F5005200232F
:10DEF00084F8C830C2F8883F94F8B032C3B394F8BD
:10DF0000E0323BB13122A6F59351A4F5C04009F0AF
:10DF1000B9FA2DE094F96A32032B02D118492C2268
:10DF2000F3E7013BDBB2012B22D83B69DB6A93F8B4
:10DF3000A030022B1CD104F15401284615F0FEFF3D
:10DF40000F48B0EE408AFFF7D5FAB4EEC08AF1EE82
:10DF500010FA0DD501AA0121284615F0C9FC38B1E7
:10DF6000B4F85C32642213FB02F3019A9342D5DCCD
:10DF7000012003B0BDEC028BF0BD00BF408C00203F
:10DF8000307A002010B52DED028B244B93F96A22D4
:10DF9000012A03D00020BDEC028B10BDA3F5804305
:10DFA000B3F94442002CB8BF6442A4B22CB9B3F90F
:10DFB0001242002CB8BF6442A4B2194BD3F84406F5
:10DFC00003689B6B984730B116491748272209F020
:10DFD00059FA0120DFE7154AA2F1200101F11000F2
:10DFE00015F018FF0028EFD1114B03F6644093EDB4
:10DFF000008A03F02BF807EE904AF8EEE77AB4EEC9
:10E00000E70AF1EE10FA44BF07EE904AB8EE670A4D
:10E01000B4EEC08AF1EE10FABCD5D5E7408C0020F2
:10E02000405C0020307A0020402C0020948C00209E
:10E030007881002070B5474C94F8B03288B005461E
:10E040008BBB454DB5F9443283EAE371A1EBE37133
:10E0500089B2002956D1414C414801F0BFFB94F8E8
:10E060005635002B3ED195F91F32022B51D13D4D33
:10E0700095F8913F9BB13C4905F5AE502DF038F92C
:10E0800068B10123282205F54C61A5F5804084F88C
:10E09000F93509F0F7F928BB002384F8F935012395
:10E0A00084F856351EE094F96A32022BA4F5005626
:10E0B0001AD103AD284615F0DFFB04F154030FCB52
:10E0C00085E80F0001A9A4F5C040FBF74DF9D6F88B
:10E0D000883F052B06D1272206F55F61A4F5C040D5
:10E0E00009F0D0F908B070BD8BF050F8D6F8683F51
:10E0F000C01AB0F57A7FA4D92846FFF743FF00285D
:10E100009FD0EFE7002BB4BF4FF0FF330123237301
:10E11000A1E7012B0ED1A4F5A04001F077FA48B198
:10E12000A4F5A040F9F7D2FA0028B8BF4042B0F5F4
:10E130007A7F9CDB95F91F32042BD3D1094D95F8DA
:10E14000913F002BABD0084905F5AE502DF04CF9AE
:10E1500096E700BF408C0020404C0020407C00200F
:10E16000402C0020406C0020848C0020022070474E
:10E1700000487047A9E10D0800487047581B0F0878
:10E18000034B0022C3F8B025C3F8B425704700BF85
:10E19000407C002038B5094D04462846F4F7D4FFEA
:10E1A0002846F5F7CBF82046F5F7E0F82846F5F7CE
:10E1B0002BFC2046BDE83840FDF700BB402C00207A
:10E1C0000D2070470048704714E30D080048704761
:10E1D0001CE30D08012070470120704701207047A3
:10E1E000002380F8273080F8383001207047000085
:10E1F0000148002101F0F2BA402C00202DE9F04145
:10E20000B54CD4E913322DED088B1343A26C1343A4
:10E2100088B005460FD1B148F5F786FDAF48F5F750
:10E2200063FC9FEDAF0A462008B0BDEC088BBDE84B
:10E23000F0415CF007BE0FF035FD90F87C32DB0753
:10E24000E9D5B5F91C3095F8271009EE103AB5F963
:10E25000243008EE903AB8EEC99AF8EEE88AA4F5B0
:10E260008056002940F0D9809FED9EAA29EE0ABA77
:10E270000122FDEECB7AA4F5C04017EE903AC6F825
:10E280002035F9F713FBA86900F57F700790B0EE11
:10E29000408A29F073FADFED947A20EE270A26F0FF
:10E2A00023FA0798F0EE409A29F0B2FAA4F5C0409C
:10E2B000F0EE40AAFCF7F0FC002879D104F1440705
:10E2C00097E80F0005F1280C8CE80F0097E80F0085
:10E2D00004F1340C8CE80F0004F1540C8CE80F00AE
:10E2E000D4ED167A8148F8EEE77AF0EE680A77EE18
:10E2F0008B7AB0EE690AFDEEE77AC4ED167A15F076
:10E30000C3FE002386F8893595F92630734803EB60
:10E31000830303EB83039B000121A6F84E35F4F73A
:10E320003FF896F89885B8F1000F76D1704B9FEDC5
:10E33000717AB3F9E83107EE903AF8EEE77A67EED2
:10E34000877AF4EEE7AAF1EE10FA66DD59F01AFFCB
